S00C000068616D64722E68657874
S31A00030000373B00F037B50003379C37BCD55037B50000379D37AF
S31A00030015BD0200C500DA003C013D01377D2B34B6EE15003D01EA
S31A0003002AB6F6F5FF379D37BD000015003D01377D0400B6F23766
S31A0003003FB5000027FA379C379D379E379F37BFFFFE37BE000093
S30F00030054FA03944C277B7A0301CECE
S31A0003005E3460373B00E0371527FA379C37BC000837B502008AEB
S31A00030073003C02377C0070B6F237B502088A003C02377C0200F3
S31A00030088B6F237B5021037FA000837B5021837FA000A37B5024C
S31A0003009D2037FA000C37B5022837FA000E37B5023037FA001034
S31A000300B237B5023837FA001E37B5024037FA002237B5024837CD
S31A000300C7FA002437B5025037FA002637B5025837FA002837B5DD
S31A000300DC026037FA002A37B5026837FA002C37B5027037FA0007
S31A000300F12E37B5027837FA0030350327F7373B00E037B5000365
S31A00030106379CF5FF27FA37B5000C37FAFC0AF50A3A01FC0CFF83
S31A0003011BFA17FAFC0FF50D3A01FC0CFFFA17FAFC0FC500B70AD0
S31A000301303A01FC0CFFFA17FAFC0F3C01B0EAF5203A01FC0CFF2B
S31A00030145FA17FAFC0F3540F60FF80AB5FEF107F1303A01FC0CFB
S31A0003015AFFFA17FAFC0F352027FB371A371F371F371F371FF65C
S31A0003016F0FF80AB5FEF107F1303A01FC0CFFFA17FAFC0F27FB1B
S31A00030184371AF60FF80AB5FEF107F1303A01FC0CFFFA17FAFCF0
S31A000301990F27FB371F371F371F371FF60FF80AB5FEF107F130EC
S31A000301AE3A01FC0CFFFA17FAFC0F27FBF60FF80AB5FEF107F116
S31A000301C3303A01FC0CFFFA17FAFC0F373B00E0371527FA17FCC4
S30B000301D800024B020000C9
S31A000301DE3460373B00E0371527FA37B5028037FA00A4F5FF2752
S31A000301F3FA37B5025237FAFA2237B5000837FAFA2437B5040034
S31A0003020837FA010E350327F7374C3420F5FF27FA277101003786
S31A0003021D4A00008A02350227F7374C373503E83725374A0000E1
S31A00030232B002374C270500008A023420F5FF27FA27710100813E
S31A00030247028A0237430000374A0000350227F7374C3420F5FFF0
S31A0003025C27FA27710100800237420000B702277527F527F03512
S31A000302710227F73423274FF5FF27FA27710100800437420002D5
S31A00030286277027F52774371C35023F0427F73420F5FF27FA3781
S31A0003029B71010237780102BAF6350227F73420F5FF27FA37F585
S31A000302B00104350227F73420F5FF27FA37B5000137FA01083511
S31A000302C50227F73420F5FF27FA27310108350227F73420F5FF94
S31A000302DA27FA27330108350227F73420F5FF27FA37350400272D
S31A000302EFF52773010E350227F73460F5FF27FA373B004037F577
S31A00030304011027350110350327F6B6FE27F717F10887730037F5
S31A00030319B8003CB55C277B17F508863713F83CB54017F5088579
S31A0003032E3713F818B53017F508843713364C371BB41E17F508D6
S31A00030343833713F80DB50E17F508823713F864B5FE371517FABB
S31A000303580882F50117FA0883F50117FA0884371517FA088537B7
S31A0003036D1517FA08863730003C3738003CB4A027FB17FA08875A
S31A00030382277108842773318827F7177508837802B70678087387
S31800030397FF7601711E27F71775088276037001731C27F77A
S31A000303AA377A2C0037B505E237FA008A27F727352C0837B5121E
S31A000303BFC037FA2C0037B5057637FA008A27F7377A2C0837B5F2
S31A000303D4807E37FA2C0637B5058C37FA008A27F737B5057637B6
S31A000303E9F0008A27F73460373B00E0371527FA37B503E437FA07
S31A000303FE008A27352C1227352C10F5FF27FA2735011627350140
S31A000304131837B5000137FA010637B5040C37FA011237B50070F2
S30D0003042837FAF70C350327F739
S31A000304303420371527FA37B506C437FA0094F5FF27FA37B54031
S31A000304450037FAF90C3920F921350227F73420F5FF27FA277695
S31A0003045AB708374C27710100374A00008A023775012117750141
S31A0003046F2317F5F90D17780123B6EA37780121B6E4350227F727
S31A000304847C023442277B27F73402351035608E008F02374A00F6
S31A00030499048A06340327F527F73402351034013508CE00CF02B4
S31A000304AE37450004850634033408354027F7274FCC0437283743
S31A000304C3CC275FDD06B7FE9C0027F7372527F7277A274FCC0416
S31A000304D8372A275C277A274FCC04372837CC375C275FDD06B726
S31A000304EDFE9C0027F7274F37DC8504372537DC374500043725DC
S31A0003050237DC277837DC27F7274FCC043725372837CC27F727AF
S31A00030517F6B726375C37CC375500009502377C0008B508370586
S31A0003052CD500277B95013CF8B704277F27FE3CFFB6F4375A0074
S31A00030541009A0227F727F6B714375C37CC37550000950227F426
S31A00030556277C3CFFB6F4375A00009A0227F7F5FF3420379C8514
S31A0003056B00350227F734023510F500B0EA34023510F502B0E20F
S31A0003058034023510B0DA37BCFC14B0D437BCF90CB0CE37BCF771
S31A0003059512B0C837BCF732B0C237BCF736B0BC37BCF73AB0B61A
S31A000305AA37BCF73EB0B036F4372527FB27F73420F5FF27FA2755
S31A000305BFF53A02F9070002F7013A10FC150002F7023A40FC1512
S31A000305D4000277013A20FC1500027702350227F73420F5FF27E5
S31A000305E9FA17F5FC153705F640350227F73420F5FF27FA17F5A1
S31A000305FEFC153705F620350227F73420F5FF27FA17F5FC15376A
S31A0003061305F610350227F73420F5FF27FA2776B7043940F9072F
S31A00030628350227F73840F907350227F73420F5FF27FA2776B7D5
S31A0003063D043904F907350227F73804F907350227F73420F5FF30
S31A0003065227FA2776B7043980F907350227F73880F907350227ED
S31A00030667F73420F5FF27FA2776B7043908F907350227F73808E7
S31A0003067CF907350227F73420F5FF27FA2776B7043910F90735CC
S31A000306910227F73810F907350227F73420F5FF27FA2776B704CD
S31A000306A63901FA41350227F73801FA41350227F73420F5FF2734
S31A000306BBFA2776B7043902FA41350227F73802FA41350227F73A
S31A000306D03420F5FF27FA2776B70C37B501F437FA010C3904FAED
S31A000306E541350227F73804FA41350227F73420F5FF27FA277F86
S31A000306FAB5023808FA41B0003908FA41277FB5023810FA41B0F4
S31A0003070F003910FA41277FB5023820FA41B0003920FA413502DD
S31A0003072427F7274FCC04B720374C37DC45003C013717370F3799
S31A000307390F370F370F71305A00F60FF130DA013D023730000263
S31A0003074EB2DC27F7374C37DC4500371737B60FF0277B371F379D
S31A0003076307371F371F370B277827FB4A003C013DFFB6DC27F74F
S31A00030778374C8500371A27F7374C8502371A277B8500371A27F2
S31A0003078DF734103FF8276F363037650000A5023F08350427F7FF
S31A000307A234103FF8276F361C37650001A5033F08350427F734BF
S31A000307B7103FF8276F360837650002A5043F08350427F7374CA1
S31A000307CC37DC9502374500023725AA06376A0004950037450025
S31A000307E1003725AA02376A000095023745000037253604950013
S31A000307F6374500023725A104AA0437630002376A0002B400279E
S31A0003080B23000027F727FB277E371E27F727FBF180371C27F750
S31A0003082027FB3401274FC400CA00371F371F371F371FC400CA79
S31A0003083500371F371FC400CA00371FC400F6013F0227F73410B7
S31A0003084A3FFC276F375C37CC271500022715000027250000C59E
S31A0003085F00F820B6003C01B0F2F82DB6FE3C01AA02C500F03027
S31A00030874B52AF809B226EA0195023755000027F4277C27F427A0
S31A000308897C91023753000027F4277CA100373300009A02375AC2
S31A0003089E00003C01B0C8A502F82DB60C27F52775900237520026
S31A000308B3009A02375A00003F04350427F7374CC500F030750A79
S31A000308C83724C101F03027F7374CC500F03075643724277BC5B4
S31A000308DD01F030750A37242778C502F0303705277827FB27F761
S31A000308F2375C37BC000A372AF130DA0137CCF130DA0027F737A8
S31A000309075C37BC000A372AF130DA0237CC37BC000A372AF13099
S31A0003091CDA0137CCF130DA0027F7375C37BC000A372AF130DADA
S31A000309310437CC37BC000A372AF130DA0337CC37BC000A372AE4
S31A00030946F130DA0237CC37BC000A372AF130DA0137CCF130DA3B
S31A0003095B0027F73B9ACA0005F5E10000989680000F42400001A6
S31A0003097086A000002710000003E8000000640000000A34303718
S31A000309855C37EC37B50003379C37BC095E37650000A50237BE81
S31A0003099A002F3E01800237420000B4F281023743000037ECDA36
S31A000309AF003D0137EC3C04377C0982B5D8F130DA001501350672
S307000309C427F70A
S31A000309C63410276F37753500FA0305B037F834F2B522173673BA
S31A000309DBBEB744373573B837B5000AFA031AF23716B73417352B
S31A000309F073BE37B5000237FA73BCF501B020173673BEB61E371B
S31A00030A053573B837B5000AFA031AF23716B70EF50117FA73BE2A
S31A00030A1A37B5000137FA73BC17FA72B5350427F73410276F37D1
S31A00030A2F7572D037380001B700FA0302F8273634F2B700FA039D
S31A00030A4409C6FA03C854350427F734103FFE276F37380067B6B2
S31A00030A5906FA03C25A37057A030AFC37380077B606FA03C27AC6
S31A00030A6E37057A030AFC37380076B616FA03C2B4277B37BD01F0
S31A00030A8368AD0037B50100FA03050A37057A030AFC37380068B1
S31A00030A98B606FA03C30E37057A030AFC37380040B3087CBFFA58
S31A00030AAD03AEB437057A030AFC7CD0277F37380001B716B50A19
S31A00030AC237380002B71837380003B71CB026FA0305983717379C
S31A00030AD705B01EFA03059E37173705B014FA0305A43717370510
S31A00030AECB00A37753500FA0305B03705B0FE27F53F02350427F8
S31A00030B01F73410276F37380040B3067CBFFA03AE8A7A030B861F
S31A00030B167CD0373800073782006227743402350837DC37B121BA
S31A00030B2BDC37DCDD005B030B34FA0305B837B60001B044FA03AA
S31A00030B4005B837B60002B03AFA0305B837B60100B030FA030577
S31A00030B55B837B60200B026FA03058637B60001B01CFA03058C35
S31A00030B6A37B68000B012FA03058C37B60800B008FA0305863744
S31A00030B7FB60004B0FE27F5350427F734103FFC276F376A0000C7
S31A00030B94EC0A275E37DCFC0A37DCEC0C9C02EC00AC02376500D0
S31A00030BA90034083540FA030982EC00C500F830B70837650000C1
S31A00030BBEFA03992EA100B018EC000601B70827230000EC00C53F
S31A00030BD300F830B7EA37650002A500FA03995A3F04350427F76E
S31A00030BE834103FF2276FAA0437380070B6102775FA030452376B
S31A00030BFD6A0006AA08ED06AD00ED08B01837380040B200A50451
S31A00030C12B0187CBFFA03AF06376A000AAA0CED0AAD00ED0CAD64
S31A00030C270237650004FA030B8A3F0E350427F734103FF6276FC8
S31A00030C3C376A0000F554EC00CA00F523CA01376500007C0217E6
S31A00030C51FC735AAC0837BD03E8A508274D372A340135082723EB
S31A00030C660008A50837FA735A34083540FA030906F52CEC00CA29
S31A00030C7B0537CCFC0637CCAC0037BC3531AC02EC02C5003705AC
S31A00030C90277BFA030A4EEA0837053401350837650000FA03090D
S31A00030CA506F52CEC00CA0337CCFC0437CCAC0027230002EC0265
S31A00030CBA377C3536B5C6EC00AC0627230000EC02C50037052785
S31A00030CCF7BFA030B02277BF530EA042776B700F531EA04E5047C
S31A00030CE4EC06CA0027230002EC02377C353EB5C80600B720F587
S31A00030CF920EC00CA0027230000EC02C5003705277B27230002E0
S31A00030D0EA500FA030BE8AA00EC020600B6D8A5003F0A350427B8
S31A00030D23F73410276F34023508277B37380009BF147CF937DCF9
S31A00030D38FC0737DC17D5FFFFF601B7E634083540FC02B0FE2785
S31A00030D4DF5350427F734103FF6276F34023508375500023402F6
S31A00030D62351037CCFCFE37CC34083540FC04AA08377C000EB258
S31A00030D770027F5B0449C02275C37DCA10837DCD5003705AA049F
S31A00030D8CD50137073715A704AA0437B58408AA00AC0237650024
S31A00030DA10837B5FFFFFA0398523401351037BD000027F0AA0824
S31A00030DB6A504A808B60037BD0001340835403F0A350427F73496
S31A00030DCB103FFE276F27365E1C3787004C373B00E017FD5E1C66
S31A00030DE0AD00B702DD0017BD5E1C373AFF1F27260000B72E376C
S31A00030DF5650000FA030D5227F6B71A37350001FA0306D0376555
S31A00030E0A00007C04ED009502FA0382FA3716B600A500B00637B8
S31A00030E1F650000FA030F4627F53F02350427F73410276F273514
S31A00030E3435C427F5277B27742774277427742774277427742785
S31A00030E4978277427743402350837DC37B135C637DC17FC35C455
S31A00030E5E9C0017BD35C4FC0137B80009B3C827F5277B2774271D
S31A00030E737427742774277427742774277827742774340235089E
S31A00030E8837DC37B149EE37DC17FC35C49C0017BD35C4FC01375E
S31A00030E9DB80009B3C827355E1E27F5277B2774277427742774F9
S31A00030EB22774277427742778277427743402350837DC37B15EB0
S31A00030EC72037DC17FC5E1E9C0017BD5E1EFC0137B80009B3C8EF
S31A00030EDC350427F73410276F373801FEB308F50117FA35C0277B
S31A00030EF1F57A030F20373B00E017FD35C4B70E950037FA35C45F
S31A00030F062715000037B501FE9A02B002F50117FA35C0373AFFEC
S31A00030F1B1F34083540350427F73410276F34023508373B00E0F2
S31A00030F3037F535C49A0017BD35C4173535C0373AFF1F350427E7
S31A00030F45F73410276F3402350827150002373B00E037F55E1E12
S31A00030F5A9A0017BD5E1E373AFF1F350427F734103FF6276F3763
S31A00030F6F6A00047C0437B58408AA00ED04DD02AD0237B5FFFFEB
S31A00030F84FA039852277B2770EC0437CCFC0237CC8500AA06ED19
S31A00030F990437DCA10637DC27FBDA0427230006ED068D00ED04A8
S31A00030FAE37DCA10637DC277A37173705277A27FBDA04376500F0
S31A00030FC3067C01374A00003F0A350427F734103FFC276F376AB6
S31A00030FD80000ED00375500027CFF373801FDB304373521ECFA6E
S31A00030FED039AF637650000FA030F68EC002705000037BD35C240
S31A00031002AD02FA0302C8273635C2B708EC02CC00AC02270600B2
S31A0003101700B6F0EC00ED029C00173635BEB602F50117FA35BEAC
S31A0003102CFA0302D63F04350427F73410276FFA0302C817363514
S31A00031041BEB602F50117FA35BEFA0302D6350427F734103FF87A
S31A00031056276F376A0002AA0437650004FA030EE0AA06B71C3750
S31A0003106B650004ED06375A0002FC04376A000037650002FA033C
S31A000310809A7037650006FA030FD03F08350427F734103FF6278C
S31A000310956F376A0000AA0227250004ED0237DCA10437DCD500A2
S31A000310AAF840B71E371FEA063705277BFA0399D6EA06EC00CAE5
S31A000310BF002723000027230004A50437B80005BFCCEC02C5069A
S31A000310D4371FEA0937B6000FAA04B728F52DEC00CA002723000A
S31A000310E900A50437B80009BF0AFCF6AA04F531EC00CA002723B9
S31A000310FE0000E505F130EC00CA0027230000EC0005003F0A355A
S31A000311130427F734103FF6276F376A0000AA0227250004ED0003
S31A0003112837DCA10437DCD500371FEA08F820B736370534013516
S31A0003113D0834083520FA0399D6EA06EC02C5003705340135083E
S31A000311522723000234083520FA0399D6EA08E506E808B6362756
S31A00031167230004EC04377C0005BFB0EC020600B706C50027236C
S31A0003117C0002F82DB61AEC00C506371FEA081728F008B610EC76
S31A00031191020600B746C50027230002F830B73C27F5B04AE5080C
S31A000311A6F809B30CF1F6EA08EC02C50027230002F831B6E2E5ED
S31A000311BB083705277BEC02C50037053401350837DCFCD037DCDD
S31A000311D02723000234083540340227793520B6BC37BD0000EC87
S31A000311E5020600B60037BD0001340835403F0A350427F73410A4
S31A000311FA3FFC276F376A0000AA02ED00D500371F3705277BFAC9
S31A0003120F0399D6ED02D800B6102723000027230002ED02160027
S31A00031224B6DA37B50001B0FE27F53F04350427F734103FFA2727
S31A000312396F376A0000AA0227250004ED02D5003705277BFA03EC
S31A0003124E99D6F82DB7083716B704F82CB700F820B600F520B0B9
S31A0003126300272300023714ED00DA002723000027230004ED0486
S31A00031278377D0005BFC2ED02D500F82DB608376500027C01FA62
S31A0003128D039AC6B0FE3715F60F3714F760ED00DA003F063504FA
S31A000312A227F734103FFC276F27FBEA00F1E0F85EB300F52EEA08
S31A000312B700E5003705277BFA0317A43F04350427F734103FF48D
S31A000312CC276F27FB34103520FA0310902725000A2600B71E279E
S31A000312E15E37DCA10A37DCD5003705277BFA0312A42723000A06
S31A000312F6275E37DCA10A37DC1600B6DA3F0C350427F734103FB9
S31A0003130BF8276F376A00003401350837DCA10037DCAD02250484
S31A000313207C07FA0312C83735003EFA0317A437650000FA031248
S31A00031335C8EC0037CCFC0E37CCB02EEC000606BC02F501EA045E
S31A0003134AB00A2604B7063735002AFA0317A425043735002CFADB
S31A0003135F0317A437650000FA0312C8EC0037CCFC0737CCAC009E
S31A00031374376500007C0737680002B20417C5FFFFF601B7B42683
S31A0003138904B7043735002AFA0317A4376500007C02376800027E
S31A0003139E37840056EC00C501F8F0B64C376A00003735003AFA43
S31A000313B30317A4B010EC0217C5FFFFEA06F80DB700F80AB6284A
S31A000313C827210002A502A800B2E2B01CEC00C500EA0627230023
S31A000313DD00F81BB300F87FB600F52EEA06E5063705277BFA0326
S31A000313F217A4EC006C02B5D6FA039BD83F08350427F7341027C4
S31A000314076F37351B58FA0303AA373501F4FA030294FA0303EEED
S31A0003141C350427F734103FFE276F2776B71237BD000AAD0037FC
S31A00031431B50004FA03050A277BFA0303AAB000FA0303EE3F02AD
S31A00031446350427F734103FD6276F376A000AAA0C37B50019AA32
S31A0003145B00341035207C04376A00023765000AA50CFA0304BCA3
S31A00031470277B376A00082725000627260004B71E3765000437C4
S31A00031485380006B7143738000CB70E3738000DB7083738001244
S31A0003149AB70237380013B644275E37DCFC0637DCAD0E376500FB
S31A000314AF0E37B50002FA0305463765000437BC000627FB372ABF
S31A000314C4AC1227250010A512A108AA16A510E3076306AA14ED1D
S31A000314D914AD06A516ED0E9A0237BD08007A03155A37B5000AFE
S31A000314EEAA00341035207C04376A00023765000AA50CFA030422
S31A00031503BC277B376A001A2725001827250006275E37DCFC0661
S31A0003151837DCAD1CA51A9A023765001C37B50001FA030546375A
S31A0003152D65000437BC000527FB372AAC202725001EA520A10818
S31A00031542AA24A51EE3076306AA22ED22AD06A524ED1C9A023774
S31A00031557BD0A00AD0437650004FA03A0D8A506AA26ED08AD28A4
S31A0003156C37650026A528FA03A0FE3F2A350427F734103FF827D5
S31A000315816F376A0000AA02A50237F031BCAA06A50017F231BB8B
S31A00031596177231BAAA0437650004A506FA03144A3F08350427C8
S31A000315ABF734103FF4276F376A0000AA02A50237B1CD7FAA0646
S31A000315C0A500F3FD73FFAA0427260004B206B62CED06377D07BF
S31A000315D5CEB324A50237B1687FAA0AA500F3F973FFAA08272627
S31A000315EA0008B206B60CED0A377D176EB304373521F6FA039A60
S31A000315FFF637650000A502FA03144A3F0C350427F734103FFC19
S31A00031614276FFA0302C817F535BEF801B21217FD31B2AD0017E4
S31A00031629FD31B4AD0237650000A502FA03157CFA0302D63F0429
S31A0003163E350427F734103FFE276F2725000017363572B70CFA23
S31A000316530305E427F6B70437350001376A0000A5003F02350488
S31A0003166827F734103FFE276F2500FA0316423716B70227F57A19
S31A0003167D0316FA17F534143705277B2776B70437380001B73259
S31A00031692B05EFA03060825003716B600F501EA002600B7041721
S31A000316A7F52C14F701B00217F52C14F70217FA2C1417F52C1464
S31A000316BCF60317FA2C14F803B72CB028FA030586F401F601EAB2
S31A000316D100B70417F52C14F704B00217F52C14F70817FA2C14AB
S31A000316E617F52C14F60C17FA2C14F80CB7FE2500E50037053F09
S31A000316FB02350427F73410276F173634ECB71A2776B60E27F5E3
S31A0003171037752C123738FFFFB62A37B50001B02427F537752CCF
S31A0003172510B0E8173631C8B704FA03A16E3705B00EFA0302A850
S31A0003173A277537F831BEB3003735000127FB350427F7341027D3
S31A0003174F6F27362C16B614FA030592277B277427742774277402
S31A00031764277427742779377A2C1637B50D9337752C1637263790
S31A00031779B1F35F37FA2C1617F52C163705350427F73410276F21
S31A0003178EFA03174C277517F831C9B3003735000127FB35042796
S31A000317A3F734103FFE276F3402351034043540EA001736735EEA
S31A000317B8B71C377573B63738004FB22E3402350837DC37B173EC
S31A000317CD6637DCDA007C01377A73B6B0181736735DB708E500CB
S31A000317E23705277BFA03C880B006E5003705277BFA0397CC3FAE
S31A000317F702350427F73410276F1736735EB70027F5B008FA03FB
S31A0003180C97A837B8FFFFB7F23705350427F734103FFE276F2718
S31A000318212500001736735EB604FA03978A27F6B7043735000149
S31A00031836376A0000A5003F02350427F734103FFA276F376A0002
S31A0003184B00AA02373500C0FA0397CC3765000C277427742774CE
S31A000318602774FA0397CCED00D500EA043705277B272300003760
S31A000318753800C0B704373800DBB70AB014373500DBFA0397CC2C
S31A0003188AF5DCB006373500DBFA0397CCF5DDEA04E50437052706
S31A0003189F7BFA0397CC27210002B6B8373500C0FA0397CC3F06C7
S31A000318B4350427F73410276F273672ACB708377572ACFA030FD5
S31A000318C924273572AC350427F734103FFE276F27FBEA0027368C
S31A000318DE72ACB75A173672B2B722173572B23705277B373800B6
S31A000318F3DCB708373800DDB708FA0318B8B03AF5C0EA00B0101B
S31A00031908F5DBEA00B00AE500F8DBB604F50117FA72B2B02037A9
S31A0003191D7572B0373801FEB2D2377572B03402350837DC37F1A7
S31A0003193272AC37DCE500DA037C01377A72B03F02350427F73488
S31A0003194710276F34023508340835403705277B27742774277805
S31A0003195C27FB27F4350427F734103FF6276F273672AC37870190
S31A000319713E273672B037870136173672B23786012E377572AC7F
S31A000319867C03376A0002EC0237CC37F172B037CCAC04EC02C580
S31A0003199B00F8FF37860100377572B037380001378600F437351E
S31A000319B0318C37B50002FA0304A2EC02C500EA062723000237A5
S31A000319C50534013508377D0002B73EBE04377D0001B706B044BA
S31A000319DA377D0003B716B03CEC02C500370527230002277BFAA8
S31A000319EF03194637FA341E7A031AA4EC02C5003705272300027F
S31A00031A04277BFA03194637FA31D67A031AA4EC02C50017FA315E
S31A00031A19C9272300027A031AA4E506F60F37860086E506371FEB
S31A00031A2E371F371F371FEA063705AA0837F8345EB71A27363497
S31A00031A435E37870068A504A00234013508EC08AC003765000206
S31A00031A58FA031842B050FA0316423716B64837F572ACFC04AA85
S31A00031A6D08EC026C08B710A504A00234013508AD003765000222
S31A00031A82A508FA039A7017FC72ACA504A002340135088D0234E1
S31A00031A97043520FA030FD0273572ACB00A376500027C0237680D
S31A00031AAC00043783FF06173572B2273572B0273672ACB60837FB
S31A00031AC13501FEFA030EE037FA72AC3F0A350427F734103FFC7A
S31A00031AD6276F37B503E8FA0304CE376A0000AA0237650000A528
S31A00031AEB023F04350427F734103FFA276F376A0000ED00375514
S31A00031B000000375700022776B724DD00AD02ED00DD02AD04377F
S31A00031B15650002A504FA0302743716B714ED00271500002715B2
S31A00031B2A000237B50001B00637650000FA03022627F53F0635A1
S31A00031B3F0427F734103FFA276F373500C0FA0397CCFA030DCAF3
S31A00031B54AA04B720EC0437CCFC0437CCED0495023775345E37FB
S31A00031B696A000034043520FA03184237650004FA030F46FA0321
S31A00031B7E97A837B8FFFFB71037B800C0B602FA031964B004378A
S31A00031B9305277BFA0318D22725000217F535BEF801B20E373534
S31A00031BA80001FA0317003716B70237BD0004AD02273635C2B752
S31A00031BBD083765000237370002376A0002173635C0B7083765B4
S31A00031BD2000237370001376A000237650002FA0306F27A031BB6
S31A00031BE7503F06350427F734103FFC276F340235082500160031
S31A00031BFCB60027F5B03EE500D400EA0037DCFC0137DCD500F878
S31A00031C112AB6E2340835207C0137B50002FA039EC63401350824
S31A00031C2637BC0000E5003705277B34083540340227793520B658
S31A00031C3B0037BC0001340435403F04350427F734103FFC276F3B
S31A00031C50376A0000250237350024FA0317A4ED00D50037052741
S31A00031C657BFA0317A4E502ED00D400EA0227230000ED0016004D
S31A00031C7AB6DE3735002AFA0317A4E5023705277BFA039B843752
S31A00031C8F35000DFA0317A43735000AFA0317A43F04350427F775
S31A00031CA43410276F1736354E3787008A17F508853705373522CD
S31A00031CB904FA0308F217F50886370537352206FA0308F217F5A5
S31A00031CCE0887370537352208FA0308F217F5088437053735223E
S31A00031CE32CFA0308F217F5088337053735222EFA0308F217F52E
S31A00031CF80882370537352230FA0308F23735220D37B572D2FA8E
S31A00031D0D033C943735221837B572D6FA033D4C37F572DC37359F
S31A00031D222224FA03090637F572DA37352228FA0309063735218A
S31A00031D37FEFA031C4A350427F734103FD8276F376A0006AA088C
S31A00031D4CE52FEA0A37BC0003AC0E37650008FA039AC6277B37E7
S31A00031D611727F8371734013508376A0012AD1037BC0064AC00FB
S31A00031D76341035207C04376A000234083520A512FA0304BCAAE4
S31A00031D8B0CB008EC08C50027230008F82EB702EC080600B6EAF2
S31A00031DA03765000427742774376100042774376A0004EC08C5BA
S31A00031DB5003705277BFA0399C23716B712376500047CD0EC08E4
S31A00031DCAC50037052778376A0004272300082721000EB6BE3763
S31A00031DDF65000C37B5EA60FA0304CE376A0014AA16A504AA1A8E
S31A00031DF427250018A516A11AAA1EA514E3196318AA1CA51CEC8C
S31A00031E09068A00A51E8A02E50AF853B700F857B622EC06CC0006
S31A00031E1EAC20EC06CC02AC2237650020A522FA039AB2376A00DF
S31A00031E3324AA26A524EC068A00A5268A023F28350427F73410FF
S31A00031E483FFE276F34023510CC00AC00ED00C500F82CB712D542
S31A00031E5D0037DCFC0137DC3716B60027F5B012D500F82CB6E6CE
S31A00031E72150037DCFC0137DC340235108D00A5003F02350427CC
S31A00031E87F734103FFA276F376A0000AA02E50DEA04341035206D
S31A00031E9CFA031E46277B2776B714ED02375A000037DCFC0237F5
S31A00031EB1DCAD022104B6DC37B50001B0FE27F53F06350427F77E
S31A00031EC634103FFE276F37BD001BAD0037B50032FA03050A3FC2
S31A00031EDB02350427F734103FFE276F37BD00F3AD0037B5007D7C
S31A00031EF0FA03050A3F02350427F73410276FF50117FA72B437F2
S31A00031F05B5000137FA72D0373572C8FA030210F50117FA72B7B0
S31A00031F1A350427F73410276FF50117FA72B6350427F734103F6F
S31A00031F2FFC276F376A0000AA02ED003755000837380167B300AA
S31A00031F4427150008FA0302E4ED02DD0017BD0882ED02DD021749
S31A00031F59BD0884ED02DD0417BD0886FA0302C817F5088417FA7F
S31A00031F6E318817F5088517FA318917F5088617FA318A17F508BE
S31A00031F838717FA318BED00DD0017BD72D2ED00DD0217BD72D424
S31A00031F98ED00DD0417BD72D6ED00DD0617BD72D8ED00DD08176A
S31A00031FADBD72DAED00DD0A17BD72DCFA0302D6FA031EFAFA0330
S31A00031FC21CA43F04350427F734103FFC276F376A0000AA02271E
S31A00031FD7753402350837DC37B12C1837DCF530DA007C013738C7
S31A00031FEC000BB3E4ED0037550000FA03992E34013510ED00375A
S31A00032001CC910037CC37350006ED005C00B3187CFF34023508ED
S31A0003201637DC37B12C1837DC37CCFCFF37CCC500DA002776B667
S31A0003202BDAED02DC000600B70CC500F82EB70637CCFC0137CC7E
S31A000320400600B6EC37350006ED025C00B3187CFF34023508372D
S31A00032055DC37B12C1E37DC37CCFCFF37CCC500DA002776B6DA7F
S31A0003206A37B52C18ED009A0037B52C1EED029A003F043504273F
S31A0003207FF734103FFC276F376A0000AA02ED021600B70CD5004D
S31A00032094F82EB70637DCFC0137DC1600B6EC3408352037600048
S31A000320A90237380006B60A37650000FA03992E37B80006B70ACC
S31A000320BE3410352034103540FC02FA031FCAFA0302E43765004F
S31A000320D3007C04FA0308C017FA0882376500007C02FA0308C030
S31A000320E817FA088337650000FA0308C017FA088437650002FAA8
S31A000320FD0308C017FA0885376500027C02FA0308C017FA0886DC
S31A00032112376500027C04FA0308C017FA08873F04350427F7345E
S31A00032127103FEA276F7C0637B50009AA0034103540FC02FA03F6
S31A0003213C1E88EA143787009C37650012A502FA032080FA031F79
S31A000321511EED04D500F841B704273572D07A0321E2FA0302C8B3
S31A0003216617F5088417FA318817F5088517FA318917F5088617E4
S31A0003217BFA318A17F5088717FA318BEC06ED08D5003705277B8F
S31A00032190376A0000373572D234043540FA031D40EC0AED0CD515
S31A000321A5003705277B376A0000373572D634043540FA031D40E2
S31A000321BA3765000EFA039AC6277B377A72DC37650010FA039A1C
S31A000321CFC6277B377A72DAFA0302D6FA031EFAFA031CA43F1691
S31A000321E4350427F73410276F377572F67C01377A72F63738276C
S31A000321F90FB300273572F6350427F734103FDE276F7C06275EED
S31A0003220E37DCFC0E37DC37B50009AA0034083540FA031E88EAA5
S31A0003222320378700F4ED161600B604173572B87A03231E376528
S31A000322380016FA039294173672B8B61A3765001637B52236FA18
S31A0003224D03994027F6B60437350001FA03425A173672B8B70C80
S31A000322623765001637B572EAFA03994027F6B702F50117FA723F
S31A00032277B5FA0302C8F50117FA72B837F572DEAA0237F572E0F6
S31A0003228CAA0437F572E2AA0637F572E4AA0837F572E6AA0A37B3
S31A000322A1F572E8AA0CED1637B5000CAA00373572EA34083540FC
S31A000322B6FA03999CEC18ED1AD5003705277B376A00003735729B
S31A000322CBDE34043540FA031D40EC1CED1ED5003705277B376AA9
S31A000322E00000373572E234043540FA031D40377572DE3768007E
S31A000322F502B61A377572E037680004B610377572E237680006ED
S31A0003230AB606377572E437680008B700FA0321E8FA0302D63F7F
S31A0003231F22350427F734103FDC276F7C0637BD000CAD003410BF
S31A000323343540FC02FA031E883716378700823765000EFA039AA7
S31A00032349C637FA73023765000CFA039AC627F63787006834107E
S31A0003235E35207C1AA512FA030848ED14D500370537B8004DB76D
S31A000323733ABE0437B80046B70CB04437B80066B70437B8006DF8
S31A00032388B724B036274E37CCFC1A37CCAC1E3765001E37B52253
S31A0003239D3CFA03A02C376A0020AA22ED20AD1AED22EC1E8D0214
S31A000323B2FA0302C8EC1A17BC7304ED1C17BD7306FA0302D63F8C
S31A000323C724350427F734103FFC276F376A0002ED02D500F847C2
S31A000323DC3786007C37BD0006AD0037B52240FA039A5627F6B6F5
S31A000323F11237650002FA031BEE3716B75C37650002FA032126D6
S31A00032406B05237BD0006AD003765000237B52248FA039A562707
S31A0003241BF6B61237650002FA031BEE3716B73037650002FA0372
S31A000324302204B02637BD0006AD003765000237B52250FA039A58
S31A000324455627F6B61037650002FA031BEE3716B70437650002F6
S31A0003245AFA0323243F04350427F734103FFE276F27FBEA00F86B
S31A0003246F0DB700F80AB6362775173672B3B606273672AEB7009F
S31A0003248437350001173572B3273572AE2776B75817F57248F876
S31A0003249924B60637357249FA0323CCB04637357248FA0386AEE5
S31A000324AEB03CE500F1E0F85FB206377572AE37380062B304F516
S31A000324C30117FA72B3B02217FD72AE274D37CC37B1724837CCA2
S31A000324D8E500CA0037DCFC0137DC17BD72AE37DC37B172483734
S31A000324EDDC15003F02350427F73410276F340235083401351081
S31A00032502377C0000BC20377CFF9DBC0037BCFF9DF52DDA003462
S31A000325170835207C013404354027F234013508FA0308F2B008E5
S31A0003252C3408352034043540FA030906350427F734103FF42752
S31A000325416F376A000634013508DC00AC08DD02AD0A37BC03E8F0
S31A00032556AC00341035207C04376A000237650008A50AFA0304AB
S31A0003256BBC37650006FA030906376500067C03A504FA03090612
S31A000325803F0C350427F73410276F27F5273672D0B60037B50064
S31A0003259501350427F73410276F27F5173672B4B702273672D00F
S31A000325AAB60037B50001350427F734103FFC276F377572D037DF
S31A000325BF380001B62237F572CA37B12710AA0237F572C8F30061
S31A000325D47300AA0037650000A502FA0302743716B70027357244
S31A000325E9D03F04350427F734103FFC276F376A0000AA021736BB
S31A000325FE31CAB70837B531CAFA0311163716B63C3765000237E6
S31A00032613360001B712173631E0B70C3765000037B531E0FA03F2
S31A0003262811163716B61C3765000237360002B71817363402B738
S31A0003263D123765000037B53402FA0311163716B70237B5000198
S31A00032652B0FE27F53F04350427F734103FF6276F27FB3410355C
S31A0003266720FA0310903735348834103540FA039F302775371602
S31A0003267CB6003735000127FB3F0A350427F734103FEC276F272F
S31A00032691250010272500123765001234103540FA03968AAA1258
S31A000326A6B736341035207C10FA0381D23716B728E50037052740
S31A000326BB7BFA0317A4E5013705277BFA0317A437350020FA03C9
S31A000326D017A4341035207C02FA039912FA039BD8B0B23F143518
S31A000326E50427F734103FEC276F376A001027250012277A3717B2
S31A000326FA3705277AFA0317A4E5113705277BFA0317A437650005
S31A0003270F1234103540FA03968AAA12B7183765000037680010EE
S31A00032724B6E237350020FA0317A4341035207C02FA0399123FBD
S31A0003273914350427F734103FEC276F376A001027250012376567
S31A0003274E001234103540FA03968AAA12B60027F5B010341035BE
S31A0003276340FC0237650010FA03994027F6B6D6A5003F143504BE
S31A0003277827F734103FFE276F376A0000277B34023510377C009D
S31A0003278D00B60037BC01683765000034043540FA03090637652B
S31A000327A200007C04A508FA030906F52FED00DA03376500007CDA
S31A000327B70727FB3F02350427F734103FEA276F376A0000AA02F3
S31A000327CC25042776378C006037650000AE0AED0A9502FA039A8D
S31A000327E1B2376A0006AA08A506AA00A508ED0A9A023765000A94
S31A000327F637B52258FA0307B6376A000CAA0EED0CAD00A50EEDFA
S31A0003280B0A9A023765000037380001BE08B6123765000E373856
S31A00032820869FB30837BD0001AD0037B5869FAA02F501EA04B0C7
S31A000328353CAE103765001037B52258FA0307B6376A0012AA144E
S31A0003284AED12AD00A514ED109A02376500003738000FBE08B6DC
S31A0003285F12376500143738423FB30837BD000FAD0037B5423FD1
S31A00032874AA023765001C37B5225CFA03995AAA1C3410354037D2
S31A0003288965001CFA03253C2604B702F52DED1CDA00A51CFC06A7
S31A0003289E3F16350427F734103FF2276F376A0006AA08A5083728
S31A000328B3B12710AA08A506F3007300AA0627260006BC0627254B
S31A000328C8000627250008B020A50637B8000BBE0CEC06377C00B4
S31A000328DD0BB610A50837B87FA2B30837BC000BAC0637B57FA2D7
S31A000328F2AA0837BC005BAC00341035207C04376A0002376500C4
S31A0003290706A508FA0304BC340135083735005B34023510372A2D
S31A0003291CAC0CE50DF121EC14CA003408354034023510372AAAE0
S31A000329310AE50BF121EC14CA01E505F121CA02F57DCA0337353E
S31A0003294600043761001427FB3F0E350427F734103FFA276F37B3
S31A0003295B6A0000AA02EC00CD0237DCFC0437DC37DCA10037DCA0
S31A00032970AD0417363487B724173672B8B71E173672EAB71837BA
S31A0003298565000437B52260FA03995AAA043765000437B572EAD7
S31A0003299AFA03995AAA04273673BCB720377573BC37BD226A378C
S31A000329AF380001B60037BD22643765000434083540FA03995A60
S31A000329C4AA04273573BCEC0227060016B71ECD161600B718F5F9
S31A000329D920EC04CA0027230004EC02CD16376500043408354096
S31A000329EEFA03995AAA04ED0437DCFCFC37DC37DCA00037DCEC6C
S31A00032A03008D023F06350427F734103FFC276F3401350827FBE1
S31A00032A18EA0234083540EA002726000AB700F530EA00E502E134
S31A00032A2D00EA023714EA023705277B3F04350427F734103FCCA1
S31A00032A42276F376A000AAA0CE53BEA0EED0CDD02AD18ED0CDDF4
S31A00032A5704AD1A37650018A51AFA039AAC376A001CAA1E37B56F
S31A00032A6CEA60AA00341035207C04376A00023765001CA51EFA27
S31A00032A810304BC277B376A0006ED04AD222725002037B503E828
S31A00032A96AA00341035207C04376A00022775A522FA0304BC2775
S31A00032AAB7B376A00083765000437BC000A27FB372AAC04ED0626
S31A00032AC0AD262725002437B5000AAA00341035207C06376A0059
S31A00032AD5022775A526FA0304BCAA12ED08AD2A2725002837B5D5
S31A00032AEA000AAA00341035207C08376A00022775A52AFA0304EE
S31A00032AFFBCAA14ED04AD2E2725002C37B5000AAA0034103520C2
S31A00032B147C04376A00022775A52EFA0304BCAA16F550EA32171C
S31A00032B29F53411EA11277AE511277A373600F8B700F541EA32B3
S31A00032B3EE513370534013510E5323705AA30277AE511277A372F
S31A00032B53360004376A000034043520FA032A0CEA32ED0ADA00DC
S31A00032B68E507370534013510277AE511277A37360002376A0065
S31A00032B7D0034043520A530FA032A0CEA32ED0ADA01E515370581
S31A00032B9234013510277AE511277A37360001376A0000340435F7
S31A00032BA720A530FA032A0CEA32ED0ADA02E5093705277BED0C34
S31A00032BBCD502F680EA32370534013510AC0037B50050FA032ACD
S31A00032BD10CEA32ED0ADA03E5173705340135102775260EB600B2
S31A00032BE637350001376A00003404352037B50050FA032A0CEADD
S31A00032BFB32ED0ADA04E505370534013510ED0CD506371F371F95
S31A00032C10371F371F371F371F371FEA323705277B37340001375B
S31A00032C256A00003404352037B50050FA032A0CEA32ED0ADA0539
S31A00032C3A17F53412F60F3714F760DA063F34350427F734103F56
S31A00032C4FD0276F376A000AAA0CEC0AAC0EEC0CCC06AC16EC0C6C
S31A00032C64CC08AC1837650016A518FA039AAC376A001AAA1C3750
S31A00032C79B5EA60AA00341035207C04376A00023765001AA51C61
S31A00032C8EFA0304BCAA103765000437BD000A274D27FB372A34E8
S31A00032CA3043520376A0004376A00202725001E37B50064AA00F0
S31A00032CB8341035207C04376A00022775A520FA0304BCAA12EC7C
S31A00032CCD10377C0009B204A51037B100BEB00C376500107C9C8C
S31A00032CE237380009B202A510FC50AA10EC12377C0009B202A5DA
S31A00032CF712FC3CAA12EC0CCC0CAC06EC0CCC0AAC083765000613
S31A00032D0C37380063B20437310320376A00063735000AA506349A
S31A00032D21023510372A27F6B6083765000837310190376A0008CB
S31A00032D362775A51037B80063B30037350001376A00003765007F
S31A00032D4B0EA50CFA032A3EEC0E37CCFC0737CCAC0E3765000EDF
S31A00032D6037B531CAFA031234EC0E37CCFC0737CCAC0E17C5FF93
S31A00032D75FFF70117CAFFFFF503CA002723000EF5F0EC0ECA00A7
S31A00032D8A2723000E37350064A51034023510372AAA10A506AA63
S31A00032D9F242725002237BC000AAC00341035207C06376A00021D
S31A00032DB42775A524FA0304BCAA14A508AA282725002637BC003D
S31A00032DC964AC00341035207C08376A00022775A528FA0304BCF6
S31A00032DDE340135083765000627742774376100062774376A00B3
S31A00032DF30637DCA10637DCF560EC0ECA00E511F11CCA01E51310
S31A00032E08F11CCA02E505F11CCA03E515F11CCA0434083540F198
S31A00032E1D1CCA05E509F11CCA06EC0CC513EC0ECA07EC0C3745D2
S31A00032E320012277A37173705277A27FBEC0ECA0837CCFC093777
S31A00032E47CCAC0E17363530B722EC0C3745000E374700102776AF
S31A00032E5CB714850EAA2ACC10AC2CEC0EAC003765002AA52CFA3B
S31A00032E710328A4AA0EA50EA00A340135083F30350427F73410E3
S31A00032E863FF4276F376A0002AA04EC0437CCFC0237CC340435B3
S31A00032E9B40FA033C94ED02D509DA07ED0437550012277A3717E0
S31A00032EB03705277A27FBED02DA0837DCFC0937DCAD02EC043733
S31A00032EC5CCFC0637CC3765000234043540FA033D4CED02D50A7F
S31A00032EDADA08ED04D513ED02DA0937DCFC0A37DCAD02ED04D5AC
S31A00032EEF13F85FB60637650002FA03C7BAB042ED042716000C57
S31A00032F04B710DC0A950CAA003765000234043540FA03277AAA24
S31A00032F190217363530B722ED043755000E375700102776B7147C
S31A00032F2E950EAA06DD10AD08ED02AD0037650006A508FA032781
S31A00032F43C0AA02A5023F0C350427F734103FE6276F376A000813
S31A00032F58A520AA0AED22AD0C37B52059AA00341035207C0437BB
S31A00032F6D6A00023765000AA50CFA0304BC277B376A0006376ADC
S31A00032F8200122725001037BD005BAD00341035207C06376A000B
S31A00032F97022775A512FA0304BC277BEA0EA504AA1627250014A7
S31A00032FAC37BD005BAD00341035207C04376A00022775A516FAFE
S31A00032FC10304BC277BEA18E50EF121ED08DA00E507F121DA01DE
S31A00032FD6E518F121DA02E505F121DA033F1A350427F734103FE6
S31A00032FEBDA276F376A0008AA0A37B50052AA04274E37CCFC0497
S31A0003300037CCAC0C37B565C08A02EC0AA5068004AA10A504C210
S31A00033015034202AA0EA50EAA04A510EC0C8A023765000C37B570
S31A0003302A2270FA0307A2376A0012AA14EC12AC04A514EC0C8AF6
S31A0003303F02376500087C01EC04AC00EC0CCC02AC02FA032F4EC6
S31A0003305437B500A4AA0437B5CB80EC0C8A02EC0AA5068108AA91
S31A0003306918A504C3074306AA16A516AA04A518EC0C8A0237656F
S31A0003307E000C37B52274FA0307A2376A001AAA1CEC1AAC04A524
S31A000330931CEC0C8A02376500087C05EC04AC00EC0CCC02AC024A
S31A000330A8FA032F4EEC0A37450012277A37173705277A27FBEC32
S31A000330BD08CA00EC0AC513EC08CA09C5003705277BFA0399C293
S31A000330D2EA20B704EC08C500F131CA00EC0837CCFC0A37CCACCA
S31A000330E708EC0A2706000CB7343745000A7C0227FB27FF27FF37
S31A000330FCEA1F3745000CFA03966A277BEA20E51FF859B200F184
S31A0003311121B0FEF521EC08CA00E520F121EC08CA01F55F7A0356
S31A00033126318AEC0A3745000E374700102776B7363765000A7C16
S31A0003313B0EFA039726340135083735005B34023510372AAC24C9
S31A00033150E525F121EC08CA003408354034023510372AAA22E549
S31A0003316523F121EC08CA01F557B01637753546FA03965A277B90
S31A0003317AEA22F57BEC08CA00E522F121CA01F54FCA02A508FC60
S31A0003318F033F26350427F734103FFC276F376A0000340135083B
S31A000331A437DCFCFF37DC6D00B52A3735000AD500F82AB616A5C2
S31A000331B90A34023510372AAA02E503F130DA0034023510A50A59
S31A000331CE372AAC0A37DCFCFF37DC6D00B4D23F04350427F734EA
S31A000331E3103FFC276F3401350827FBA10AAA0227FBFC09AA0031
S31A000331F837680000B4221600B71ED50034023510CA0037DCFC30
S31A0003320D0137DC7C0137680000B5E2B006F52034023510CA00CC
S31A000332227C0137680002B5EC27FB3F04350427F734103FFC276D
S31A000332376F376A0000AA02B00027230002ED02D500F82CB7F032
S31A0003324CF820B7ECED021600B72A37650000A502FA031234ED50
S31A000332610037DCFC0737DCAD00ED021600B7D0D500F82CB7C677
S31A00033276ED02D500F820B7C227230002B0E2ED0017D5FFFFF739
S31A0003328B0117DAFFFFA5003F04350427F734103FF6276F376A46
S31A000332A0000017363498B74227363494B706377572FE3778341D
S31A000332B594B44027363496B72C37753496FA031AD2376A000267
S31A000332CAAA04A50437F172BEAA08A50217F372BD177372BCAA43
S31A000332DF0637650006A508FA0302743716B60A37BC339AED004F
S31A000332F49C1437BC3503B014373572BCFA030210273572FE3771
S31A00033309BC3498ED009C1437BC350C9C163F0A350427F73410B7
S31A0003331E3FFC276F376A0000AA0237BC21D4173633EAB7003733
S31A00033333BC33EA3765000034043540FA031234ED0037DCFC0714
S31A0003334837DCAD003765000037B531CAFA031234ED0037DCFCE5
S31A0003335D0737DCAD00ED02DC143765000034043540FA03323202
S31A00033372AA00F503ED00DA0027230000F5F0ED00DA0027230094
S31A0003338700A5003F04350427F734103FF6276F376A0002AA0489
S31A0003339CFA03331CAA06EC040619378700D8C5183705277B3780
S31A000333B1380001B708373800023787008C7A033484F53BEC06F4
S31A000333C6CA0027230006EC06AC08ED0437DCFC1937DC37B50011
S31A000333DB09AA003765000634083540FA0331E2AA06EC04CC0052
S31A000333F0AC0037650008FA033196F52AEC06CA00F57ACA073759
S31A000334056500067C0117F53188370534013508FA0308F23765BB
S31A0003341A00067C0317F53189370534013508FA0308F237650008
S31A0003342F067C0517F5318A370534013508FA0308F2EC0637CC97
S31A00033444FC0837CCAC06B03EF529EC06CA0027230006EC06ACFB
S31A0003345908ED0437DCFC1937DC37B50003AA00376500063408AA
S31A0003346E3540FA0331E2AA06EC04CC00AC0037650008FA0331D1
S31A0003348396F521EC06CA00272300061736346FB7083765000622
S31A00033498A504FA032FE8B00637650006A504FA032E84AA06A059
S31A000334AD02340135083F0A350427F734103FF6276F376A000439
S31A000334C2AA06FA030D24AA08B73A3765000837600004340235C1
S31A000334D70837650006340835402779376A000637BC8408AC000A
S31A000334ECEC06AC023765000837B5FFFFFA039852340135083407
S31A000335010835202770377A73003F0A350427F734103FFC276FDF
S31A00033516376A0002ED0227150000151837F533F69A1237F572FD
S31A0003352BD29A0237F572D49A0437F572D69A0637F572D89A08D8
S31A0003354037F572DA9A0A37F572DC9A0C37F573049A0E37F57347
S31A00033555069A1017363464B71EEC0237CCFC1937CC37BD000AE7
S31A0003356AAD003735346434043540FA039A7017F5346EED02DA67
S31A0003357F18FA0325863716B70AED022715000E2715001027159F
S31A00033594000C377572DC37380001B202ED022715000C3765001C
S31A000335A902FA0332983F04350427F734103FD8276F3410352017
S31A000335BE7C02FA0335102726000EB70AA50E37FA72F8EC0C17B6
S31A000335D3BC72FAB000273572F8173572B5173572BA373572C0B3
S31A000335E8FA030210173672B4B75A373501FEFA030EE0AA2637D5
S31A000335FD87018217363410B70E376500267C0434103540FC0257
S31A00033612FA032C4CB00C376500267C0434103540FC02FA033340
S31A0003362790EC268A023765002634103540FC02FA0329543765C8
S31A0003363C00267C04EC268502FA0334B837650026FA030FD01793
S31A00033651363531B73E373501FEFA030EE0AA263787011E37652B
S31A0003366600267C0434103540FC02FA03331C277BFA030C362795
S31A0003367B7B3402350837DCFCFC37DC37DCA02637DCEC268D0298
S31A0003369037650026FA030FD017367308B742373501FEFA030E47
S31A000336A5E0AA26378700D6376500267C0434103540FC02FA03CD
S31A000336BA331C277B37B5730AFA03995A277B3402350837DCFC84
S31A000336CFFC37DC37DCA02637DCEC268D0237650026FA030FD0A3
S31A000336E4173672B837870096173634703787008E373501FEFA5B
S31A000336F9030EE0AA2637870080373572EA17363471B7003735D7
S31A0003370E3471275E37DCFC1B37DC37B5000AAA0034083540FAEB
S31A00033723039A7017FC72F6AC0217F53470EA1A17FC354CAC144A
S31A0003373837F572DEAA0417FC72E0AC0637F572E2AA0817FC727B
S31A0003374DE4AC0A37F572E6AA0C17FC72E8AC0E17F572B917FA1B
S31A0003376272B8376500267C0434103540FC02FA033390277BECD8
S31A0003377726374A000237650026FA030FD03F28350427F73410EB
S31A0003378C3FE6276F376A0004274E37CCFC0437CCAC108A0217E5
S31A000337A1FC72D2AC0817FC72D4AC0A37650008A50AFA039AAC71
S31A000337B6376A000CAA0E37BCEA60AC00272500023765000CA50C
S31A000337CB0EFA0304BC37BD005A340835202779FA039684AA00D5
S31A000337E037650004EC108502FA0304F2376A0004EC108A023751
S31A000337F565001037B50008FA030516EC04AC16EC10CC02AC18F5
S31A0003380A37BC021CAC002725000237650016A518FA0304BC3F2A
S31A0003381F1A350427F734103FF8276F376A0004AA0637BD021CA2
S31A00033834AD002725000237650004A506FA0304BC3F08350427CC
S31A00033849F734103FE6276F376A0004274E37CCFC0437CCAC108F
S31A0003385E8A0217FC72D2AC0817FC72D4AC0A37650008A50AFA59
S31A00033873039AAC376A000CAA0E37BCEA60AC00272500023765B6
S31A00033888000CA50EFA0304BC37BD005A340835202779FA039694
S31A0003389D84AA0037650004EC108502FA0304F2376A0004EC1028
S31A000338B28A023765001037B50008FA0305163765001037B522FA
S31A000338C778FA0307B6376A0016AA1837650016A5183F1A350437
S31A000338DC27F734103FF8276F376A0000275E9A02340835203715
S31A000338F1B52278FA0307B6376A0004AA0637650004A5063F08C9
S31A00033906350427F734103FEE276F376A0000AA02ED18AD04ED55
S31A0003391B1AAD06173672B4378700982726001C37870090A5029A
S31A0003393037F072D4AA02A50017F272D3177272D2AA00272600A9
S31A0003394500BC1437650000A502FA039AB2376A000AAA0CED0AB0
S31A0003395AAD00ED0CAD0237650000A502FA033824AA08A81CB236
S31A0003396F52A50637F072D8AA06A50417F272D7177272D6AA04A2
S31A0003398427260004BC1437650004A506FA039AB2376A000EAA17
S31A0003399910ED0EAD04ED10AD0637650004A506FA03378AA81CD7
S31A000339AEB21237650008FA039896277B3768001CB20237B5006B
S31A000339C301B0FE27F53F12350427F734103FF4276F376A0000C5
S31A000339D837BC3436AC02F575EA0627250008B00027230002EC30
S31A000339ED02C500EA0AF820B7EEF82CB7EAEC020600378700FAD3
S31A00033A02C500F82D3786007627230002EC02C5003705340135E4
S31A00033A1708377D0061B70ABF10377D006CB702377D0075B60428
S31A00033A2CEC02C500EA06B03E37650000FA03992E3401350837E2
S31A00033A41DCA10037DCAD04EC0437CCFCFD37CCAC046C00B31C4C
S31A00033A56C500F82DB616C501F831B610C502EA0AF82FB308F852
S31A00033A6B35B204C502F111CA010502EC0206003787FF6C7A031D
S31A00033A8039E8EC00AC04EC04C50037053401350834083520FA7D
S31A00033A950399D6EA0AEC02C800B6123716B70EF820B70AF82C20
S31A00033AAAB7062723000427230002B0CCEC0406003787009837A8
S31A00033ABF650004376000003402350837650008340835403402EB
S31A00033AD427793520BC0CAD08B008EC02C500F82CB70C272300C6
S31A00033AE902EC020600B70AC500F820B6E4EC0206003786FEECF6
S31A00033AFE27260008B710ED0037DCA10837DC37650000340835C5
S31A00033B1340FA03995AE506370534013508377D006CB734378FFA
S31A00033B280056377D00753786004EEC00AC04060037870084EC25
S31A00033B3D04C5003705277BFA0399D6EC04CA0027230004EC045F
S31A00033B520600B6E2B02627F57A033BD4EC00AC040600378700D9
S31A00033B6758EC04C5003705277BFA0399E6EC04CA0027230004D1
S31A00033B7CEC040600B6E2EC00AC040600B734EC04C500370534EB
S31A00033B91013508377D002AB70CBE04377D0024B704B010377D6E
S31A00033BA6002CB60AA504FC0137650004FA03995AB000272300E5
S31A00033BBB04EC040600B6C437BD0000EC000600B70037BD0001E6
S31A00033BD0340835403F0C350427F73410276F37BC000037B500CB
S31A00033BE51A3404352037263401350837DC37B173C237DC37755D
S31A00033BFA73C0375A001817BD73C037CCFC0137CC377C0063B3FE
S31A00033C0FCE350427F734103FFE276F376A0000ED00D5023705BA
S31A00033C24277BFA039C243735002EFA0317A4ED00D501370527AB
S31A00033C397BFA039C243735002EFA0317A4ED00D5003705277B43
S31A00033C4EFA039C2437350020FA0317A4ED00D5033705277BFABA
S31A00033C63039C243735003AFA0317A4ED00D5043705277BFA0381
S31A00033C789C243735003AFA0317A4ED00D5053705277BFA039CD2
S31A00033C8D243F02350427F734103FEE276F376A0008340135083B
S31A00033CA21600BC1CF553EC08CA099500AA0EDD02AD1037650082
S31A00033CB70EA510FA039AB2376A000AAA0CB00AF54EEC08CA09BE
S31A00033CCC9500AA0ADD02AD0C37BC03E8AC00341035207C04371F
S31A00033CE16A00023765000AA50CFA0304BC277B376A000C2725AA
S31A00033CF6000A37B5003CAA00341035207C06376A00022775A5D5
S31A00033D0B0CFA0304BC3401350837650008FA0308F23765000820
S31A00033D207C02ED0634083540FA0308F2376500087C05ED043422
S31A00033D35083540FA030906F52EEC08CA04F52CCA083F12350485
S31A00033D4A27F734103FEE276F376A0008340135081600BC1CF538
S31A00033D5F57EC08CA0A9500AA0EDD02AD103765000EA510FA03E2
S31A00033D749AB2376A000AAA0CB00AF545EC08CA0A9500AA0ADDA2
S31A00033D8902AD0C37BC03E8AC00341035207C04376A000237657F
S31A00033D9E000AA50CFA0304BC277B376A000C2725000A37B500FE
S31A00033DB33CAA00341035207C06376A00022775A50CFA0304BC44
S31A00033DC83401350837650008FA030906376500087C03ED063471
S31A00033DDD083540FA0308F2376500087C06ED0434083540FA038F
S31A00033DF20906F52EEC08CA05F52CCA093F12350427F734103F9F
S31A00033E07FC276F376A0000AA02EC0237CCFC0A37CC3404354017
S31A00033E1CFA033C94F52CED00DA0A37DCFC0B37DCAD00EC0237CA
S31A00033E31CCFC0E37CC3765000034043540FA033D4CED00150BBE
S31A00033E4637DCFC0B37DCAD00A5003F04350427F734103FFC279F
S31A00033E5B6F376A0000AA02ED02D503370534013510FA0308F219
S31A00033E70376500007C03ED02D504370534013510FA0308F2376D
S31A00033E856500007C07ED02D502370534013510FA0308F2376528
S31A00033E9A00007C0AED02D501370534013510FA0308F2F53AEDF6
S31A00033EAF00DA02F57ADA05F520DA06F52EDA0CDA09376500004E
S31A00033EC47C0D27FB3F04350427F734103FFA276F376A000037B0
S31A00033ED9BD2C24AD0217F5340E3705277B37380001B70C373841
S31A00033EEE0002B60637352C2437B5227CB0043765000237B52252
S31A00033F0384FA03995AAA02F52CED02DA002723000237650002AC
S31A00033F18A500FA033E04AA02F52CED02DA002723000217F53485
S31A00033F2D0EF802B624F530ED02DA0027230002F52CED02DA0070
S31A00033F4227230002F54DED02DA0027230002F52CED02DA0027AD
S31A00033F5723000237650002A500FA03995A37650002FA0339CE52
S31A00033F6C3716B75017F5340EF802B64037650002FA03992E271C
S31A00033F817B37610002376A0002F52CED02DA0027230002EC0048
S31A00033F9637CCFC1237CC3765000234043540FA033E56AA02F57C
S31A00033FAB2CED02DA0027230002F561ED02DA00150137352C24C6
S31A00033FC0FA031C4A3F06350427F734103FFC276F376A00002707
S31A00033FD5F6B650373803E7B206FA039BE83735228AB04CA50088
S31A00033FEA37B8270FB22E3735006434023510372AAC0037B50070
S31A00033FFF0AAA02EC02A500372A34043520FA039BE83735002E53
S31A00034014FA0317A4A500EC02372A277BB00A37BC03E8A50037CC
S31A000340292AAC0037650000FA039BE83735228EFA0399123F0480
S31A0003403E350427F734103FE0276F376A0004272500102512F5E7
S31A000340534EEA13F545EA14ED04950C37F072D4AA08950A17F273
S31A0003406872D3177272D2AA0627260006BC1037650006A508FA10
S31A0003407D039AB2376A0006AA08F553EA1337650006A508FA03EC
S31A0003409238DE376A0006AA08ED04951037F072D8AA0C950E172A
S31A000340A7F272D7177272D6AA0A2726000ABC103765000AA50CC1
S31A000340BCFA039AB2376A000AAA0CF557EA143765000AA50CFAA1
S31A000340D103384A376A000AAA0C37650006376700082776B60A46
S31A000340E63765000A3767000C2776378700A027260006BE16B694
S31A000340FB04ED08377D752FB20C2726000ABE06B656A50C37B8D1
S31A00034110752FB34EA50837B101F4AA18A506F3007300AA163798
S31A00034125BD03E8AD002725000237650016A518FA0304BCAA0EF5
S31A0003413AA50C37B101F4AA1CA50AF3007300AA1A37B503E8AAB9
S31A0003414F00272500023765001AA51CFA0304BCAA1EF501EA1216
S31A00034164B004ED08AD0EA50CAA1E37BC0003A51E372A6C0EB319
S31A00034179FE251337BC0003A50E372A6C1EB3FE25143765000ECA
S31A0003418EA51EFA039896AA10A51037B803E7B30A2612B70637F4
S31A000341A3352292FA039912B04027260010B60A2612B606373500
S31A000341B82296FA039912B02CE512370537650010FA033FCA3791
S31A000341CD350020FA0317A42613B706E5133705277BFA0317A443
S31A000341E22614B706E5143705277BFA0317A43F20350427F7344F
S31A000341F7103FE2276F376A001C7C12FA033C1437350020FA03C2
S31A0003420C17A43765001CFA0399123765001CFA03992E277B3724
S31A0003422131229CFA03991234103520A51CFA033E0434103520B6
S31A00034236FA039912173672B4B70C37350020FA0317A4376500AC
S31A0003424B1CFA034042FA039BD83F1E350427F734103FFC276F81
S31A00034260376A000017FD73C0B01EED021600B71C27260000B7AE
S31A000342750637650002FA033ECEB00437650002FA0341F6ED0209
S31A0003428ADD18AD02B6D63F04350427F734103FF8276F376A009A
S31A0003429F0237BD73C0AD06EC06CC00AC040600B71A3765000440
S31A000342B4A502FA03994027F6B71CED0427160018B70437DCFC6F
S31A000342C91837DCB0D237BC000AAC0037650004A502FA03999C08
S31A000342DEED04DC18ED069C0017FC73C0ED049C1817BD73C03F1D
S31A000342F308350427F734103FFE276F376A000027367360B71A95
S31A0003430817F5354F3705277B27743402350837DC37B10AB2372D
S31A0003431DDCDD00D500F832B33E37350002FA03C96A1733735D21
S31A0003433237650000FA03C8E2173672B4B70C37350020FA03C8A3
S31A000343478037650000FA034042EC00177C7DEAB60437350004AD
S31A0003435CFA03C8801731735DFA03C9C43F02350427F734103F41
S31A00034371E4276F376A0010AA12EC22AC14EC24AC16EC26AC18D1
S31A00034386EC28AC1AEC18AC00EC1AAC0217FC3492AC04376500B6
S31A0003439B14A516FA03390A37163787006827260010B702EC1070
S31A000343B00600B610274E37CCFC0637CCAC1037650010A512FA8D
S31A000343C503109037650010FA03429617FD73C0EC149C0AEC16C7
S31A000343DA9C0CEC189C0EEC1A9C1017FC08829C1217FC08849C37
S31A000343EF1417FC08869C161736354FB70434083520FA0342F8F5
S31A000344041736340FB704377573C0FA033ECE173634EDB718EC3E
S31A0003441918AC00EC1AAC0217FC34EEAC0437650014A516FA03C0
S31A0003442E390A17FA72BB3F1C350427F734103FFC276F376A0087
S31A00034443003401350837DCA10037DCAD02EC00C5003705277BE4
S31A00034458FA0399C23716B70C27230000EC006C02B5E237B500B7
S31A0003446D01B0FE27F53F04350427F734103FEE276F376A000222
S31A00034482AA04272500082725000A2725000CED02D500F1DFEAEE
S31A000344970627230002F85AB24A37B5005BAA003765000AA50C1F
S31A000344ACFA0304F2376A000AAA0CE5063705277B376A001027FD
S31A000344C125000EA50CA110AA0CA50AE30F630EAA0A272300087A
S31A000344D6ED08377D0004B6AEA50AED049A00A50C9A0237B50044
S31A000344EB01B0FE27F53F12350427F734103FE0276F376A00089E
S31A00034500AA0A34103540FA03447827F6B710376500087C04343B
S31A00034515103540FC04FA03447827F6B60227F57A0345BAAE0C23
S31A0003452A3765000C37B522AAFA03078E376A000EAA10ED0EAD70
S31A0003453F00ED10EC0C8D0237BD0052EC0A8D0037BD65C08D0269
S31A000345548502A002AA148500E2016200AA12ED128D00ED148DC2
S31A0003456902274E37CCFC0437CCAC163765001637B522AEFA038A
S31A0003457E078E376A0018AA1AED18AD04ED1AEC168D02ED04ECE2
S31A00034593268D00EC16CD02EC268D02850237B13480AA1E850075
S31A000345A8F35B73FFAA1CED1C8D00ED1E8D0237B500013F2035BE
S31A000345BD0427F734103FF8276F376A0002AA063765000E376A0F
S31A000345D20004376A000037650006A502FA039A70ED0237DCA133
S31A000345E70437DC150027210004BD0AED0237DCA10437DCD500E8
S31A000345FCF820B7DE37650004277027FB3717370527FF27FF279E
S31A00034611FF27FF27FF27FF27FF3F08350427F734103FFC276F41
S31A00034626AA0037BC0000275C37DCA10037DCD500EA02F81FB304
S31A0003463B3CF821B720F85FB71C3402350834043540375C2778B9
S31A00034650375CE502DA0037CCFC0137CC377C0009BFC6B01437B9
S31A000346657C0002BF0E3402350834043540375C2778375C1500F2
S31A0003467AB0FE27F53F04350427F734103FEC276F34023508AA9C
S31A0003468F10D50BF1E0F85BB24434083540FC02274E37CCFC08D8
S31A000346A437CCAC12341035207C0C376A0000277BA512FA0344DB
S31A000346B9F627F6B71EEC08AC00EC12CC02AC02EC0CAC04EC0E3F
S31A000346CEAC0637650010A51AFA03436E37B50001B0FE27F53F0D
S31A000346E314350427F734103FF2276F376A0000FA0308C0AA062D
S31A000346F8376500007C02FA0308C03401351037650006277427E7
S31A0003470D7427742774376000062774277427FB374C2778374C4A
S31A00034722373503E834043540FA0304CE376A0002AA04376500B9
S31A00034737007C05FA0308C0340135103404352027742774277842
S31A0003474C2774376A000A27FB371727F83717AA08A504A10AAA7C
S31A0003476104A502E3096308AA02ED00D507F853B60C3765000218
S31A00034776A504FA039AB2376A0002AA0437650002A5043F0E3519
S31A0003478B0427F734103FF2276F376A0000FA0308D0AA06376521
S31A000347A000007C03FA0308C0340135103765000627742774273E
S31A000347B5742774376000062774277427FB374C2778374C3735D1
S31A000347CA03E834043540FA0304CE376A0002AA04376500007C01
S31A000347DF06FA0308C0340135103404352027742774277827747A
S31A000347F4376A000A27FB371727F83717AA08A504A10AAA04A5C6
S31A0003480902E3096308AA02ED00D508F857B60C37650002A5046A
S31A0003481EFA039AB2376A0002AA0437650002A5043F0E350427EE
S31A00034833F734103FEA276F376A0008AA0AEC08C505F82E37866F
S31A000348480082C508EA14F84EB702F85337860074EC08C50FF8CA
S31A0003485D2E3786006AC512EA14F845B700F857B65CEC08C509FC
S31A000348723705277BC513370534013508FA0396CCEA14B7443735
S31A000348876500087C0137B50004FA03443A27F6B7323765000814
S31A0003489C7C0637B50002FA03443A27F6B720376500087C0A37BE
S31A000348B1B50005FA03443A27F6B70E376500087C1037B50002B4
S31A000348C6FA03443A27F6B60027F5B03C2723000837650008FA8E
S31A000348DB0346E8376A000CAA0E376500087C09FA03478E376A8D
S31A000348F00010AA12EC0CAC00A50EAA02EC10AC04A512AA063791
S31A0003490565000AA51CFA03436E37B500013F16350427F73410D9
S31A0003491A3FE8276F376A000EAA10A50EA11EAA12376500107C03
S31A0003492F0B37680012378201622502EC10C5003705277B37385D
S31A00034944002F378700A6BE1237380021378700E8378F0142377C
S31A00034959380029B7207A034A9C3738003D378700D2BE06373836
S31A0003496E003BB74C7A034A9C37380040378700727A034A9C2721
S31A00034983230010341035207C02A510FA034620277B27763787B7
S31A0003499801003402350837DCA11037DCD500F821378600EE37E6
S31A000349AD610010376A00107C0B376800123783007E7A034A9CF7
S31A000349C227230010EC10C509F82A378600CA37B50009AA003437
S31A000349D71035207C02A510FA0345C0EA16378700B2EC1037CCB9
S31A000349ECFC0937CCAC1027230010ED10EC1037CCFC0637CCACE2
S31A00034A0110376500107C0B376800123782008AD5063705277BA7
S31A00034A1637380068B70EBE063738002FB7067A034A9C373800F5
S31A00034A2B7AB66A3408352037B50006FA03443A27F6B75AEC10AB
S31A00034A40C5013705277BC50A370534013508FA0396E8277B27F3
S31A00034A5576B7183765000E7C07376A00003765001034103540CB
S31A00034A6AFC02FA0346843705B026376500107C1337680012B2B9
S31A00034A7F183765000E7C07376A00003765001034103540FC02D0
S31A00034A94FA0348343705B0FE27F53F18350427F73410276F37C6
S31A00034AA938004FBF0227FBFCB0B00C37380040BE0227FBFCD0C0
S31A00034ABEB00027FBFCBF350427F734103FB2276F376A000EAAD2
S31A00034AD310376500107C09A50EA154340227793520378200F602
S31A00034AE8EC10C500370534013508377D0027B704377D00603760
S31A00034AFD8600DEEC10C5083705AA4CC507370534013508376526
S31A00034B12004CFA0396CCEA4A378700C037BC0001AC4CED4C37CC
S31A00034B27DCA11037DCD500F1E4F863378200A82723004C376538
S31A00034B3C004C37380006BFDC2725004CED4C37DCA10E37DCD584
S31A00034B5100371FEA20F1B3F80237830080E520F85A3782007886
S31A00034B66F82F37830072F1C6F8063783006A275E37DCA14C3749
S31A00034B7BDCE520DA082723004CEC4C377C0005BFB8EC10C5019A
S31A00034B903705FCE4AA12E50CF840B306376500127C64376A001E
S31A00034BA512A51237B800C7B22EEC12377C00BDB30A37650012BA
S31A00034BBA3731FF42376A0012B008A51237B800B3B300FCB0AA67
S31A00034BCF12EC10C5023705FCE4AA1437B80045B30227F57A0397
S31A00034BE44DD2376500143738003BB3027CC4376A0014EC10C5CF
S31A00034BF9033705FCE4AA1637650012376A00242725002237B5F2
S31A00034C0EEA60AA002775A524FA0304F2376A0026AA2837B503B4
S31A00034C23E837650014372634013508AD2C2725002AA528A12C23
S31A00034C38AA1EA526E32B632AAA1CA51627F427F4A11627F4AAFD
S31A00034C4D4837650048376A00302725002EA51EA130AA1EA51CB5
S31A00034C62E32F632EAA1CE50DF840B30C3765001CA51EFA039AD0
S31A00034C77B2376A001CAA1EE50837053401350834083520FA03BF
S31A00034C8C4AA4AA32E50937053401350834083520FA034AA434F4
S31A00034CA1013508A53227F427F4A13227F4AA4837DCA14837DCBB
S31A00034CB6AD12E50A37053401350834083520FA034AA4AA34E545
S31A00034CCB0B37053401350834083520FA034AA434013508A5344B
S31A00034CE027F427F4A13427F4AA4837DCA14837DCAD14E50C37A6
S31A00034CF5053401350834083520FA034AA4AA36E50D370534016B
S31A00034D0A350834083520FA034AA434013508A53627F427F4A1AE
S31A00034D1F3627F4AA4837DCA14837DCAD16EC12AC3A27250038F9
S31A00034D343735EA60376A00002775A53AFA0304F2376A003CAA15
S31A00034D493E37B503E837650014372634013508AD42272500403D
S31A00034D5EA53EA142AA1AA53CE3416340AA18A51627F427F4A1B1
S31A00034D731627F4AA4837650048376A004627250044A51AA146FE
S31A00034D88AA1AA518E3456344AA18E50BF840B20C37650018A5BC
S31A00034D9D1AFA039AB2376A0018AA1AED0E37DCFC0737DCEC18F0
S31A00034DB2AC003765001A376A0002A51CAA04EC1EAC06277534E3
S31A00034DC7083540FA03436E37B500013F4E350427F734103FF857
S31A00034DDC276F376A0002AA042725000637BD0006AD00FA039A42
S31A00034DF15627F6B608ED02D506ED04D406F61EB70237BD00011C
S31A00034E06AD06A5063F08350427F734103FFE276F3402350827E1
S31A00034E1B7BB0223402351017C5FFFF3705AA0037B8000DB70E30
S31A00034E30BE0437B8000AB706B012A50037B80020B60A7CFF3407
S31A00034E45083540340227793520B2CA3408354027793402350867
S31A00034E5A340835403F02350427F734103FF0276F376A0002AA9B
S31A00034E6F0427365E16378700B6FA030D24AA0A378700ACED02A1
S31A00034E8437DCA10437DC3765000A34083540FA034E10AA0E37A4
S31A00034E99BC5E16AC0817FC5E167A034F2A376500067C0BA502CA
S31A00034EAEFC07FA034DD8371637860068376500067C04EC0685B6
S31A00034EC302FA030D24AA0CB604373522B2FA039AF6EC06CD02A3
S31A00034ED837DCFC0437DC37DCA10637DC3765000C34083540FA76
S31A00034EED034E103765000E340227793520B624376A000037655A
S31A00034F02000AA50CFA039A5627F6B612EC0637450000EC08376B
S31A00034F174A000037650006FA030F24B008EC06AC08CC00AC0684
S31A00034F2C3786FF743F10350427F73410276FFA03059237B60036
S31A00034F4103350427F734103FF6276F376A0002AA0437BD5E1630
S31A00034F56AD0817FC5E16B026376500067C0BA502FC07FA034D0E
S31A00034F6BD83716B60EED06DC00ED089C0037650006FA030F240D
S31A00034F80B006ED06AD08DC00AC06B6CE37650004FA030EE0AA6E
S31A00034F9506B74437650004ED06375A0002FC04376A000037659A
S31A00034FAA0002FA039A70EC0827060000B708ED08DD00AD082752
S31A00034FBF160000B6F027365E16B60CFA034F3637F134F037354B
S31A00034FD45E18FA030226ED06EC088D003F0A350427F734103F8D
S31A00034FE9FE276FB028ED00DD0017BD5E1637650000FA030FD0B4
S31A00034FFE1736340FB612373522B8FA039912376500007C04ED46
S31A00035013009502FA03130817FD5E16AD00B6C83F02350427F785
S31A000350283410276F3402350837DCFC0637DCD500F61E371FF1C5
S31A0003503DFF17181E003714D700DA00350427F734103FF6276FA7
S31A00035052376A0000AA02ED00D50DF601B65A37DCFC0E37DCAD40
S31A00035067047C15A502A100340227793520B2441606BC083765B1
S31A0003507C0000A502FA034E64B0343765000437B50001FA03252D
S31A00035091F03716B724ED04D506F601EA063765000437B531CAAF
S31A000350A6FA031234E506F780ED04D706DA0637650000A502FA5C
S31A000350BB034F463F0A350427F734103FF4276F376A0004AA063D
S31A000350D0FA030D24AA08376500047C0737BD8408AD0037BD009E
S31A000350E507AD0237B5FFFFFA039852AA0A37BD8408AD0037BD51
S31A000350FA0006AD0237650004FA039852AA0A27260008B71CA5DB
S31A0003510F04A10637650008FA034E1037BD8408AD00AA02376563
S31A000351240008A50AFA039852AA0AA50A3F0C350427F734103F47
S31A00035139FA276F273681EE3786005A273681ECB65237BD7DECB6
S31A0003514EAD00377D81ECB44617FD81EEEC008D0017BC81EE3706
S31A00035163CCFC0837CCAC00377C81ECB5E2B02AED00DD04AD02A1
S31A00035178EC00CC06AC0437650002A504FA0302743716B718EDE8
S31A0003518D00DD0017BD81EC17FD81EEEC008D0017BC81EE17FC95
S31A000351A281ECAC00B6C63F06350427F73410276FFA0350C417BC
S31A000351B7FD81ECB71237550002340227793520B60237B5000149
S31A000351CCB002DD00B6E627F5350427F734103FFA276F376A0073
S31A000351E100AA0217FC81EEAC04B756CC0017BC81EEEC0427059B
S31A000351F60000FA031052376500047C0437F53578FA03022637E7
S31A0003520B650000A502FA0350C4EC048A021736340FB60E37352C
S31A0003522022C0FA03991237650000A502FA03130837BD81EC2703
S31A000352353681ECB704DD0027160000B6F4EC049C003F0635042F
S31A0003524A27F734103FF2276F376A0002AA04FA035136376500AC
S31A0003525F02A504FA0351AE3716378601DA3765000237B500011A
S31A00035274FA0325F03716378601C8376500027C0737B50001FA2F
S31A000352890325F03716378601B4EC0237CCFC0E37CCAC0617C5A4
S31A0003529EFFFFF601B70027250006EC02C506F61EB7142726000F
S31A000352B306B702EC060606BD0837650002FA0350287A03540077
S31A000352C827260006378701763765000637B522C8FA031116376D
S31A000352DD1637870146EC06C506F780CA0637CCFC0737CCAC06D9
S31A000352F217C5FFFFF6013786014A7A03542AEC06C506EA0837E4
S31A000353078D01003765000637B522CEFA0311F83716B732E50853
S31A0003531CF61E378700C437650006FA035028E508EC06C404F629
S31A000353311EB738A502FC0E37650006340227793520B72837CCF1
S31A00035346FCF937CCAC067A0353E63765000637B522D4FA031157
S31A0003535BF83716B74CE508F61E3787007E37650006FA03502898
S31A00035370EC0437CCFC0737CCAC0A377C01FE378E00C4EC06370C
S31A00035385CCFC0737CCAC0CED0237DCA10437DC37DCA00637DCFA
S31A0003539AAD0037650006A50CFA039A703765000A376A0004B0F3
S31A000353AF323765000637B522C8FA0311F8371637860084376506
S31A000353C4000637B531E0FA0311163716B6123765000637B531D0
S31A000353D9CAFA0311163716B60E7A03544825083765000637B5E3
S31A000353EE31CAFA031234E508F601F780EC06C706CA06376500DD
S31A0003540302A504FA0351D8B038E508F601B6323765000627F548
S31A00035418FA0325F03716B624EC0637CCFC0737CCAC06376500F4
S31A0003542D067C07ED0437DCFCFF37DC34083540A102340227799C
S31A0003544235203783FEB63F0E350427F73410276F173581F41733
S31A000354573581F6173581F5373581F737B50100FA039A443504E4
S31A0003546C27F73410276F3402350834083540373500A5F8A1B7A5
S31A0003548104F81FB3003705277B27FB350427F73410276F17F502
S31A0003549681F637053401350837DC37B181F737DC27FBDA00173A
S31A000354AB3381F6350427F734103FF2276F376A0000AA0227253E
S31A000354C0000837650008373600FF3402350837DC37B181F73799
S31A000354D5DC27230008D500F8A13786005EEC00AC04EC02AC06C6
S31A000354EA37650008373600FF373181F7376A000AEC04C500371D
S31A000354FF052723000427230008277BFA03546EEA0CEC0AC500D8
S31A00035514E80CB62627210006B6C837650008373600FF34023562
S31A000355290837DC37B181F737DC1600B702D500F8DBB60237B5BB
S31A0003553E0001B008EC08377C00FF3783FF7427F53F0E350427FA
S31A00035553F734103FFA276F376A000034013510ED0037CC910094
S31A0003556837CC37550000376A000234043540340227793520B467
S31A0003557D4AED02D500F820B218376500027C01ED00375A000087
S31A00035592376A000234043540340227793520B5D8ED003755007A
S31A000355A700376A0002B00E17C5FFFFF820B21237CCFCFF37CCCE
S31A000355BC3765000234043540340227793520B5DE34043540ED2E
S31A000355D10090003F06350427F734103FEE276F376A000AAA0C28
S31A000355E6A518341035207C18A51AFA035554AA1A378700C037DF
S31A000355FB650018FA0354B23716378600B2373500DBFA0354902E
S31A0003561017F581F617FA81F534103520A50AFA031090AE0E26AB
S31A0003562500B716EC0EC500F82DB70E37052723000E277BFA03BE
S31A0003563A5490EC0E0600B6E22726000CB7283735002FFA0354B2
S31A0003564F90EC0C37CCFC0537CCAC0EEC0CC500F820B30437052C
S31A00035664277BFA0354902723000CEC0C6C0EB5E2373500A1FA3F
S31A00035679035490274E37CCFC1837CCAC10EC10CD00D500370507
S31A0003568E37DCFC0137DC8D00277BFA03546E3705277BFA0354BE
S31A000356A3902721001AB6D8F50117FA81F4373581F037B507D04D
S31A000356B8FA0302343F12350427F734103FFC276F173681F437EB
S31A000356CD8700BE27367360378600B6377581F037F581F2FA031E
S31A000356E202743716378700A437350004FA03C96A17F581F5EA79
S31A000356F700E5003705277B3402350837DC37B181F737DCD50004
S31A0003570C3705277BFA03C8802300E50017F881F6B63CFA03C916
S31A00035721C4373581F037B507D0FA030234F50117FA81F417F54B
S31A0003573681F63705277B3402350837DC37B181F737DCF501EA27
S31A0003574B021600B70217F581F6EA02E50217FA81F5B02EFA03B7
S31A00035760C9A427F6B68EFA03C9C417F581F437BD07D0F802B6D7
S31A000357750037BD00FA373581F034083540FA030234F50217FA5F
S31A0003578A81F4173381F53F04350427F734103FF8276F376A0080
S31A0003579F00AA022736736037860094173681F43786008C373548
S31A000357B40004FA03C96A1733735DED0037DCFC0737DC34083502
S31A000357C920FA0312C83735003EFA03C88037650000FA0312C869
S31A000357DEFA03C9A4AA0437B80001B34A37650000A502FA030D5B
S31A000357F324AA06B73CEC0617C5FFFFF8F0B63237350020FA03AC
S31A00035808C88027210004ED0037DCA10237DC37DCA00637DC3735
S31A0003581D65000434083540340227793520B3FEAD043765000624
S31A00035832A504FA03C93A1731735DFA03C9C43F08350427F7343B
S31A00035847103FD8276F17FC319417BC31961736354FB71437350C
S31A0003585C0004FA03C96A3735319837F53194FA03C90AFA03C93E
S31A00035871C4273631943787014837753194373800043786008CFF
S31A0003588617F5319BF823378600823735319837B50003FA03446D
S31A0003589B3A27F63787007017FC31B2AC0617FC31B4AC0837BC23
S31A000358B003E8AC002725000237650006A508FA0304BCAA0C270C
S31A000358C525000A37BC03E8AC002775A50CFA0304F2376A000E1D
S31A000358DAAA1037353198FA039AC6AA14371727F83717AA12A58A
S31A000358EF10A114AA18A50EE3136312AA16EC1617BC31B2EC187A
S31A0003590417BC31B4273531B6273531B87A0359BC37753194370B
S31A00035919380007B63C17F5319EF823B6343735319837B5000638
S31A0003592EFA03443A27F6B7241735319E37353198FA03790E37DD
S31A000359436A001CAA1EEC1C17BC31B2EC1E17BC31B4273531B635
S31A00035958273531B8B05A3775319437380003B65817F5319AF822
S31A0003596D23B6503735319837B50002FA03443A27F6B7403735D5
S31A000359823198FA039AC637B80018B22E277B2774277427742760
S31A00035997743402350837DC37B131AC37DCDC4617BC31B2DC4824
S31A000359AC17BC31B4DC4A17BC31B6DD4C17BD31B8FA0316102715
S31A000359C13531943F28350427F734103FFE276F250017F5355043
S31A000359D63705277B37380001B70437380002B70EB04025001748
S31A000359EBF531A8F82AB636F501EA00B030FA0306082500371685
S31A00035A00B600F501EA002600B70417F52C76F701B00217F52C81
S31A00035A1576F70217FA2C7617F52C76F60317FA2C76F803B7FE47
S31A00035A2A2500E50037053F02350427F73410276F7CFF373800BC
S31A00035A3F27378200E627743402350837DC37B1232037DCDD0047
S31A00035A545B035A5837B522DA7A035B30F50117FA72B537B522F8
S31A00035A69E47A035B3037B522EC7A035B30FA03544EF50217FA8A
S31A00035A7E735C27357DEA173572B9173572B837B522F27A035BB3
S31A00035A933037B522FA7A035B30377573607CFF377A73602736DA
S31A00035AA87DEAB70C17FD7DEADD1817BD7DEAB7001600B6103741
S31A00035ABDF573C037FA7DEA17FD73C01600B60027357DEA377589
S31A00035AD27DEAB6003735230027FBB04E37B52306B048FA0321BF
S31A00035AE7E837F572D237FA72DE37F572D437FA72E037F572D65F
S31A00035AFC37FA72E237F572D837FA72E437F572DA37FA72E637D2
S31A00035B11F572DC37FA72E8F50117FA72B917FA72B817FA72B503
S31A00035B2637B5230CB00037B52316350427F734103FFE276FAA59
S31A00035B3B001736354FB712FA03C96A27260000B70437650000DE
S31A00035B50FA03C8E2FA03C9C43F02350427F73410276FFA035A3D
S31A00035B653637350004FA035B343735736237B503E8FA030234A5
S31A00035B7A350427F73410276F27367360B61AFA0359CA37163738
S31A00035B8F87006E37BD000117BD736037350001FA035B5E7A03C7
S31A00035BA45C02FA0359CA3716B7143775736237F57364FA0302CA
S31A00035BB9743716B740377573607C01B01037F5736037B8000963
S31A00035BCEB210277B2774277427782774377A7360FA035B5EB0FB
S31A00035BE31A3775736237F57364FA0302743716B70A3735000415
S31A00035BF827F5FA035B3427357360350427F734103FFC276F3418
S31A00035C0D0235081600B73AD500F82DB62A17D5FFFFF1D0EA02C2
S31A00035C22D501F1D0EA00E502F809B220E500F809B21A1602B6A9
S31A00035C3716E502E800B310E000EA02F130DA01B00637DCFC0119
S31A00035C4C37DC1600B6BE3F04350427F734103FF0276F376A0059
S31A00035C610AAA0CED0CB008ED0E1606BC5037DCFC0737DCAD0EAD
S31A00035C7617D5FFFFF601B7E6B03EED0E37DCFCF937DCAD0E349F
S31A00035C8B103520A50EFA0310903410352037B522C8FA03994001
S31A00035CA027F6B71A34103520FA035C063765000A34103540FAA7
S31A00035CB50312343765000A7C07376A000AED0E6D0CB2B4A50A2B
S31A00035CCA3F10350427F734103FFE276F376A000034013510F5EF
S31A00035CDF3AED00DA00272300003765000034043540FA03109076
S31A00035CF43765000037B52370FA039B62376500007C0937B5234D
S31A00035D097AFA03995AAA00B01CED08D5003705277BFA039B2A32
S31A00035D1E3716B718ED08D500ED00DA00272300082723000037E7
S31A00035D3365000A2721000A2776B6D0A5003F02350427F73410ED
S31A00035D483FF2276F376A0004AA06373501FEFA030EE0AA0837E2
S31A00035D5D8700AEEC0837CCFC0437CCAC0A37BD21D4173633EAF0
S31A00035D72B70037BD33EA3765000A34083540FA031234EC0A3784
S31A00035D87CCFC0737CCAC0A3765000A37B531CAFA031234EC0AB0
S31A00035D9C37CCFC0737CCAC0AED0437DCFC0E37DC3765000A342F
S31A00035DB1083540FA035C58AA0AEC0A17C5FFFFF70117CAFFFF4B
S31A00035DC6F503CA002723000AF5F0EC0ACA002723000AED043788
S31A00035DDBDCFC0737DCA506AA00EC14AC023765000A340835405E
S31A00035DF0FA035CD0AA0AED0A37DCFCFC37DC37DCA00837DCECE9
S31A00035E05088D0237650008FA030FD03F0E350427F734103FFC45
S31A00035E1A276F376A0002277BEC0AAC00A502FA039A70ED023719
S31A00035E2FDCA10A37DC15002721000ABD38ED0237DCA10A37DC9F
S31A00035E44D500F820B7DE2726000ABF24ED0237DCA10A37DCD5EF
S31A00035E5900F830B6162721000AED0237DCA10A37DCD500F82D2B
S31A00035E6EB6041500B00027230002EC02C500F820B7F03765003D
S31A00035E8302FA0399F6A5023F04350427F734103FFA276F376A7E
S31A00035E980000AA02ED02D5003705277BFA0399D6EA04ED00D582
S31A00035EAD00E804B60A3716B7062723000027230002B0D8277567
S31A00035EC2ED001600B610ED021600B706D500F820B700F82CB6B9
S31A00035ED7003735000127FB3F06350427F734103FFC276F376ACC
S31A00035EEC000037BD3551AD02B00027230002ED02D500F820B7E0
S31A00035F01F0F82CB7EC37650000A502FA035E903716B70E37B59F
S31A00035F160001B01CED02D500F82CB70C27230002ED021600B7ED
S31A00035F2B08D500F820B6E4ED021600B6BE27F53F04350427F79A
S31A00035F4034103FF8276F376A0000AA02ED02D5003705277BFA49
S31A00035F550399D6EA04ED00D500E804B60A3716B70C2723000006
S31A00035F6A27230002B0D8ED001600B62027250006ED021600B75E
S31A00035F7F0C3765000237B52380FA03994027F6B60237BD00012B
S31A00035F94AD06A506B0FE27F53F08350427F734103FE2276F37F7
S31A00035FA96A000EAA10E527EA12EC0E37CCA12437CCAC1437657F
S31A00035FBE00107C0B37680014B20AEC10C500F83AB602C50AF84D
S31A00035FD33AB72A27F57A036166A518FC01AA1CA514A01834010F
S31A00035FE8350837DCFCFF37DCAD003765000EA51CFA035D46EC99
S31A00035FFD18AC147A03607AED1037DCFC0137DC37B50009AA0098
S31A00036012341035207C0434083540FA035E16AA16A510FC0BAA0F
S31A00036027103765001637B531CAFA035F40EA1AB61C376500168E
S31A0003603C37B531E0FA035F403716B60C3765001637B53402FAD0
S31A00036051035F403716B738EC1437CCFCFF37CCAC186C10B5104D
S31A00036066EC18C500F87B3787FF6A27210018A518A810B4E83711
S31A0003607B65000E7C07EC10AC00A514A01034013508AD0227F5C3
S31A000360907A03615E2612378700C63765001637B52384FA03991F
S31A000360A54027F6B71C3765001637B52388FA03994027F6B70CAE
S31A000360BA3765001637B5238CFA03994027F6B620EC1437CCFCB3
S31A000360CFFF37CCAC186C1037850066EC18C500F87BB7522721C2
S31A000360E40018A518A810B4EAB05037BC0003AC003765001637E8
S31A000360F9B52390FA039972277B2776B634EC16C5033705277B48
S31A0003610EFA039B2A3716B724EC1637CCFC0437CCAC161736353D
S31A0003612351B7180600B71437650016FA035EE43716B608B0269B
S31A00036138EC18AC14B0002725001627260016B7163765000E7C1D
S31A0003614D07A510AA00A514A01034013508AD02A516FA0355DA5D
S31A0003616237B500013F1E350427F734103FDE276F376A0000AA3C
S31A000361770225042725000AED00D500EA20F820B704F82BB70010
S31A0003618CF82DB60E2504ED00D50027230000F82DB600F501EA1C
S31A000361A10437650000FA039AC6AA06ED00D5003705277BFA0396
S31A000361B699C23716B70227230000B0E6ED00D500F82EB6503765
S31A000361CB351770376A000827230000ED00D5003705277BFA036A
S31A000361E099C23716B73427260008B72EED00D50037053401356C
S31A000361F51037CCFCD037CC340435403765000837253401351083
S31A0003620A37CCA10A37CCAC0A37BC000AA508372AAC08B0B037B9
S31A0003621F65000637B5EA60FA0304CE376A000CAA0EED0AAD12D6
S31A0003623427250010A50EA112AA16A50CE3116310AA1437650058
S31A0003624914ED02375A0000A5169A022604B726DD00AD18376507
S31A0003625E0016376A001A37650018A516FA039AB2376A001CAA32
S31A000362731E3765001CED02375A0000A51E9A023F22350427F7A0
S31A0003628834103FFE276F37BD0040AD0037B50067FA03050A3F62
S31A0003629D02350427F734103FDE276FAA0E37610028376A001466
S31A000362B23765000E7C0637680014B21437B50006AA00376500F1
S31A000362C70E37B52394FA039A56277B2776B70227F57A0363AE79
S31A000362DCA50EFC06AA10ED10AD0EA814B40EED0ED500272300E5
S31A000362F10EF82CB702A50EA814B5EAED0EAD126D14B40EED0E9E
S31A00036306D5002723000EF82CB702A50EA814B5EA3765000E7C3B
S31A0003631B04376800143782007E3765000E37B50004FA03443A61
S31A0003633027F63787006C3765000E37B50004FA039E70AA16B6ED
S31A000363450237B50001AA16275E37DCFC0637DCAD18376500106D
S31A0003635AA518FA03616C275E37DCFC0A37DCAD1A37650012A5D3
S31A0003636F1AFA03616C37650016FA036288277BA506AA1CED187B
S31A00036384DD02AD1EA50AAA00ED1ADD02AD02376A000437650022
S31A000363991CA51EFA03390AEA20B702F50117FA72B537B50001E9
S31A000363AE3F22350427F734103FF4276F376A0004AA06FA030DAD
S31A000363C324AA081736340FB60637650004A506FA0313081736EA
S31A000363D8354FB70637650004A506FA035796272600083787011D
S31A000363ED14EC0817C5FFFEF8033786010817C5FFFFF8F0378671
S31A0003640200FE173672BAB63E376500047C0727F5FA0325F03789
S31A0003641716B72E37B58408AA00ED0437DCA10637DC37DCA008D1
S31A0003642C37DCAD023765000837B5FFFFFA039852277B277037AB
S31A00036441787300B602F50117FA72BAF5FF17FA72BB173634882C
S31A00036456B71C37650004FA03265C3716B710EC06AC0027250038
S31A0003646B0237650004A508FA035FA2B046A506AA0037650004DB
S31A00036480A508FA034918EA0AB634EC06AC0037650004A508FA30
S31A00036495034AC8EA0AB622A506AA0037BC0001AC023765000471
S31A000364AAA508FA035FA2EA0AB60AA506AA0037650004A508FAD9
S31A000364BF0362A2FA0316423716B63617F534ED3705277B3738B0
S31A000364D40001B70437380002B712B02017F572BBF801B61837AD
S31A000364E9650004A506FA03504CB00C173672BBB7063765000455
S31A000364FEA506FA03524C3F0C350427F73410276F2779340235B3
S31A0003651308377D00B4BF0437DC37B1FE9837DC377DFF4CBC04D4
S31A0003652837DC37B1016837DC34083540350427F734103FE82744
S31A0003653D6F377572CA37702C7A376A000227250004273672DCFE
S31A00036552B706377572DCFA031EE0AA0427260004B72837B503AC
S31A00036567E8AA0037650004A502FA03050A34013510340435202A
S31A0003657C377172FC377A72FC37CC37F172FE37CC17BC72FE27C4
S31A0003659136345CB75C273672DCB756273672F8B750377572DA95
S31A000365A637F572FAFA03650AAA06377572DCFA031EC6340135DE
S31A000365BB1027260006B730377C0000B72A3775345C27FB372A25
S31A000365D0AC0837650006FA039AA4277BED0837DCFC0137DC342E
S31A000365E5083540340227793520B302F50117FA72B5273634E894
S31A000365FA378701AC2725000A2725000C27362C7EB7542726000B
S31A0003660F04B74EED02377D09C3B246377572DA37F52C7CFA0334
S31A00036624650AAA0AB7363765000AFA039AA4AA1437650014FAFF
S31A000366390396843401350837650004372527F427F4AA0C37BCD9
S31A0003664E000AA502372AA50C372AAC0C2726000ABC00272200F6
S31A000366630C273635BCB71C3765000AFA039C603735239CFA0325
S31A00036678991237650004FA039BE8373523A0FA03991237752C8A
S31A0003668D847C013736000F376A0014377A2C84A514B016376541
S31A000366A200023731FC18376A000237F52C84FC0137B6000F37AD
S31A000366B7FA2C8427F437B12C86AA163765000CED16375A00006A
S31A000366CCA50237B805DBB2C8273635BCB70C373523A8FA0399E2
S31A000366E1123765000CFA039C60ED0C17BD2C823765000437385E
S31A000366F600023783006237BC0003A504372AAC0E37752C84371B
S31A0003670B6A0010377C0010B30237B50010AA0E272100103765D6
S31A0003672000103736000F376A0010A51027F437B12C86AA1237C1
S31A00036735752C82ED1237510000377A2C82273635BCB70E3735BE
S31A0003674A23A8FA039912ED1237550000FA039C602721000EB62E
S31A0003675FB6273635BCB710373523AAFA03991237752C82FA0319
S31A000367749C60FA039BD837752C82FA039AA437F834E8B302F511
S31A000367890117FA2C8037752C82FA039AA437F834EAB20C173647
S31A0003679E2C80B702F50117FA72B517352C8017FD72C817BD2C04
S31A000367B378377572CA377A2C7A37F572DA37FA2C7C17FD72DC5E
S31A000367C817BD2C7E3F18350427F734103FF8276FFA03164237EA
S31A000367DD16B66CFA03259A3716B6642736345AB72C3775345A3B
S31A000367F2FA031AD2376A0000AA02A50237F172C2AA06A50017E4
S31A00036807F372C1177372C0AA0437650004A506FA0302743716D8
S31A0003681CB72E173672B5B62227363398B70C377572C437F572C2
S31A00036831C6FA0302743716B60C27363396B70C377572FC37784F
S31A000368463396B30237B50001B0FE27F53F08350427F734103FDE
S31A0003685BFE276FFA030DCAAA00B712376500007C04ED009502A4
S31A00036870FA0363B437650000FA030F463F02350427F734103FED
S31A00036885EA276FAE0437650004FA030210ED0017BD72C8ED0428
S31A0003689ADD0217BD72CAED0017BD72C417FD72CA17BD72C63767
S31A000368AF75345AFA031AD2376A0006AA08A502A008AA0CA500DC
S31A000368C4E2076206AA0AED0A17BD72C0ED0C17BD72C2377534D3
S31A000368D996FA031AD2376A000EAA10A502A010AA14A500E20F0E
S31A000368EE620EAA12ED1217BD72BCED1417BD72BE3F16350427A5
S31A00036903F73410276F173572B5273572FC37F53398373572C4CF
S31A00036918FA030226350427F734103FFC276F377572D037380073
S31A0003692D02B60237B50001B02E377572D037380001B70617F5A0
S31A0003694272B6173572B6B01837F572CAFC32AA0237F572C8F338
S31A00036957007300AA0037650000A502FA03027437053F04350497
S31A0003696C27F73410276F7C1637BC002D27FB372A34043520272C
S31A00036981743402350837DC37B123B237DC3755000027FB350447
S31A0003699627F734103FD2276F376A0008AA0AED0A950237B165A2
S31A000369ABC0AA0E9500F3527300AA0C37B509C4AA003410352057
S31A000369C07C04376A00023765000CA50EFA0304BC277B376A003B
S31A000369D506376A00122725001037BD00F0AD00341035207C06E3
S31A000369EA376A00022775A512FA0304BC277BF141ED08DA01A593
S31A000369FF06AA162725001437BD0018AD00341035207C06376ADF
S31A00036A1400022775A516FA0304BC277BF130ED08DA03275E37FD
S31A00036A29DCFC0637DCAD18D501F141ED08DA05A504AA1C272502
S31A00036A3E001A37BD00FAAD00341035207C04376A00022775A588
S31A00036A531CFA0304BC277BF130ED08DA073765000437BC000B15
S31A00036A6827FB372A34043540F141DA09ED0A950637B1CB80AA5C
S31A00036A7D209504F3A47300AA1E37B51388AA00341035207C0426
S31A00036A92376A00023765001EA520FA0304BC277B376A00063787
S31A00036AA76A00242725002237BD00F0AD00ED18AD022775A5242B
S31A00036ABCFA0304BC277BF141ED08DA00A506AA28272500263736
S31A00036AD1BD0018AD00ED18AD022775A528FA0304BC277BF13088
S31A00036AE6ED08DA02ED18D501F141ED08DA04A504AA2C27250016
S31A00036AFB2A37BD01F4AD00341035207C04376A00022775A52C94
S31A00036B10FA0304BC277BF130ED08DA063765000437BC00152743
S31A00036B25FB372A34043540F141DA083F2E350427F734103FF8F6
S31A00036B3A276F17FD72D2AD0017FD72D4AD0217FD72D6AD041775
S31A00036B4FFD72D8AD0634103540FA0369983F08350427F7341095
S31A00036B64276F1735735C37350001FA03C96A173672B9B704375B
S31A00036B79350005FA03C880FA03C9C4350427F734103FF6276F8F
S31A00036B8EF50117FA735C34103520FA036B3637350001FA03C9A9
S31A00036BA36A1733735D273672DCB7323410352037B50006FA0334
S31A00036BB8C90A37350020FA03C880377572DCFA031EC6277BFAA4
S31A00036BCD039BE8373523DCFA03C8E2377572DAFA03696E277BA4
S31A00036BE2B01C3410352037B5000AFA03C90A37350020FA03C819
S31A00036BF78037357304FA039CFA3735228AFA03C8E2173672B953
S31A00036C0CB70437350005FA03C8801731735DFA03C9C427367D7D
S31A00036C21EAB70237757DEAB00817FD73C01600B704340835203E
S31A00036C36FA0342F83F0A350427F73410276FFA0397A837B8FF65
S31A00036C4BFFB7141736340EB704277BFA03AC1EB0E43705277B3C
S31A00036C60FA032464B0DA350427F734103FFE276F377572D03774
S31A00036C75380002B600FA036B88173672B4B6083735000137B597
S31A00036C8A23E2FA035B34FA03AC80FA036882173672B7B70E17F9
S31A00036C9F3572B7FA0365381736354FB700FA036B88173635BE27
S31A00036CB4B628FA03166A3716B604FA0367D23716B71817F534CE
S31A00036CC9EDF802B708F50117FA35BFFA031036B000FA0335B433
S31A00036CDEFA036904FA036858FA036C40FA0325B41736354FB76A
S31A00036CF30E1736735CB708FA0325863716B700FA036B621736D7
S31A00036D083550B700FA035B7E3775319437783196B700FA035868
S31A00036D1D4627365E16B71037755E1837F55E1AFA0302743716F4
S31A00036D32B700FA034FE62725000017F535BEF801B20E373500EA
S31A00036D4701FA0317003716B70237B50004AA00FA0369203716A6
S31A00036D5CB704A50037B70002AA00173672BAB704A50037B70058
S31A00036D7101AA0037650000FA0306F2173681F4B7061736354F78
S31A00036D86B700FA0356C2FA030A2A7A036C983F02350427F734A5
S31A00036D9B103FD8276F373501FEFA030EE0AA243787009417F59B
S31A00036DB034133705277B37380001B70E37380002B7383765006F
S31A00036DC524FA030F247A036E44376500247C0437B523F4FA03ED
S31A00036DDA1234376500247C0B37B531CAFA031234ED24D511F7F6
S31A00036DEF01DA11F503DA1237B5000F9A02B02234103520FA03B7
S31A00036E043510376500247C0434103540FA032C4CED249A0237D9
S31A00036E1965002434103540FA032954FA0303B83775341EFA03EC
S31A00036E2E029437650024FA0303CEFA0303E427F6B6F4FA030377
S31A00036E43EE3F28350427F734103FF6276F376A0000FA03164280
S31A00036E583716B704373523F8FA039AF637350001FA03069C37BD
S31A00036E6D3500E1FA03A13617FD31B6AD0217FD31B8AD04377519
S31A00036E8231B6377731B82776B60817FD31B2AD0217FD31B4ADCD
S31A00036E970437650002A504FA0315AC377531ECFA03029437350C
S31A00036EAC00D1FA03A136173634F5B604FA03A16627F6B70A17FA
S31A00036EC1F531C63705277BFA03A174B0022775FA0306F23775E8
S31A00036ED631EEFA03029427260000B700FA03140427363462B729
S31A00036EEB0437753462FA031420FA03166A3716B6F427363462AB
S31A00036F00B7022775FA03142017363413B706173631CAB700FAA3
S31A00036F15036D9A37350003FA03A17437350002FA030294373566
S31A00036F2A00E1FA03A13617FD31B2AD0617FD31B4AD08376500A0
S31A00036F3F06A508FA03157C2775FA03069C3F0A350427F73410D4
S31A00036F54276F27F5377531B6377731B82776B71A377531B6370B
S31A00036F697831B2B606377531B8377831B4B706173631F0B700E8
S31A00036F7E37B50001350427F73410276F17F531C6370537B800A9
S31A00036F9301B714BE0227F6B714B00237B80002B7002775B00CBA
S31A00036FA837350004B00637350006B00037350007FA0306F235E6
S31A00036FBD0427F734103FFE276FFA0302A8AA0037F831C0B40058
S31A00036FD22775B02037650000377831C2B40237350004B01037DA
S31A00036FE7650000377831C4B40237350006B00037350007FA033B
S31A00036FFC06F21736354FB70437650000FA03CA1E3F02350427D1
S31A00037011F734103FFC276F37350001FA03064E373500E1FA034D
S31A00037026A13637BD000117BD82F8273582FA273582FC273582A2
S31A0003703BFE273583003F04350427F734103FFE276F2775FA0310
S31A00037050064E37350061FA03A136273582F8273582FA273582A1
S31A00037065FC3F02350427F73410276F173631C8B704FA03A16E92
S31A0003707A3705B00EFA0302A8277B27F5377831BEB30037B5005C
S31A0003708F01350427F734103FF0276F273682F8B748273582FED0
S31A000370A427358300FA03706C27F6B756377582FA377782FC2771
S31A000370B976B60837F531DA373582FAFA03023417FD82FAAD00F6
S31A000370CE17FD82FCAD0237650000A502FA0302743716378700A2
S31A000370E38AFA0370467A037170FA0302A837F831DEB3083735E8
S31A000370F882FE37B501F4FA030234FA03706C27F6B70627358255
S31A0003710DFA273582FCB058377582FA377782FC2776B60837F5AD
S31A0003712231DC373582FAFA030234377582FE377783002776B776
S31A000371371617FD82FEAD0817FD8300AD0A37650008A50AFA033D
S31A0003714C02743716B71617FD82FAAD0C17FD82FCAD0E37650063
S31A000371610CA50EFA0302743716B700FA0370123F10350427F7B5
S31A000371763410276F37F53418FA030226350427F734103FFE2785
S31A0003718B6FFA030DCAAA00B712376500007C04ED009502FA0393
S31A000371A0130837650000FA030F463F02350427F734103FFA278C
S31A000371B56F376A000037350003FA03C96A1733735DEC00CC003B
S31A000371CAAC02EC00CC02AC0437650002A504FA03788A373500DD
S31A000371DF20FA03C88037350006FA03C88037350020FA03C880A5
S31A000371F417F531C63705277B27743402350837DC37B10A2C3726
S31A00037209DC37550000FA03C8E21731735DFA03C9C43F06350438
S31A0003721E27F73410276F37350003FA03C96A37352404FA03C862
S31A00037233E2FA03C9C4350427F734103FF6276F1736354FB704DF
S31A00037248373531B2FA0371B034103520FA037176FA037186FA50
S31A0003725D03166A3716B73AFA0370122775FA030668FA036F86DA
S31A0003727227250004273682F8B70AFA036F523716B70237BD005E
S31A0003728701AD0437650004FA036E4A37350001FA0306683410C6
S31A0003729C3520FA037176FA036FC0FA037094273682F8B60434A9
S31A000372B1103520FA037176173631F1B712ED00AD06ED02AD08FA
S31A000372C637650006A508FA0302743716B614FA036C403775314B
S31A000372DB94377831963787FF72FA0358467A0372583F0A3504F8
S31A000372F027F734103FFA276F376A0000AA02FA03164237163729
S31A000373058600A0EC02377C0015378F0096EC00C50DF6013786C0
S31A0003731A008C3765000037B50001FA0325F037163786007AECBE
S31A0003732F0037CCFC0E37CCAC04376500007C15B04EEC04060659
S31A00037344BD203765000437B50001FA0325F03716B750EC04C5A6
S31A0003735906F780CA0637650000A502FA031052B03CEC04C50680
S31A0003736EF601B6343765000437B50001FA0325F03716B624EC6E
S31A000373830437CCFC0737CCAC04376500047C07ED0237DCFCFF0F
S31A0003739837DC34083540A1003402277935203783FF943F063580
S31A000373AD0427F734103FFA276FFA030DCAAA02B726ED0237DC2E
S31A000373C2FC0437DCAD04ED02950237650004FA0372F2ED0295DE
S31A000373D70237650004FA03130837650002FA030F4627250000A2
S31A000373EC17F535BEF801B21037350001FA0317003716B7043709
S31A00037401350004376A0000273635C2B708376500003737000274
S31A00037416376A0000173635C0B7083765000037370001376A000A
S31A0003742B0037650000FA0306F27A0373B63F06350427F734102C
S31A000374403FFA276F376A000037B50019EC00374500007C01379D
S31A000374554A000037380018B30027050000EC0037450000277466
S31A0003746A2774277427743402350837DC37B131AC37DC37550049
S31A0003747F46375700482776B600FCFFB6BC37752CA63734000228
S31A00037494377A2CA6FA0306F2FA037012EC0037450000277427B9
S31A000374A974277427743402350837DC37B131AC37DCDC46AC02ED
S31A000374BEDD48AD0437650002A504FA03157C3F06350427F73435
S31A000374D310276FFA037186FA036C403775319437783196B700BA
S31A000374E8FA035846FA03166A3705350427F734103FDE276F37AD
S31A000374FDBCFFFFAC103410352037B50010FA039A4417FC31B295
S31A00037512AC0017FC31B4AC0217FC31B6AC0417FC31B8AC06179A
S31A0003752736354FB700FA037220341035207C10FA03743E373506
S31A0003753C0032FA030294FA0374D227F6378600C8FA037094FA8C
S31A0003755103706C27F6B7D437F531DA341035207C12FA03023404
S31A00037566EC12AC16EC14AC1837650016A518FA0302743716B69E
S31A0003757BA6FA0374D227F63786008EFA037094273682F8B6D241
S31A000375903765001027742774277427743402350837DC37B13126
S31A000375A5AC37DCDC46AC00DC48AC02DC4AAC04DC4CAC06DC4E8F
S31A000375BAAC08DC50AC0ADC52AC0CDD54AD0E1736354FB704348B
S31A000375CF103520FA0371B0FA0374D227F6B634FA036FC0FA03A8
S31A000375E47094273682F8B716EC12AC1AEC14AC1C3765001AA5FA
S31A000375F91CFA03027437163786FF20B0CC37F534163410352031
S31A0003760E7C12FA030226B0BCEC0017BC31B2EC0217BC31B4EC0B
S31A000376230417BC31B6EC0617BC31B83F22350427F734103FFEA4
S31A00037638276F3410354037350001273635C2B7267C0117FD3581
S31A0003764DC237510002340135108D0037F535C234013510CC0063
S31A0003766217BC35C227363382B7D237783382B5CC34013510271F
S31A00037677050000A5003F02350427F73410276F37358302FA03EB
S31A0003768C0210173635BEB72EFA03178A3716B62617F531C7F8E6
S31A000376A101B60A173635BFB704173535BFFA0335B4273635C294
S31A000376B6B70637BD773017BD240AB000173535BE350427F734E2
S31A000376CB10276F2775FA0317003716B61637BD76F817BD240ACE
S31A000376E037358306FA03025637B80064B300FA03768227F535F6
S31A000376F50427F73410276F2775FA0317003716B70E37358306C4
S31A0003770AFA03021037BD76CA17BD240AB00E37358302FA03026E
S31A0003771F5637F831D6B300FA03768227F5350427F734103FFC26
S31A00037734276FF50217FA35BE37350001FA0306B637F531B6AAC3
S31A000377490037F531B8AA02377531B6377731B82776B60837F5B0
S31A0003775E31B2AA0037F531B4AA0237650000A502FA0315AC378B
S31A00037773B5778637FA240A377531EC27FB3F04350427F734101E
S31A00037788276FFA0316423716B7043735207AFA039AF6373500F1
S31A0003779D51FA03A136173634F5B604FA03A16627F6B70A17F58B
S31A000377B231C63705277BFA03A174B0022775FA0306F2FA03038F
S31A000377C7B837BD77DE17BD240A377531EE27FB37F1341E350401
S31A000377DC27F73410276FF50317FA35BE273635C2B706FA037617
S31A000377F134277BFA0303CE37B5780637FA240A27F5350427F79A
S31A000378063410276FFA0303E427F6B618F50417FA35BE37350052
S31A0003781B03FA03A17437B5783437FA240A37B50002B0FE27F58B
S31A00037830350427F734103FFC276F37350061FA03A13617FD31E8
S31A00037845B2AD0017FD31B4AD0237650000A502FA03157CFA0350
S31A0003785A03EE2775FA0306B63715273635C2B7FEF50117FA3539
S31A0003786FBE37358302FA03021037BD76F817BD240A37B50002EB
S31A000378843F04350427F734103FEE276F376A000C275E37DCFC04
S31A000378990C37DC9A023410352034083540FA03098227250010E8
S31A000378AEE500F830B616EC10377C0005BE0E27230010275E374D
S31A000378C3DCA11037DCD500F830B7E2275E37DCA11037DCD50040
S31A000378D83705277BFA0317A427260010B70AEC10377C0003B775
S31A000378ED02377C0006B6043735002EFA0317A427230010EC1060
S31A00037902377C0009BFC23F12350427F734103FF0276F376A00D8
S31A000379170227250004272500067A037978ED02D500F82EB7445B
S31A0003792CF1D0F809B302277527F5B04A37B5000AAA00376500D8
S31A0003794104A506FA0304F2376A0008AA0AED02D5003705277B87
S31A000379567CD0376A000E27FB371727F83717AA0CA50AA10EAA7D
S31A0003796B06A508E30D630CAA0427230002ED0216003786FFA28F
S31A0003798037650004A5063F10350427F734103FFE276F34023576
S31A0003799510CD00B00237DCFC0137DCD500F820B7F0AD001600CB
S31A000379AAB728D500F820B618150037DCFC0137DCD500F820B64A
S31A000379BF1437DCFC0137DCD500F820B7F0B00637DCFC0137DC06
S31A000379D41600B6D0340235108D00A5003F02350427F734103F31
S31A000379E9FA276F376A000037BC240CAC0437352410FA03991234
S31A000379FE27250002EC00270600003787006227260002B718378F
S31A00037A1365000227743402350837DCA10037DC27160002B60222
S31A00037A2837BC2422AC0437650004FA03991237BC2428AC0437E9
S31A00037A3D65000227743402350837DCA10037DC37550000FA0366
S31A00037A529912272300023765000227743402350837DCA1003788
S31A00037A67DC271600003786FF9AFA039BD83F06350427F7341042
S31A00037A7C3FEE276FAA0037B50002FA039CAE3735240CFA039918
S31A00037A9112ED0037550000375700022776B6043735242C7A032C
S31A00037AA67B50ED00DD00AD02ED00DD02AD0437650002A504FAC0
S31A00037ABB03788A373523A8FA039912ED003755000437570006B8
S31A00037AD02776B6043735243A7A037B50ED00DD04AD06ED00DDE4
S31A00037AE506AD0837650006A508FA03788A373523A8FA0399129B
S31A00037AFAED003755000037580004B208B62637550002375800AF
S31A00037B0F06B31CED0095029006AA0C9500D2055204AA0A3765A1
S31A00037B24000AA50CFA03788A37352442B01AED0095069002AA29
S31A00037B39109504D2015200AA0E3765000EA510FA03788A3735DE
S31A00037B4E2444FA03991237352446FA0399123F12350427F734AF
S31A00037B63103FF0276F376A0000ED00DD04AD02ED003755000296
S31A00037B78FA039912ED0037550002FA03992EAA04373523A8FA29
S31A00037B8D03991227230004A50437B8000FBFE8ED003755000017
S31A00037BA23402351037CCFCFF37CC377C0007B214340435202715
S31A00037BB7743402350837DC37B1248C37DCDD005B037BCA37351F
S31A00037BCC244AFA039912ED00950637650002FA039DEA3735244B
S31A00037BE14C7A037D1A376500027A037D1A37BC0C5CED02160014
S31A00037BF6B70037BC245C34043520FA039912ED0037550006375C
S31A00037C0B3800013787010A37352460FA039AF67A037D1EED02D5
S31A00037C20D5003705277BFA039BE87A037D1EED0237550000FA86
S31A00037C35039BE87A037D1EED02DD00AD06ED02DD02AD083765F5
S31A00037C4A0006A508FA03788A7A037D1E27250004ED00DD0CAD7F
S31A00037C5F0EEC0E27160000B740ED02D5003705AA0AA504A80ABC
S31A00037C74B71A2723000437650004277434023508340435403741
S31A00037C895C2778375C27160000B6D8376500042774ED003751D4
S31A00037C9E000C376A000CED0C27160000B60EED02D500370527EE
S31A00037CB37BFA039BE83735246AB012376500042774ED0037514C
S31A00037CC8000C376A000CED0C37550000FA039912ED003755003F
S31A00037CDD0637380001B7363735247AFA039AF6B02CED02D500EF
S31A00037CF2370534013510D5013705AA0C34043520FA0396CCEA20
S31A00037D070AB708ED0237550000FA0326E8B00437352484FA034A
S31A00037D1C9912FA039BD83F10350427F734103FEC276F376A00E2
S31A00037D3102AA04ED02DD04AD06ED02375500007CFF3738000795
S31A00037D46B21027743402350837DC37B1250037DCDD005B037D64
S31A00037D5B5C272600043787009CED0237550002FA039912373572
S31A00037D70249C7A037DFE27260004B710ED02DD06AD003765000A
S31A00037D8506A504FA03999C7A037F6AED02950637650006FA0370
S31A00037D9A9A447A037F6A27260004378701423765000437B50B9E
S31A00037DAFDAFA03994027F6B70C3765000437B50C5CFA039A1E7D
S31A00037DC427F6B604272500087A037EF23765000437B50B12FAE6
S31A00037DD903994027F6B70C3765000437B5245CFA039A1E27F6F2
S31A00037DEEB60637B50001AA087A037EF2373524BEFA0399122712
S31A00037E03F57A037F6E27260004B70837650004FA039AC67A0378
S31A00037E187EF4ED02D50B7A037EF427260004378701363765003A
S31A00037E2D04FA039AC67A037F6627260004B70C37650004FA03C3
S31A00037E42790E376A000AAA0CB008ED02DD08AD0AED02DD0AAD74
S31A00037E570CA50AED069A00A50C9A027A037F6A27260004378703
S31A00037E6C007C27250008ED02DD0CAD12EC122716000037870098
S31A00037E815A3765000827743402350834043540375C2778375C65
S31A00037E9637550000A504FA039A1E277B2776B71C27230008ED93
S31A00037EAB02DC0C376500082774340435402778376A0010ED1096
S31A00037EC027160000B6B8376500082774ED023751000C376A0096
S31A00037ED510ED1027160000B610ED023755000CFA0379E67A031F
S31A00037EEA7E02ED02DD0AAD08E509ED06DA007A037F6A27260001
S31A00037EFF04B75CED04D5003705277BD501370534013510FA0321
S31A00037F1496CCEA0EB71CED04D5003707371534013510D501374B
S31A00037F2905277B34043767FFFE3F0234023510B00837650004AC
S31A00037F3EFA03273E34013510377C0000B60C373524DAFA0399D4
S31A00037F5312FA039BD87A037E02ED069C00B004ED02950AED06CD
S31A00037F689A0037B500013F14350427F73410276F37352510FA55
S31A00037F7D039912FA03A16E37350BDA3716B70037350B12FA0351
S31A00037F92991237352516FA039912FA0302A8277B37B50005FAA3
S31A00037FA7039CAE3735251EFA039912FA03060827753716B6006E
S31A00037FBC37350001FA039BE837352526FA039912FA03058627AC
S31A00037FD17B3736000137340001FA039BE83735252EFA03991256
S31A00037FE6FA030586277B277F277F3734000137360001FA039B95
S31A00037FFBE837352534FA039912FA0305B8277BFA039D8437352D
S31A00038010253EFA03991237753500FA0305B0277B37B50003FA29
S31A00038025039CAEFA03A1663735255027F6B70037352546FA0363
S31A0003803A9912350427F73410276F373580003771357AFA000807
S31A0003804F14350427F734103FFA276F34023508AA00373580008C
S31A000380643771357A376A0002AD043765000227230002EC04C5B4
S31A0003807900370527230004FA00085027210000B6E03F063504B1
S31A0003808E27F73410276F37BD03CE17BD31AC37BD7A8017BD3173
S31A000380A3AE37BD0D0117BD31B037BD7A8017BD354837BD0D0218
S31A000380B817BD354A3775357A37342000377A357A37352CA8379A
S31A000380CDB503CEFA03CD5E3775357A37342000377A357A373535
S31A000380E2255AFA039912FA03804037752CAA37387A80B6423782
S31A000380F7752CAC37380D01B6383775357A37342000377A357A6D
S31A0003810C37352CA837B503CEFA03805437352CA837B503CEFA90
S31A0003812103CD7427F6B70437352562FA0399123775357A3734C3
S31A000381362000377A357A37352570FA039912373531AC37B503CA
S31A0003814BCEFA03805437352578FA039912373531AC37B503CEC0
S31A00038160FA03CD7427F6B70837352588FA03991227F5B008371B
S31A00038175352582FA03991237B50001350427F734103FFA276F11
S31A0003818A376A00002725000237650002277427742774376100E1
S31A0003819F02277437310CB2376A0004ED0437550002A500FA0339
S31A000381B49A1E27F6B600A504B00A27230002ED02377D0055B3C8
S31A000381C9C427F53F06350427F734103FFA276F376A000027360B
S31A000381DE21D23787006E2736338437870066EC00CC00AC04EDD7
S31A000381F30437DCFC0137DCEC008D0037F53384FCFF340835205F
S31A00038208340227793520B54037352592FA039912FA0317FCEA73
S31A0003821D023735259AFA039912E502370537B8000AB720BE08B5
S31A0003823227F6B71037B80003B70AB00C37B8000DB70C37B8002D
S31A0003824771B60027F5B006EC002705000037B500013F0635049D
S31A0003825C27F73410276F1733735E273573B6FA0386AE17317380
S31A000382715E350427F734103FF8276FAA0237B50007AA0037B5F4
S31A000382863076FA039A703801307C3735307D37B531CAFA031239
S31A0003829B3417F53083F70117FA3083F50317FA3084F5EC17FA67
S31A000382B03085F50117FA3086E50317FA308737F573B6AA043754
S31A000382C5B80050B30237B50050AA04A504AA003735736637B570
S31A000382DA3088FA039A70ED0437DCFC1237DC373530763408351F
S31A000382EF40FA0310523F08350427F734103FFA276F376A000080
S31A00038304340135081736735E37860094173631CA3787008C17D1
S31A000383193633863787008437DCA10037DCAD02EC0037CCFC12A2
S31A0003832E37CCAC046D043783006CEC00C50EF803B662C50FF849
S31A00038343ECB65C0610B6581716FFFFB6523765000437B5338682
S31A00038358FA03994027F6B6423765000037B50003FA0325F03748
S31A0003836D16B73237650004FA03992E34013508340835203761F4
S31A0003838200007C1337680002B410FA03825E376500007C07EC01
S31A0003839700C5113705FA03827637B50001B0FE27F53F0635048C
S31A000383AC27F734103FF0276F376A0000EA0227250008FA030DA1
S31A000383C1CAAA06378700D8EC0637CCFC0437CCAC04EC06CD0225
S31A000383D637DCFC0437DC3408352037610006FC15340227793518
S31A000383EB20B32CEC04C50EF803B624C50FF8ECB61EC510F80183
S31A00038400B618C511E802B6123765000427F5FA0325F03716B736
S31A000384150437350001376A00082726000837870072EC06CD02E9
S31A0003842A37DCA10637DCAD0C3765000C7CF237600004376A005C
S31A0003843F0CEC0437CCFC0737CCAC0E3765000EA500FA031116ED
S31A000384543716B6103765000EFA0312C8373525A4FA039912FA9F
S31A00038469039BD82725000A3765000A3768000CBC18ED0437DC00
S31A0003847EA10A37DCD5123705277BFA0317A42723000AEC0A6CEF
S31A000384930CBDE0FA039BD837650006FA030F46E50937053F1045
S31A000384A8350427F734103FD0276F376A0020FA03992E37B80002
S31A000384BD09B308373525A6FA0399127A03860E34103520A5208F
S31A000384D2FA03995A341035207C0C34103540FA03995A277B37F9
S31A000384E7B525C0FA03995A373530D834103540FA031234373511
S31A000384FC30DF37B531CAFA03123417F530E5F70117FA30E5F5F5
S31A000385110317FA30E6F5EC17FA30E7173530E8373525C4FA0363
S31A000385269086AA22378700DEEC220600378700D637650022FA59
S31A0003853B03992E37B8000FBED8373530EAA522FA03995AAA24B9
S31A0003855027230024373525D0FA039912341035207C0CFA0390E8
S31A0003856586AA22378700A0EC220600B7E637650022FA03992E15
S31A0003857A277B7C0137B5313AA02434013508340227793520BF4D
S31A0003858F02373525F0B0BE37650024A522FA03995AAA2627234C
S31A000385A40026173330E937BC0003AC28341035207C1C37B50B3E
S31A000385B9B8FA030234373530D8A52637B030D8FA03105217F520
S31A000385CE30E9370534103520FA0383AE37163786FF7AFA03975C
S31A000385E38A27F63786FF70A51CAA2AEC1EAC2C3765002AA52C99
S31A000385F8FA030274EA2EB7C827210028B6A63735260A7A0385F1
S31A0003860D583F30350427F73410276F3402350834083540F874C7
S31A00038622B60237B50002B026F864B60237B50008B01CF86BB6D1
S31A000386370237B50004B012F876B60237B50001B008F873B70084
S31A0003864C27F5B00037B50010350427F734103FFC276F376A003B
S31A0003866100FA039D84373523A8FA03991227250002B002A50257
S31A00038676FC02AA02ED003755000037DCFC0237DCAD002776B79E
S31A0003868BE437650000FA039D84373523A8FA03991237650002B6
S31A000386A0FA039BE8FA039BD83F04350427F734103FC8276F371A
S31A000386B56A000227250004341035207C02FA03798CAA06376586
S31A000386CA000637B52618FA039A1E27F6B6022775FA0301CE3739
S31A000386DF65000637B52620FA039A1E27F6B6083735318C37B53B
S31A000386F40001FA0304A23765000637B52628FA039A1E27F6B75F
S31A000387092E3765000637B5262CFA039A1E27F6B608373509D06F
S31A0003871EFA0399127A038B863765000637B52634FA039A1E2743
S31A00038733F6B60A2775FA03425A37B500017A038F48376500065A
S31A0003874837B5263EFA03994027F6B612341035207C02FA03797B
S31A0003875D8C277BFA039AC637FA35BCB0CE3765000637B52644DB
S31A00038772FA039A1E27F6B60E37753500FA0305B0277BFA039B86
S31A00038787E87A038B863765000637B5264AFA03994027F63786B0
S31A0003879C009434103540FC02AA0E3765000EFA03798CAA0C3723
S31A000387B165000EFA03798C277BFA039AC6AA10ED0C1600B710A6
S31A000387C63765000CFA03992E3765000CFA039EC637FA313A275D
S31A000387DB260010B60237B50001AA10341035207C04FA0381D282
S31A000387F037163787FF4437350BDAFA0399123775313AFA039D73
S31A00038805843735240CFA0399123775313AFA030570277BFA0365
S31A0003881A9D84FA039BD83775313A7C02377A313A27210010B6F0
S31A0003882FB27A03873C3765000637B52650FA03994027F6378685
S31A00038844009434103540FC02AA1437650014FA03798CAA123768
S31A00038859650014FA03798C277BFA039AC6AA16ED121600B710EB
S31A0003886E37650012FA03992E37650012FA039EC637FA313C27A6
S31A00038883260016B60237B50001AA16341035207C04FA0381D2CD
S31A0003889837163787FE9C37350B10FA0399123775313CFA039D3B
S31A000388AD843735240CFA0399123775313CFA030578277BFA03B3
S31A000388C29D84FA039BD83775313C7C02377A313C27210016B63E
S31A000388D7B27A03873C3765000637B52658FA03994027F63786D5
S31A000388EC009434103540FC02AA1A3765001AFA03798CAA1837AE
S31A0003890165001AFA03798C277BFA039AC6AA1CED181600B71030
S31A0003891637650018FA03992E37650018FA039EC637FA313E27EF
S31A0003892B26001CB60237B50001AA1C341035207C04FA0381D218
S31A0003894037163787FDF437352662FA0399123775313EFA039DCC
S31A00038955843735240CFA0399123775313EFA030580277BFA0300
S31A0003896A9D84FA039BD83775313E7C02377A313E2721001CB68B
S31A0003897FB27A03873C3765000637B52664FA03994027F6B6081F
S31A000389943735A7F4FA0386587A03873C3765000637B5266CFA89
S31A000389A903994027F6B60837350882FA033C147A038B8637658C
S31A000389BE000637B52676FA039A1E27F63786009CED021600B726
S31A000389D348341035207C02FA03798C277BFA039AC6AA0837B885
S31A000389E80003B3043735267E7A038F1437650008277A370737CD
S31A000389FD1527F427F427F427F427F4277A377A357A373531AC76
S31A00038A1237B503CEFA03CD5EFA038F4EB01037F5357A37173767
S31A00038A270527FF27FF27FF27FF27FFAA0837650008FA039BE898
S31A00038A3C1736344AB71237352698FA0399123735344AFA039936
S31A00038A51123735244AB0003735269CFA039912373526ACFA035A
S31A00038A6699127A038B863765000637B526C0FA039A1E27F6B6BD
S31A00038A7B04FA0380907A03873C3765000637B526C6FA039A1E5D
S31A00038A9027F637860074F5FFEA1EED021600B71C251EED02D59F
S31A00038AA5003705277BFA038614E71EEA1EED0237DCFC0137DC1F
S31A00038ABAAD021600B6DE27250008376500082774277427743745
S31A00038ACF610008277437310CB2376A0020E51EED20D610B714DD
S31A00038AE4341035207C04FA0381D237163787FC4637650020FA08
S31A00038AF9037B6227230008A50837B80055B3B87A03873C3765F5
S31A00038B0E000637B526CCFA039A1E27F6B62E27250008376500BF
S31A00038B230827742774277437610008277437310CB227F5FA03E1
S31A00038B387D2827230008ED08377D0055B3D6373526DC7A038F27
S31A00038B4D143765000637B52700FA039A1E27F6B62C37352706F4
S31A00038B62FA039912FA037F74373523A8FA0399123735014DFACA
S31A00038B77030294FA03181A3716B7D8FA0317FCFA039BD87A033F
S31A00038B8C873C3765000637B52708FA039A1E27F63786012AEDA4
S31A00038BA1021600378600722725002227250008A50827F427F4CA
S31A00038BB627F427F4AA24ED2437DC37B131AC37DC375500463798
S31A00038BCB5700482776B71C341035207C04FA0381D23716B71AF6
S31A00038BE0A52437B131F237650008FA037A7A2723002227230058
S31A00038BF508ED08377D0018B3AEA50837B800193786FB3227264C
S31A00038C0A00223786FB2A37352710FA0399127A03873C34103544
S31A00038C1F207C02FA03798C277BFA039AC6AA0837B80018B30428
S31A00038C343735272A7A038F14ED021600B616376500082774270E
S31A00038C49742774277427FB37B131F2376500087A038CC4341081
S31A00038C5E3540FC02AA2637650026FA03798C277BFA03790E3794
S31A00038C736A0028AA2AA50827F427F427F427F4AA2C37B131ACC9
S31A00038C88AA2EA528ED2E9A46A52A9A4837650026FA03798C2792
S31A00038C9D7BFA03790E376A0030AA32A530ED2E9A4AA5329A4C7C
S31A00038CB2EC2C37CC37B131F237CC3765000834043540FA037AB3
S31A00038CC77A7A03873C3765000637B52742FA039A1E27F6B61640
S31A00038CDCED021600B6043735274A7A038F1437650002FA03849F
S31A00038CF1AC7A03873C3765000637B52770FA039A1E27F6B6309C
S31A00038D06ED021600B722FA0302C8EC0237BD0050AD00373573EC
S31A00038D1B0A34043540FA03999CF50117FA7308FA0302D67A037D
S31A00038D30873C173573087A03873C3765000637B5277AFA039A95
S31A00038D451E27F6B606F50117FA72B57A03873C3765000637B51D
S31A00038D5A2782FA039A1E27F63786012E3765000237B52788FA61
S31A00038D6F039A1E27F6B604FA03268A7A03873CEC0206003787B5
S31A00038D8400A234043520FA038184AA0A378700783765000AFA16
S31A00038D99037B62ED0A375500007CFF37380005B24A277434029D
S31A00038DAE350837DC37B1281437DCDD005B038DBEED0A37550017
S31A00038DC30CFA0379E6B02A373524BEB02037352790B01A3735D9
S31A00038DD827A4B014373527BAFA039912ED0A375500067CFFFAFB
S31A00038DED039BE8373527C0FA039912ED0A2716000E3787F938B6
S31A00038E023755000EFA0399127A038B86373527CEFA0399123742
S31A00038E17650002FA039912373527DCFA0399127A03873C27258B
S31A00038E2C00342725000837650008FA03967EEA363787F8FA27F4
S31A00038E41260034B60C341035207C04FA0381D237163787F8E4A7
S31A00038E56E536F80AB606FA039BD827250034B026E536F809B68D
S31A00038E6B1237350020FA0317A427230034ED34377D0011BFE888
S31A00038E80B00AE5363705277BFA0317A42723003427230008B0E9
S31A00038E95983765000637B527E8FA03994027F6B602373527F05C
S31A00038EAAB0643765000637B527FCFA039A1E27F6B65C34103588
S31A00038EBF207C02FA03798CAA0637650006FA038184AA0AB7280E
S31A00038ED43765000237BC0000340235081600B7003402351037FD
S31A00038EE965000A34043540FA037D283765000AFA037B627A03B0
S31A00038EFE873C37352800FA03991237650006FA0399123735277A
S31A00038F13DCFA0399127A03873C37650006FA038184AA0AB71A53
S31A00038F28EC020600B7083765000A34043540FA037D28376500E7
S31A00038F3D0AFA037B627A03873C27F53F38350427F734103FFC89
S31A00038F52276F377531AE37387A80B616377531B037380D01B6EB
S31A00038F670C377531AC373800FFB30237382000B300273531ACB9
S31A00038F7C373531AC377131AC376A00003735357A37680000B3FB
S31A00038F911037600000340235083765000034083540FA039A4480
S31A00038FA627250002376500022774277427743761000227743487
S31A00038FBB02350837DC37B10CB237DC3755000437680000B506A3
S31A00038FD03408352027F5FA037D2827230002EC02377C0055B33F
S31A00038FE5C03F04350427F734103FF8276F3410352037F52828EE
S31A00038FFAFA030234FA0397A837B8FFFF3786006AEC00AC04EC4E
S31A0003900F02AC0637650004A506FA0302743716B7DA37752828F7
S31A0003902437380064B31227FB27FF27FF27FF27FF27FF277934E2
S31A0003903902350817BD28283410352037F52828FA0302343775C2
S31A0003904E314027FB37B6000327F43401350837DC37B12820377A
S31A00039063DC7C01377A314037550000FA0306F27A038FFE37BCF6
S31A0003907807D017BC282837053F08350427F734103FFA276F37BC
S31A0003908D6A000027260000B70437650000FA03991227250004BF
S31A000390A2FA038FECEA023705277B3738000A37870072BE1C37B4
S31A000390B7380003B74EBE042776B7547A03916437380004B74A0B
S31A000390CC37380008B76A7A03916437380024B718BE06373800E7
S31A000390E10DB7407A0391643738007FB74E373800C0B70A7A039B
S31A000390F6916427260004B662F501B0FEF50217FA31C727F57AC4
S31A0003910B0391A23735282AFA0399127A03909037352830FA034C
S31A00039120991227F57A0391A2FA039BD8ED0437DC37B1314237B4
S31A00039135DC150037B531427A0391A227260004378FFF58272166
S31A0003914A0004ED0437DC37B1314237DC150037352836FA03991C
S31A0003915F127A0390A2E502F1E0F85E3782FF32A50437B800445D
S31A000391743782FF28ED0437DC37B1314237DCE502DA0027230080
S31A0003918904ED0437DC37B1314237DC15003705277BFA0317A4A7
S31A0003919E7A0390A23F06350427F734103FFE276FFA039BD837AA
S31A000391B37531AC373803CEB610377531AE37387A80B6063775EA
S31A000391C831B037380D01B7043735283AFA03991237352890FADC
S31A000391DD039086AA00B724ED001600B7EA37650000FA0386AE65
S31A000391F23716B6DE3735244AFA03991237650000FA0399123781
S31A0003920735289AB0C43F02350427F734103FFE276F173634208E
S31A0003921CB76C1736342BB76637353420FA03992E277B340235B7
S31A000392310837DC37B131AB37DC17D502743705277B376A00004C
S31A00039246373572D237B53420FA031D403735342BFA03992E270A
S31A0003925B7B3402350837DC37B131AB37DC17D5027F3705277BD2
S31A00039270376A0000373572D637B5342BFA031D4037B5000237C1
S31A00039285FA72D0F50117FA72B43F02350427F734103FFC276FB5
S31A0003929A376A0000272500023765000227742774277427742796
S31A000392AFFB37B1357C37650000FA039A1E27F6B65AA5023707AA
S31A000392C4371527F427F427F427F427F43775357A340227793553
S31A000392D920B738173635BEB6F637650002277A3707371527F498
S31A000392EE27F427F427F427F4277A377A357A373531AC37B503BD
S31A00039303CEFA03CD5EFA038F4E3735318C37B50003FA0304A2C1
S31A0003931837B50001B00C27230002A50237B800033783FF742755
S31A0003932DF53F04350427F734103FFC276F37B50003AA02376547
S31A000393420002277A3707371527F427F427F427F427F4277A3781
S31A000393577A357A373531AC37B503CEFA03CD5EFA038F4E37652B
S31A0003936C000227742774277427743731357C37B50010AA00377F
S31A00039381B5344AFA03999C27210002BCAE3F04350427F73410D7
S31A000393963FFE276F27FBEA00F82AB60417F53550F801B72A375C
S31A000393AB7531943738000FB2123402350837DC37B1319837DCDE
S31A000393C0E500DA007C01377A31943775319437380010B6002710
S31A000393D53531943F02350427F734103FFA276F376A0004FA0333
S31A000393EA9798ED04377D0001B20637650004FA039776B0442713
S31A000393FF2500043765000437360001FA039776FA0397A837B8E4
S31A00039414FFFFB6F234103520FA03021034103520FA03025637C7
S31A00039429B803E7B208FA0397A837B8FFFFB60AB0E22723000400
S31A0003943EED04377D001DB3B83F06350427F734103FFA276FFA3A
S31A0003945303005E37350001FA0306F2FA03CD0AFA030E2EFA032E
S31A000394683BDA37354B0027F5FA0397F2FA0301DE37350003FA33
S31A0003947D03A17437350061FA03A136FA0303EE373AFF1F37352F
S31A000394920002FA0306F2FA039334373B00E017F5357337052798
S31A000394A77B37380001B70437380002B704B006FA030430B0003E
S31A000394BCFA03CCD8373AFF1F17F533F63705277B17F533F737E2
S31A000394D10534013508FA0396CCEA04B60437B52F3E37FA33F64C
S31A000394E637350004FA0306F237F531B2AA0037F531B4AA023756
S31A000394FB650000A502FA03157C3735318CFA03048C3735000592
S31A00039510FA0306F2FA03C200FA031610FA0318B837350006FA2D
S31A000395250306F2273631D8B706377531D827F5FA0397F2277517
S31A0003953AFA0306342775FA03061A2775FA03068237350001FA9B
S31A0003954F03066837350001FA03064EFA0397A837B8FFFFB6F2FE
S31A0003956437350007FA0306F21736354FB71A17F5354F370527EC
S31A000395797B27743402350837DC37B10AB237DC37550000FA03F8
S31A0003958ECB6EFA0305F63716B60837B5000137FA21D2FA0391E4
S31A000395A3A8377531AE37387A80B6E6377531B037380D01B6DCD6
S31A000395B8273521D2FA031610FA03921237350001FA03069CFA7C
S31A000395CD0302B63735FFFFFA0306F217F5341B3705277BFA0330
S31A000395E293DE2775FA0306F217F531C73705277B37380004B262
S31A000395F79C27743402350837DC37B128A037DCDD005B03960CF9
S31A0003960CFA036C6AB01EFA031B42B018FA0373B0B0122775FA05
S31A0003962103069CFA03723C2775FA03069CFA0374F6B0E63F065E
S30900039636350427F7D0
S31A0003963A342037B50003379C37BCCE7C3C0237480000B2F43725
S31A0003964FCC37B0CE7E27FF350227F737B59F12372527FC3733FD
S31A000396640000277FB0CC7C01B0C8342037B50003379C27C53798
S31A0003967905350227F737BCCFEBB0E637BCCF36B0E0342037DC47
S31A0003968E37B50003379C37BCD248374D27F5377CD464B422F599
S31A000396A32F377CD3E7B5FEF55CDA003D01277527C527DA7C01EB
S31A000396B827C527DAB6F47C01374D37CC37B0D248350227F7277C
S31A000396CD7AF82FB730F85CB72CF830B524F839B330F841B51CA1
S31A000396E2F85AB328B016277AF82FB714F85CB710F841B508F8DB
S31A000396F75AB314F861B500F86AB30C27F527F7277AF821B5F26A
S31A0003970CF87EB2EE27F7277A37BC28AAC800B7F03C01377C281E
S31A00039721BAB6F0B0D83420374C3745000085022776BA00277575
S31A0003973627F5B702277537B5FFFF277BB72A37BDD46437B5001F
S31A0003974B03379D3D0437580000B2F43750FFFC950037D0FFFC9A
S31A0003976037CC950237D0FFFE3725372837CC37D1FFFE3502272C
S30600039775F7F3
S31A0003977637BC00002776B6020801F90727F70901F90727F73707
S31A0003978BBC830A37C5100237C0100027F737BC931037C51002A0
S31A000397A037C01000B6F227F737B5FFFF37BC830A3745100237AF
S31A000397B5481000B70C27857C0237360FFF374A100237C6100432
S31A000397CA27F727FB37BC93103745100027CA27F57C0137360F19
S31A000397DFFF37481002B706374A100037CC0980FC0B27F7344069
S31A000397F437380096B40037354B0037BC00FF37BD002CF800B726
S31A000398091437BD0E2CF801B70C37BD062CF802B70437BC01FF75
S31A0003981E37BD022C17BC930E374C3735000837B500003728371D
S31A000398334C3733000037B506DC37BC0000373B00E08AA0374AA3
S30F00039848FC08178DFC0A350127F70B
S31A000398523410276F374CC4003C0127FFB4FEA40627FFB4FEA49C
S31A000398670627FFB4FEA40627FFB4FEA40627FFB4FEA40627FF31
S31A0003987CB4FEA40627FFB4FEA40627FFB4FEA40627210008B668
S30A00039891C2350427F7B0
S31A000398962776B720277A2776B71A37CC27FB3725340337CC274F
S31A000398AB7B3725274F8102374300003F04B40237B5FFFF27F754
S31A000398C034033FFA274F37B500108A0227050004270500002799
S31A000398D5040008270C0006270C000427040008270C0006270C5A
S31A000398EA000427040000850027F4FC01374500042779B5043784
S318000398FF4A00042703000027010002B6C435403F0827F757
S31A000399123412276FB0083C01AC023705277BFA0317A4EC02C56F
S31A0003992700B6EA352427F7374C277527C5B7027C0127C5B6F632
S31A0003993C27FB27F7374C37DC2775274527D5370AB6027C013786
S31A0003995116B6EE371727F827F7374C37DC2775B0FE7C0127D55A
S31A0003996627CAB6F437CC277827FB27F73410276F374C37DCA551
S31A0003997B06B7162775274527D5370AB6083716B7087C013768D0
S31A000399900006B6E8371727F8350427F7274FCC04374C37DC373E
S31A000399A5300001B510B70CD500B7FE3D01CA003C0137300001B4
S31A000399BAB6EC050037CC27F727FBF830B506F83AB40237B500EE
S31A000399CF0127F727F527F727FB3705F861B502F87BB4FEF4207A
S31A000399E427F727FB3705F841B502F85BB4FEF42027F7374C2718
S31A000399F975B00427F9FFD827CA7C0127C5B6F027F7374C2775F3
S31A00039A0EB00427F9FFD427CA7C0127C5B6F027F7374C37DC27B8
S31A00039A237527C527F9FFAE370727D527F9FFA6370AB6047C0180
S31A00039A383716B6E427F7371727F827F7374C277B3715B0FE273A
S31A00039A4DCA37300001B4F427F7274FCC04374C37DC27F5B00259
S31A00039A6227C527D0B60237300001B4F027F73410276FEC06B79E
S31A00039A7724340227793520374C37DCB50C277527C527DA7C0125
S31A00039A8C37680006B6F0B0083730000127C527DA2776B6F035EC
S30800039AA10427F797
S31A00039AA427FBBAFE27F227F72776BBFE27F727F02770FC01373D
S31A00039AB933000027F73C01C800B7F627F7374C2775F52036EE16
S31A00039ACEF53036EA3705C500F030B514F80AB41037DC27FB2729
S31800039AE37427742778277437DC27783C01B0DE277A27F7E2
S31A00039AF634103FFE276F376A00003735FFFFFA0306F2373528A7
S31A00039B0BE2FA03991237650000FA039912FA03979837350001D5
S31A00039B20FA0301CE3F02350427F734103FFA276F27FBEA00277D
S31A00039B35250002F1BFF819B312E500F19FF819B30AE500370501
S31A00039B4A277BFA0399C23716B70237B50001AA02A5023F063543
S31A00039B5F0427F734103FFC276F376A0000AA02FA03992E376504
S31A00039B7400002778A502FA03995A3F04350427F734103FFC275D
S31A00039B896F27FBEA01371F371F371F371FEA023705277B3402EA
S31A00039B9E350837DC37B128EA37DCD5003705277BFA0317A427BA
S31A00039BB37AE501277A3736000F3402350837DC37B128EA37DC84
S31A00039BC8D5003705277BFA0317A43F04350427F73410276F3769
S31A00039BDD3528FCFA039912350427F734103FFE276F376A00005A
S31A00039BF237380009B30C37BC000AA500372A34043520FA039BF6
S31A00039C07E83735000AA50034023510372A277B37370030FA0323
S31A00039C1C17A43F02350427F734103FF8276F376A000037B50039
S31A00039C310AAA02EC02A500372AAC06E507F130EA043705277BE0
S31A00039C46FA0317A4A500EC02372A277B37370030FA0317A43F1D
S31A00039C5B08350427F734103FFE276F376A0000BF0E3735002B70
S31A00039C70FA0317A437650000FA039BE8B02627260000BC1037DC
S31A00039C8535002DFA0317A4376500002772FA039BE8B00C3735CA
S31A00039C9A0020FA0317A437350030FA0317A43F02350427F734B4
S31A00039CAF103FFE276F376A0000277B37380001BF1A37BC000A2B
S31A00039CC4A500372A3402350837DCFCFF37DC34043520340835EA
S31A00039CD940FA039CAE3735000AA50034023510372A277B3737DF
S31A00039CEE0030FA0317A43F02350427F734103FE4276F376A003A
S31A00039D0310EC1027060000BC323735002DFA0317A4EC10CC0002
S31A00039D18AC14EC10CC02AC1637650014A516FA039AB2376A008C
S31A00039D2D0C275E37DCFC0C37DC9A023410352034083540B002C1
S31A00039D4234103520A510FA030982AE12E500F830B620EC120686
S31A00039D5701B71A27230012EC12C500F830B7EAB00CEC12C500B5
S31A00039D6C370527230012277BFA0317A4EC120600B6E63F1C35B7
S31A00039D810427F734103FFE276F376A0000277A37173705277A1E
S31A00039D96FA039B84E5013705277BFA039B843F02350427F734E7
S31A00039DAB103FFE276F376A0000ED00D5003705277BFA039B845A
S31A00039DC0ED00D5013705277BFA039B84ED00D5023705277BFA2C
S31A00039DD5039B84ED00D5033705277BFA039B843F02350427F7F7
S31A00039DEA34103FFC276F376A0000AA02B00CED00D50037052718
S31A00039DFF230000277BFA039B8427210002ED02377DFFFFB6E0E4
S31A00039E143F04350427F734103FFC276F376A0000AA02B032ED65
S31A00039E2900D500F1DFF85DB202D500F85CB61237352900FA03EA
S31A00039E3E9912ED00D5003705277BFA039B84B008ED00D50037EE
S31A00039E5305277BFA0317A42723000027210002ED02377DFFFF5D
S31A00039E68B6BA3F04350427F734103FFA276F376A0000AA043739
S31A00039E7DBD0000EC00C50027230000F1D0EA02F809B22834084B
S31A00039E92352027742774340835402778277434023508E50237AB
S31A00039EA705277B375C2778375C27210004B6C634083540B00008
S31A00039EBC37B5FFFF3F06350427F734103FFC276F34023510343E
S31A00039ED10135082775C500EA0037CCFC0137CCF1D0EA02F80939
S31A00039EE6B31CE500F1BFF805B202E500F1C9B00EE500F19FF87F
S31A00039EFB05B30237B5FFFFB022E500F1A9EA0027742774277499
S31A00039F102774E500370534013767FFFE3F0237DCFCFF37DC370E
S31A00039F2586FFAC27FB3F04350427F734103FFC276F376A00007B
S31A00039F3AAA027A039F9CED00D500F82AB62E27230000ED00D5D1
S31A00039F4F00F82AB7F0ED0016003787004EB00EA502272300026B
S31A00039F6437650000FA039F303716B638ED021600B6E427F5B0D1
S31A00039F7932ED00D500F83FB604ED021600B608B0E8ED02D500C6
S31A00039F8EED00D800B6DE2723000227230000ED0016003786FF07
S31A00039FA39A27F5ED021600B60037B500013F04350427F7341064
S31A00039FB83FE8276F376A0004AA0627260004BC3C37650004A5EB
S31A00039FCD06FA039AB2376A000CAA0EED1EAD00ED20AD023765B2
S31A00039FE2000CA50EFA0304D2376A0010AA1237650010A512FA05
S31A00039FF7039AB2376A0008AA0A37650008A50AB01AED1EAD00CB
S31A0003A00CED20AD0237650004A506FA0304D2376A0014AA1637B0
S31A0003A021650014A5163F18350427F734103FE6276F34023508CD
S31A0003A036AA0427160000BC3EDC00AC06DD02AD0837650006A5BE
S31A0003A04B08FA039AB2376A0000275E9A0234083520A504FA03AD
S31A0003A060078E376A0012AA1437650012A514FA039AB2376A008B
S31A0003A0750EAA103765000EA510B01234083520A504FA03078E18
S3170003A08A376A0016AA1837650016A5183F1A350427F723
S31A0003A09C341C351C27F7B5023808FA19B0003908FA1936E83982
S31A0003A0B104FA1936E23804FA1927F736DA3910FA1936D4381037
S31A0003A0C6FA1927F736CC3902FA1936C63802FA1927F73420F54B
S31A0003A0DBFF27FA27F9FFC0277C277CF50E277C27F9FFB2371163
S31A0003A0F0B6F227F9FFB227F9FFC0350227F7277A371E277E37D3
S31A0003A1050E3420F5FF27FAF50B3704277C27F9FF8A3711B6F050
S31A0003A11A27F9FF84F506277C27F9FF7A3711B6F227F9FF7427A3
S31A0003A12FF9FF88350227F73420F5FF27FA27FB7508371C27F9C2
S31A0003A144FF5A3701B6F227F9FF7A3920FA19350227F73420F521
S31A0003A159FF27FA17F5F7073705350227F736EA3710F62027F792
S31A0003A16E36E2F60827F73420F5FF27FA39C0FA1937380003B404
S31A0003A1830C277FB5003840FA19277FB5003880FA19350227F751
S31A0003A1983410276F27FB3771A466377AA466277BFA0397CC3509
S31A0003A1AD0427F734103FFE276F376A0000ED00D5003705277B1A
S31A0003A1C2FA03A19827230000ED001600B6E63F02350427F73494
S31A0003A1D7103FFE276F376A0000E5003705277BFA03A198275E68
S31A0003A1ECD5013705277BFA03A1983F02350427F734103FFC272D
S31A0003A2016F27250000277537B59600FA0397F23735A0A2FA0335
S31A0003A216A1D637350018FA03A1D62735A46627250002ED0237E1
S31A0003A22BDC37B1290437DCD5003705277BFA03A19827230002DC
S31A0003A240EC02377C0017B3DC3775A46637367FFFFA03A1D6376D
S31A0003A25535B0B3FA03A1D6FA039798373512C027F5FA0397F2D3
S31A0003A26A3F04350427F734103FF0276FAA04FA030780376A0060
S31A0003A27F00AE0EED0E9A023765000E37B5291CFA03A02C376A29
S31A0003A294000AAA0CED0AEC048D00ED0C8D023F10350427F73416
S31A0003A2A9103FE4276F3735A470FA030778277B3736001C3786EA
S31A0003A2BE00B43735A486FA03077837BD0064274D372AEA02376C
S31A0003A2D335A484FA030778EA033735A482FA030778EA0437353F
S31A0003A2E8A488FA030778EA053735A48AFA030778EA063735A4AB
S31A0003A2FD8CFA030778EA07341035207C08376A00143735A492D6
S31A0003A312A514FA03A27034103540FC0C3735A496FA03A27037B8
S31A0003A32735A4A0FA030780376A0016AA1837BC01CFAC00376597
S31A0003A33C001837B50009FA03050AAA123735A4A4FA030778AA54
S31A0003A3511A37352C85376A00003765001A37B5028DFA03050AD9
S31A0003A366AA103765001434103540FC02FA031F2C3F1C350427B5
S31A0003A37BF734103FFA276FAA00376A000227250004A5023765DA
S31A0003A39000027C02376A0002277BFA030778A104AA04272100D3
S31A0003A3A500B6E027F527260004B60037B500013F06350427F758
S31A0003A3BA34103FFE276F27FB17FDA314377D0009378200823752
S31A0003A3CFDC37B1A31A37DCDA003775A3147C01377AA31437384B
S31A0003A3E4000A378600CA3735A31AFA03077837B881FFB63A378F
S31A0003A3F935A31A37B50005FA03A37C3716B72A3735A31CFA03F1
S31A0003A40E077837FAA3163735A31EFA03077827F6B70A277B7C22
S31A0003A423012774377AA3187A03A4B62735A3147A03A4B63775A6
S31A0003A438A3147CFF377AA314376A00003735A31B37B5A31AFAFE
S31A0003A44D039A70B0603775A316373803E8B61017FDA314377DD0
S31A0003A462006DB20637DC37B1A45E37DCDA0017FDA31437DCFCF3
S31A0003A4770137DC17BDA31437F5A318FC0A3408352034022779D4
S31A0003A48C3520B5222735A3143775A316373803E8B6143735A4DA
S31A0003A4A16837B50032FA03A37C3716B704FA031F1EFA03A2A872
S31A0003A4B63F02350427F734103FFE276F37BD00F9AD0037B50053
S31A0003A4CB79FA03050A3F02350427F734103FFE276F37BD0080CB
S31A0003A4E0AD0037B5002DFA03050A3F02350427F734103FFA2750
S31A0003A4F56FAA0037B52920FA03A02C376A0002AA04EC02ED0006
S31A0003A50A9C00EC049C023F06350427F734103FEC276F277A17B0
S31A0003A51FF5A4CE277A3736000F37380004378E007C3738000374
S31A0003A534378D007437BD0006AD003735A4E434103540FC02FA85
S31A0003A549039A70341035207C0237B50006FA03075234103540CF
S31A0003A55EFC083735A4CFFA03A4F034103540FC0C3735A4D3FACD
S31A0003A57303A4F017FDA4DEAD123775A4DE3738014CB204FA0341
S31A0003A588A4BCAA12B00237BD00A2AD123775A4DBFA03A4D6AA46
S31A0003A59D10341035207C0834103540FC02FA031F2C3F143504E8
S31A0003A5B227F734103FFC276F17F5A32537053401350837DC378C
S31A0003A5C7B1A32637DC17F5A324D00017FAA32427FBEA02DA0086
S31A0003A5DCE50217F1A32417FAA3241733A32517F5A325F82CB613
S31A0003A5F1001735A32527FBF80D3786008A17F5A324F80D378635
S31A0003A606008017F5A3253705277B3402350837DC37B1A3263796
S31A0003A61BDCD500F8CAB66417F5A325F82AB2007C01B0FE277525
S31A0003A6303402350837DC37B1A32637DCD500F8CAB64417F5A382
S31A0003A645253705277B3731A32637BD002C375C2779375CAD0030
S31A0003A65A37B5A4CCFA039A7017F5A32537053401350837DC37B3
S31A0003A66FB1A4CC37DCAA003735A32634083540FA039A70FA0305
S31A0003A6841F1EFA03A5163F04350427F734103FE8276F376A0087
S31A0003A69900AA02ED00D50137053735EA60FA0304CE376A0004CE
S31A0003A6AEAA06EC00CC02AC0A27250008A506A10AAA0EA504E380
S31A0003A6C3096308AA0CEC0CED029C00EC0E9C02ED001600B7205A
S31A0003A6D8EC02CC00AC10ED0EAD1237650010A50EFA039AB23755
S31A0003A6ED6A0014AA16ED14EC028D00ED168D023F18350427F755
S31A0003A70234103FF4276F3735A4F834103540FA03A690341035BF
S31A0003A71740FC043735A4FCFA03A69017FDA500AD0817FDA5027C
S31A0003A72CAD0A3410352037B5A504FA031F2C3F0C350427F7340C
S31A0003A741103FFE276F3402351034013508373600303402351012
S31A0003A7563404354027FF27FF27FF3735002D3726340135103422
S31A0003A76B08354037B6003F27F4AA0037CCA10037CC340435400E
S31A0003A7803F02350427F734103FFC276F376A0000273635BCB768
S31A0003A79518EC00277AC501277A3736000F27FBFC033765000061
S31A0003A7AAFA039DEAFA039BD8EC00C5003705277B373800533715
S31A0003A7BF870156BE12373800513787008C378E012E3738005011
S31A0003A7D4B72A7A03A994373800563787018EBE083738005437FA
S31A0003A7E987014A7A03A99437380058378700BC373800A53787B3
S31A0003A7FE018E7A03A994376500007C03FA03077834013508ECFF
S31A0003A81300C50217FAA4F93408354037B67FFFAA02376500024C
S31A0003A82827742774376100022774377AA4FA34083520277A37EF
S31A0003A83D17370527FF27FF27FF27FF27FF27FF27FF277A27FBDD
S31A0003A85217FAA4F87A03A994376500007C03FA03077834013580
S31A0003A86708EC00C50217FAA4FD3408352037367FFF27FB27F4AD
S31A0003A87C27F4AA0237610002376A0002A50227F437FAA4FE34F1
S31A0003A891083520277A3717370527FF27FF27FF27FF27FF27FF3D
S31A0003A8A627FF277A27FBF40117FAA4FC7A03A994EC00C5021781
S31A0003A8BBFAA4F9376500007C03FA030778277B377AA4FAEC0074
S31A0003A8D0C501F60117FAA4F8C50517FAA4FD376500007C06FA6C
S31A0003A8E5030778277B377AA4FEEC00C501371FF401F60117FAD9
S31A0003A8FAA4FC7A03A994376500007C02FA030778277B37BC00BB
S31A0003A90F0A372A17BCA5027A03A994EC00C5013705277BC50234
S31A0003A924370534013508FA03A740277B377AA5007A03A994379A
S31A0003A9396500007C01FA030778277B277F277F277F277F340232
S31A0003A94E3508EC00C50317FAA507C502371F371F17FAA50834D8
S31A0003A963083540F63F17FAA509FA03A702B01EEC00C50317FA2C
S31A0003A978A504C501371F371F371F371F17FAA505C50217FAA5C2
S31A0003A98D06B000FA031F1E3F04350427F73410276F27FB37B837
S31A0003A9A200FFB300273529243775292437380011B23234023574
S31A0003A9B70837DC37B1A35237DCDA007C01377A292437380002B1
S31A0003A9CCB318277A17F5A353277A3736000F7C0337782924B6B1
S31A0003A9E1043735A352FA03A786350427F734103FF0276F376AC8
S31A0003A9F6000EAA04ED0EDD00AD06EC0ECC02AC0837BD003CADA3
S31A0003AA0B002725000237650006A508FA039FB6376A000AAA0CDD
S31A0003AA20ED0AEC048D00ED0C8D023F10350427F734103FE427E8
S31A0003AA356F376A0014AA16EC14CD043735006434083540340297
S31A0003AA4A3510372AAA1AE51BEA02EC14C502EA03C503EA04C569
S31A0003AA5F06EA05C507EA06C508EA07376500147C0D3410354078
S31A0003AA74FC08AA18FA03A9EE376500147C11275E37DCFC0C3756
S31A0003AA89DC34083540FA03A9EEEC163745000037B501CFAA00AA
S31A0003AA9E37B50009FA03050A277B376A0012EC1637450002378D
S31A0003AAB3BD000A274D27FB372A34043520376A001037650018D5
S31A0003AAC834103540FC02FA031F2C3F1C350427F734103FFE2717
S31A0003AADD6F34023508274D37CCFC1D37CC375500003738456145
S31A0003AAF2B718B20437384261B70CB05837384861B72637384838
S31A0003AB0762B70CB04AD53EB0FED546F6B0EA00B73AB02A274D66
S31A0003AB1C37CCFC1F37CC2500D527F6E0F89FB314B016274D3734
S31A0003AB31CCFC2F37CC2500D57FF6E0F89FB300F501EA0026006D
S31A0003AB46B70A3408352034043540FA03AA30B000FA031F1E3FF2
S31A0003AB5B02350427F734103FFC276F27FB17F4A36417FAA36422
S31A0003AB7017F5A36537053401350837DC37B1A36637DC27FBDAF2
S31A0003AB85001733A36517F5A365EA02F80337830080F804B64A2F
S31A0003AB9A3775A36637384040B61817F5A368EA02F840B30EF837
S31A0003ABAF5AB20A17F5A369EA02F860B300F87AB316F50317FA1F
S31A0003ABC4A36537B50003AA003735A36737B5A366FA039A70B0B0
S31A0003ABD93A17F5A36817F4A36917FAA364B02C17F5A365F807EF
S31A0003ABEEB324370534013510275C37DC37B1A36437DC37550098
S31A0003AC030037380D0AB60AFCFB3735A368FA03AAD81735A365AC
S31A0003AC183F04350427F734103FFE276F376A000017F5340E3747
S31A0003AC2D05277B37380009B21027743402350837DC37B12926D0
S31A0003AC4237DCDD005B03AC4A37650000FA032464B02237650021
S31A0003AC5700FA03A3BAB01837650000FA03A5B4B00E3765000071
S31A0003AC6CFA03A99AB00437650000FA03AB603F02350427F73466
S31A0003AC8110276FFA039798273631D8B606373512C027F5FA036A
S31A0003AC9697F217F5340E3705277B7CFD373800063782005E27BF
S31A0003ACAB743402350837DC37B1295237DCDD005B03ACBE37350A
S31A0003ACC0258037B50002B03AFA03A1FCB038373512C027F5FA23
S31A0003ACD50397F23735293AFA03A1B0B0243735258027F5FA03BA
S31A0003ACEA97F237352946FA03A1B0B010373512C037B50003B0FD
S3140003ACFF023735258027F5FA0397F2350427F731
S31A0003AD0E7580D5003D02F1FC370EB4F24A003C0127F734203716
S31A0003AD234C37DCF5FF27FA379D37B57FFF277B2773FD2027736D
S31A0003AD38FD242773FD282773FD2C2773FD302773FD342773FD31
S31A0003AD4D382773FD3C375C27FB37B80010B30037B50010371132
S31A0003AD6227F9009437BDFD0037380008B3FE3698369637300005
S31A0003AD7710B2D6350227F73420F5FF27FA37B57FFF277B2773C2
S31A0003AD8CFD2037B50001366437B5FFFF3775FD02B7123731FC43
S31A0003ADA10027FC3775FD00B7063731FC0027FC37B6000335025D
S31A0003ADB627F73430374C277AF5FF27FA379DC50045013C023671
S31A0003ADCB042776B6F0350627F737BDFD1E3D0237BE000127FE61
S31A0003ADE0B40037BE7FFF9E0037300001B702377DFD3EB6E037B3
S31A0003ADF5DC37B0FD2027FF371A37FAFC1CF52275C337FAFC180C
S31A0003AE0A371517FAFC1F758037FAFC1A3A80FC1FFFFA3880FCF4
S31A0003AE1F1F27F73420F5FF27FAF5C317FAFC183804FC1738010A
S31A0003AE34FC173902FC173902FC153902FC163901FC16F540374E
S31A0003AE4907277B2773FD402773FD442773FD482773FD4C277532
S31A0003AE5E27FB27F02773FD2037B5010037FAFC1CF50017FAFCAE
S31A0003AE731EF5FF368837F5FD02B70427F0B70037B50001350219
S3070003AE8827F7A1
S31A0003AE8A3410276F3778A658B416277427743402351037CC376E
S31A0003AE9FB1A61437CCCD00D50037058602B0FE27F5350427F7A0
S31A0003AEB43410276F27FB37F1A65837F8A65AB50027F5B0362751
S31A0003AEC97B277427743402350837DC37B1A61437DC37550002F1
S31A0003AEDE37380001B702DD009500B014277B27742774340235B4
S31A0003AEF30837DC37B1A61437DCDD00D5003705350427F73410E8
S31A0003AF083FFC276F3771A65A3778A65CB41E277427743402358E
S31A0003AF1D0837DC37B1A61437DCDD00DC00AC00DD02AD023765B7
S31A0003AF320000A502B000277527F53F04350427F73410276F2757
S31A0003AF4736A65EB60027F5B05217FDA65E375500002774277404
S31A0003AF5C2774375100003402350837BC000534083540277527D5
S31A0003AF71FD27FC373200003729275C37DCFC4137DC3408352062
S31A0003AF86277A3717370527FF27FF27FF27FF27FF27FF27FF2751
S31A0003AF9B7A340835402778277D27FB350427F73410276F27367A
S31A0003AFB0A65EB60027F5B00417FDA65E950027FD350427F7349D
S31A0003AFC5103FFC276F376A0002AA0037F5A65C37B8000FB21E44
S31A0003AFDA277B277427743402350837DC37B1A61437DCEC029CBC
S31A0003AFEF00EC009C02277B7C01377AA65C3F04350427F734100A
S31A0003B0043FF8276F2735A65E2735A65C37B5A50C7A03B0D6ED16
S31A0003B01900D5083705277B37380003B728BE0637380002B7120F
S31A0003B02E7A03B0D237380004B74A37380005378700727A03B0C0
S31A0003B043D2376500007C0A37B500017A03B0CEED0037DCFC0A0D
S31A0003B05837DCAD043765000437B50004FA03AFC4ED04D500F65A
S31A0003B06D40B75E3765000437B50008FA03AFC43765000437B5E0
S31A0003B0820080B04427250002ED0237DC37B128DA37DCD50037E3
S31A0003B0970534013508376500007C0AFA03AFC427230002A5029F
S31A0003B0AC37B80007BFD4B01AA500FC0AAA063765000637B5004A
S31A0003B0C101FA03AFC43765000637B50004FA03AFC4A500FC1647
S31A0003B0D6AA0037F8A50A3785FF3617FDA65C17BDA65837B5A56A
S31A0003B0EB0C7A03B1ACED00D5083705277B37380009378200A6E2
S31A0003B10027743402350837DC37B1296037DCDD005B03B1143755
S31A0003B1156500007C0A377AA65E37B50002FA03AFC47A03B1A848
S31A0003B12A27250002ED0237DCFC0A37DC3408352037610000373E
S31A0003B13FB50001FA03AFC427230002A50237B80003BFD8B05050
S31A0003B154376500007C0A37B50002FA03AFC4376500007C0C3702
S31A0003B169B50001FA03AFC4B032376500007C0A37B50002FA03B3
S31A0003B17EAFC427250002ED0237DCFC0C37DC34083520376100AC
S31A0003B1930037B50001FA03AFC427230002A50237B80002BFD8C6
S31A0003B1A8A500FC16AA0037F8A50A3785FF3817FDA65C17BDA6C7
S31A0003B1BD5A37B5A50CB03EED00D508370537B80006B62E272564
S31A0003B1D2000237650002277427743402350837DCFC0A37DC34B6
S31A0003B1E70835203761000037B50004FA03AFC427230002A50202
S31A0003B1FC37B80001BFCEA500FC16AA0037F8A50AB5B23F083596
S31A0003B2110427F734103FFC276F376A000037BC0006AC02ED00B3
S31A0003B22637DCA10237DCD5003705277BFA039B8427210002BE6A
S31A0003B23BE43F04350427F734103FFC276F27FBEA00F604EA0270
S31A0003B2503735297A3716B70037352974FA039912E500F601B68A
S31A0003B2650437352980FA039912E500F610B7043735298AFA0348
S31A0003B27A99123F04350427F734103FFE276F376A000037352924
S31A0003B28F94FA03991237650000277DFA039C6037352996FA0304
S31A0003B2A499123F02350427F734103FFC276F376A0000FA03B2E4
S31A0003B2B9143735299AFA039912ED00D5083705277B373800096C
S31A0003B2CE3782016427743402350837DC37B129A237DCDD005B25
S31A0003B2E303B2E6ED003755000AFA03B2827A03B438ED00D50AC9
S31A0003B2F8F6017A03B36AED00D50A3705277BFA03B242ED00D54A
S31A0003B30D0AF640378701223735299CFA039912ED00D50A371F06
S31A0003B3223705277BFA03B2423735299CFA0399123735297AED69
S31A0003B33700160ABC36B0303735299EFA039912ED00D50A7A03E2
S31A0003B34CB3FAED00D50AF6013735297A3716B70037352974FA5D
S31A0003B361039912ED00D50AF6043735297A3716B700373529743E
S31A0003B376FA0399127A03B438272500023735299EFA0399123748
S31A0003B38B650002277427743402350837DCFC0A37DC34083520D7
S31A0003B3A037610000FA039DAA27230002A50237B80001BFCA7ACD
S31A0003B3B503B438272500023735299EFA039912ED0037DCA102BF
S31A0003B3CA37DCD50A3705277BFA039B8427230002A50237B80097
S31A0003B3DF03BFD6B050ED003755000AFA03B2823735299EFA03D4
S31A0003B3F49912ED00D50C3705277BFA039B84B030ED003755006F
S31A0003B4090AFA03B282272500023735299EFA039912ED0037DCC1
S31A0003B41EA10237DCD50C3705277BFA039B8427230002A5023755
S31A0003B433B80002BFD6FA039BD83F04350427F734103FFE276F8B
S31A0003B44827FBEA003410352037B50001FA03ADB83F0235042751
S31A0003B45DF734103FFE276F27FBEA00FA03AE223410352037B565
S31A0003B4720008FA03ADB83F02350427F734103FFC276F376A0004
S31A0003B48700AA02373500CCFA03B45E27260002B70CA50227F4E0
S31A0003B49C27F427F437650000FA03ADB82726000AB710376500A4
S31A0003B4B10037610002A50A27F427F427F4FA03AD203F0435049D
S31A0003B4C627F734103FFC276F27FBEA02341035207C02272500C4
S31A0003B4DB0037B50001FA03B47E3F04350427F734103FFC276F88
S31A0003B4F0376A0000AA0237350055FA03B45E3765000037B50099
S31A0003B50540FA03ADB82726000AB70CA50A27F427F427F43765D0
S31A0003B51A0002FA03ADB82726000CB710376500023761000AA5AA
S31A0003B52F0C27F427F427F4FA03AD203F04350427F734103FFAC0
S31A0003B544276F376A0000AA02373500F0FA03B45EEC00C50037B3
S31A0003B5590537B70100AA0427230000FA03AD7E340135103765AA
S31A0003B56E0004373600013402350837DC37B128DA37DCD50037BE
S31A0003B583053404352034013766FFFE3F02B61EE5053705277B6C
S31A0003B598FA03B442A50427FFAA0437B80001B6B827210002B6C7
S31A0003B5ADA237B50001B0FE27F53F06350427F734103FFA276F78
S31A0003B5C22725000217F5A6603705277B3738001F378700CABE59
S31A0003B5D7403738001037870096BE143738000137870074378F09
S31A0003B5EC00F837380005378700747A03B6E83738001B37870040
S31A0003B6018ABE0837380012378700747A03B6E83738001D3787C3
S31A0003B616007E7A03B6E837380028378700A4BE1E3738002237E0
S31A0003B62B870086BE0837380020378700727A03B6E837380026BF
S31A0003B6403787007A7A03B6E83738003A3787008C378E00923718
S31A0003B655380029378700767A03B6E8F50CEA0437B529B67A03F0
S31A0003B66AB6E6F502EA0437B529BC7A03B6E6250437B529C27ADD
S31A0003B67F03B6E6F503EA0437B529C87A03B6E6F508EA0437B55B
S31A0003B69429CEB04AF506EA0437B529D4B040F50BEA0437B529E2
S31A0003B6A9DAB036F507EA0437B529E0B02CF501EA0437B529E629
S31A0003B6BEB022F509EA0437B529ECB018F501EA0437B529F2B04C
S31A0003B6D30EF504EA0437B529F8B004F505EA0437B529FEAA02FC
S31A0003B6E8273635BCB7423735A660FA03B21437352994FA039909
S31A0003B6FD1227260002B71437650002FA0399123775A50A3738F3
S31A0003B712A614B51637352A04B00C17F5A6603705277BFA039BB6
S31A0003B7278437352A0EFA039912FA039BD827260002B74AE5048B
S31A0003B73CF809B22417FDA50A377DA614B41ADA0837B50008AA99
S31A0003B751003735A66037F5A50AFA039A703775A50A7C16377AE8
S31A0003B766A50AE5043705277B27743402350837DC37B128BA372D
S31A0003B77BDC3775A65637570000377AA6563F06350427F7341011
S31A0003B7903FFA276F3401350827FBEA0134083540EA02F601EACF
S31A0003B7A504B72EE501371F371F371F37053401351037CC37B114
S31A0003B7BAA66037CC277AE501277A373600073402350837DC370F
S31A0003B7CFB128DA37DCC500D700B02EE501371F371F371F3705F8
S31A0003B7E43401351037CC37B1A66037CC277AE501277A37360044
S31A0003B7F9073402350837DC37B128DA37DCD5003710C600CA00FC
S31A0003B80EE5023705277BFA03B4423F06350427F734103FFA2724
S31A0003B8236F27FBEA0127250002371F371F371FEA043705277B6F
S31A0003B8383402351037CC37B1A66037CC277AE501277A373600EE
S31A0003B84D073402350837DC37B128DA37DCC500D600EA04B70211
S31A0003B86237B50001AA02A5023F06350427F734103FFA276F27B2
S31A0003B877FBEA01373500F0FA03B45E2502B01EE5023705277BA8
S31A0003B88CFA03B81EEA0437143714F703EA003410352037B500DE
S31A0003B8A103FA03ADB82302E502E801B5D4F503EA00341035202B
S31A0003B8B637B50002FA03ADB83F06350427F734103FF6276F2752
S31A0003B8CBFBEA04F83FB258FA03AD7E277BEA05F8023782006C5D
S31A0003B8E03716B622E5043705AA063765000627F5FA03B78EE56B
S31A0003B8F504F101EA083705277BFA03B8C437650006FA03B8702F
S31A0003B90AE5043705277B37BD0000E505F802B70037BD000134A0
S31A0003B91F083540FA03B78E2304E504F83FB3A037B5008CAA008F
S31A0003B93437B50008AA023735A66027F5FA039852277B2776B6EB
S31A0003B94900FA03B5BC3F0A350427F734103FFE276FF50117FAB4
S31A0003B95EA6603735A66037B50001FA03B540EA00B70437350063
S31A0003B97308FA03B8C43F02350427F734103FFE276F27FB272518
S31A0003B9880000B014277BFA030810376500007C2D376A00003709
S31A0003B99D380167B208277B3736FFFD37380001B6DA37B8000335
S31A0003B9B2B606376500007C16376A0000A5003F02350427F7347B
S31A0003B9C7103FFE276F3402351037BD00103408354027F43401FF
S31A0003B9DC3508C500F854B2063408354037B70010B00AC500F821
S31A0003B9F1A9B2083408354037B700013401350837CCFC0137CCC0
S31A0003BA063408352037360100B7C034083520FA03B97E3F023571
S31A0003BA1B0427F734103FF0276F376A000EF5BEEA0437BD00019D
S31A0003BA30AD0037B50009AA0234103540FC04FA03B4EA341035DD
S31A0003BA45207C0537BD008CAD0037B50009AA0227F5FA03985271
S31A0003BA5A277B2776B70027F5B01E341035207C05FA0307782731
S31A0003BA6F7BED0E1608B702277D277D277DED0E375A000A37B5FE
S31A0003BA8400013F10350427F734103FFC276F376A000037B5005B
S31A0003BA9908FA03B5403716B708FA03AD7EEA02B704F803B70008
S31A0003BAAE27F5B008E502F601ED00DA0A37B500013F0435042767
S31A0003BAC3F73410276F27F5350427F734103FF2276F376A000C69
S31A0003BAD8F5F5EA04F5D5EA05F5FFEA0637BD0003AD0037B5004B
S31A0003BAED04AA0234103540FC04FA03B4EA37BDA001AD0037B509
S31A0003BB020007AA02341035207C0427F5FA039852277B3738B095
S31A0003BB1701B608E507ED0CDA0A37B50001B0FE27F53F0E35044B
S31A0003BB2C27F734103FF4276F3401350837B6000334013508F507
S31A0003BB4155EA04F507EA052506340835403714371437143714B0
S31A0003BB563714F71FEA0737B50004AA0037B50002AA02341035D2
S31A0003BB6B40FC04FA03B4EA37B5A001AA0037B50006AA023410C8
S31A0003BB8035207C0427F5FA039852340135082775377DB001B6A6
S31A0003BB95003735000127FB3F0C350427F734103FEC276F376ABB
S31A0003BBAA0012F5F0EA04F588EA05250637BD0003AD0037B50071
S31A0003BBBF0AAA0234103540FC04FA03B4EA37BDA001AD0037B530
S31A0003BBD4000DAA02341035207C0427F5FA039852277B3738B0BD
S31A0003BBE901B608E507ED12DA0A37B50001B0FE27F53F1435046D
S31A0003BBFE27F734103FF2276F376A000AF55AEA04F5FFEA052510
S31A0003BC130637BD0003AD0037B50002AA0234103540FC04FA0319
S31A0003BC28B4EAE507F8AAB608E508ED0ADA0A37B50001B0FE278A
S31A0003BC3DF53F0E350427F734103FF0276F376A000AF55AEA045F
S31A0003BC52F5FFEA05250637BD0003AD0037B50002AA023410350F
S31A0003BC6740FC04FA03B4EAE507F8AAB61EE508F4F0EA0C371F65
S31A0003BC7C371F371F371FE40CF60FEA0EB608E50CED0ADA0A37FA
S31A0003BC91B50001B0FE27F53F10350427F734103FE4276F376AD1
S31A0003BCA600122725001627250014F5A5EA0427260014B700F517
S31A0003BCBBFFB0FEF5DFEA05F501EA0637B50003AA0037B5000B85
S31A0003BCD0AA023765001234103540FC04FA03B4EA376500127C7E
S31A0003BCE512FA03021037B5A001AA0037B5000EAA0234103520AA
S31A0003BCFA7C0427F5FA039852277B3738B001B62A272300163473
S31A0003BD0F1035207C08FA030780376A0018AA1A376500142774E1
S31A0003BD2427743402350837DCA11237DCA5189A0AA51A9A0C272D
S31A0003BD39230014A51437B80001378FFF682775A51637B8000297
S31A0003BD4EB6003735000127FB3F1C350427F734103FF0276F34A3
S31A0003BD63013510ED1634083540EA0CF555EA0434043540EA05FE
S31A0003BD7837173705AA0EE50FEA0634083540EA0737B50004AA4B
S31A0003BD8D0037B50003AA0234103540FC04FA03B4EA37B5A0011C
S31A0003BDA2AA0037B50006AA02341035207C0427F5FA03985227F8
S31A0003BDB77B3738B001B70027F5B00A2775E50AE80CB6003735A5
S31A0003BDCC000127FB3F10350427F734103FFA276F376A000227B3
S31A0003BDE1250004EC0437CCFC0837CCED0437DC37B12A1A37DCDE
S31A0003BDF6D5003705AA003765000234043540FA03BD5C3716B610
S31A0003BE0B0027F5B00C27230004EC04377C0007B3C437B50001E5
S31A0003BE203F06350427F734103FEC276F376A0012F5AAEA0425FE
S31A0003BE3505250637BD0003AD0037B5000AAA0234103540FC04C0
S31A0003BE4AFA03B4EA37BDA001AD0037B5000DAA02341035207C43
S31A0003BE5F0427F5FA039852277B3738B001B614E508ED12DA0A62
S31A0003BE74E50ADA0BE50CDA0CE50EDA0D37B50001B0FE27F53F35
S31A0003BE8914350427F734103FF6276FF53CEA04F50FEA05F555C5
S31A0003BE9EEA0637B50002AA00341035207C0437B50003FA03B445
S31A0003BEB37E37B5A001AA0037B50005AA02341035207C0427F5EA
S31A0003BEC8FA039852340135082775377DB001B6003735000127B8
S31A0003BEDDFB3F0A350427F734103FF2276F376A00083765000458
S31A0003BEF2373600FF376A00043737B200376A00043736FF0037B9
S31A0003BF076A000437370060376A0004275E37DCFC0437DCAD0AD9
S31A0003BF1C37B50002AA0037BD0002AD0237650008A50AFA03B4C6
S31A0003BF31EAED0A37DCFC0237DCAD0C3765000CFA030778277B6E
S31A0003BF46277D277D277D277D277D277D277DED08375A000AF5DC
S31A0003BF5BB2EA04F577ED0ADA0137B50002AA0037BD0002AD02AD
S31A0003BF7037650008A50AFA03B4EA3765000CFA030778277B27D8
S31A0003BF857F277F27FBED08DA0C37B500013F0E350427F73410A7
S31A0003BF9A3FFA276FF54EEA022503F501EA0427250000341035BA
S31A0003BFAF207C0237B50003FA03B47E3F06350427F734103FFC9D
S31A0003BFC4276F37650002373600FF376A00023737B800376A0055
S31A0003BFD9023736FF00376A0002341035207C022725000037B5EA
S31A0003BFEE0002FA03B47E3F04350427F734103FEE276F376A00C2
S31A0003C00310F5BEEA04250537BD0002AD0037B50009AA023410BC
S31A0003C0183540FC04FA03B4EA341035207C0637BD008CAD00377B
S31A0003C02DB50009AA0227F5FA039852277B2776378600563410F2
S31A0003C04235207C07FA030778277B277D277D277D277D277D278F
S31A0003C0577D277DED10375A000A341035207C0BFA030778277BD4
S31A0003C06C277F277F277F27FBED10DA0C341035207C09FA03079D
S31A0003C08178277B277F277F27FBED10DA0DF5FFDA0E37B500016C
S31A0003C096B0FE27F53F12350427F734103FFE276F376A0000ED75
S31A0003C0AB00D5083705277B373800093782007E277434023508FF
S31A0003C0C037DC37B12A2237DCDD005B03C0CE37650000FA03BAEC
S31A0003C0D51E3705B05E37650000FA03BA8C3705B052376500002C
S31A0003C0EAFA03BACE3705B04637650000FA03BC003705B03A37CF
S31A0003C0FF650000FA03BC443705B02E37650000FA03BC9E370578
S31A0003C114B02237650000FA03BE263705B01637650000FA03BE65
S31A0003C129E43705B00A37650000FA03BFFA3705B0FE27F53F0285
S31A0003C13E350427F734103FFE276F3735A50CB01C37650000FAF6
S31A0003C15303C0A03716B70A273635BCB70437650000FA03B2AC5D
S31A0003C168376500007C16376A00003778A50AB5D23F0235042764
S31A0003C17DF73410276F2736A656378700703775A6563736030034
S31A0003C192B7243775A6547C01377AA65437360001B7063735004F
S31A0003C1A7B4FA03B4C8B04A3775A65637360200B700FA03BFC009
S31A0003C1BCFA03C1422736A65CB600FA03B0021736A657BC00FAA1
S31A0003C1D103BE8E3775A65637360203B70437350044FA03B4C803
S31A0003C1E63775A65637360100B704373500D2FA03B4C8FA03B9FD
S31A0003C1FB54350427F73410276F2736A50AB600FA03AE222735B6
S31A0003C210A6562735A65A2735A6582735A65C37BDA50C17BDA5E2
S31A0003C2250A3735A50C37B50108FA039A44FA03AE223716B7181B
S31A0003C23A373500F0FA03B45E2775FA03B8C43775A6563736024F
S3100003C24F00B700FA03BF98350427F779
S31A0003C25A3410276F27F537BDA6A49800B4FE950037DCFC02376B
S31A0003C26FDC377DA6E0B5EA350427F734103FFE276F277517FDDE
S31A0003C2842A38F506EA0037DCFCFE37DC377DA6A4B40037BDA6E9
S31A0003C299DE375100002100B6E437BC000627FB372A340435403D
S31A0003C2AE3F02350427F734103FF4276F27250004272500062704
S31A0003C2C32500082725000A37BDA674A5069102AA06A504D30161
S31A0003C2D85300AA04A50A9106AA0AA508D3055304AA0837DCFCB0
S31A0003C2ED0837DC377DA6A4B5D4EC08AC00EC0AAC0237650004AD
S31A0003C302A506FA03C6A43F0C350427F734103FFA276FFA030554
S31A0003C317AAAA02FA03AFAA34013508377DFFCEBC0237BDFFCEEA
S31A0003C32CB006377D0064BF0037BD006437650002373828F5B331
S31A0003C341063731D70A376A0002B00027250002340835403735D1
S31A0003C35600463726AA0437BD86FD375C2779375CAD00376500F2
S31A0003C36B0237B53F01FA03050AAA02376500027C64376A0002AD
S31A0003C38037BC00C8A502372A377C0064B30037BC00643404354E
S31A0003C395403F06350427F734103FF4276FAA00B60237B5000152
S31A0003C3AAAA002502373800B3B300F501EA022602B7003731FFA7
S31A0003C3BF4CFA03968437650000FA0304CE376A0004AA06260215
S31A0003C3D4B60437650004A506B01237650004A506FA039AB237B9
S31A0003C3E96A0008AA0A37650008A50A3F0C350427F734103FF4A4
S31A0003C3FE276F376A0000AA02FA03C39C376A0004AA06A500FCEC
S31A0003C4135AAA0037B80167B30237B1FE98AA0037650000A50290
S31A0003C428FA03C39C376A0008AA0AFA0302C817FD2A36A5049ABF
S31A0003C43D00A5069A02A5089A04A50A9A0637DCFC0837DC17BD02
S31A0003C4522A36377DA6A4B50437B5A67437FA2A3617FD2A38A503
S31A0003C467129A0037752A387C02377A2A383738A6E0B50437B5D2
S31A0003C47CA6A437FA2A38FA0302D63F0C350427F734103FFE27A6
S31A0003C4916F37BD0298AD0037B50241FA03050A3F02350427F710
S31A0003C4A634103FFE276F37BD03EEAD0037B50653FA03050A3F3F
S31A0003C4BB02350427F734103FEE276F376A000434103520FA03C8
S31A0003C4D00452376A000AAA0CA50C37F0A66EAA08A50A17F2A69B
S31A0003C4E56D1772A66CAA06A50837F1A66EAA10A50617F3A66D16
S31A0003C4FA1773A66CAA0EED0E17BDA66CEC1017BCA66E272600BF
S31A0003C50F06B3062725000637BDFFFFAD08ED08EC048D00A5023D
S31A0003C52437F0A66AAA08A50017F2A6691772A668AA06EC001709
S31A0003C539BCA668ED0217BDA66A27260006B3042725000627259F
S31A0003C54E0008A5083F12350427F734103FF6276F341035207C4E
S31A0003C56302FA03C4C0AA04378700BEFA03CD22277B27743402AE
S31A0003C578350837DC37B12A3A37DC375500003402350837DC37AD
S31A0003C58DF1357437DC373501683408354034023510372AAA08CF
S31A0003C5A23765000217FD34F6A504AA0034083540FA03050A2768
S31A0003C5B77B37BD000A274D372AAC06ED02AC00376500083408EB
S31A0003C5CC3540FA03C3FA17363576B75237352ABAFA03991237F2
S31A0003C5E1650008FA039BE837352ABEFA03991237650006FA03B4
S31A0003C5F6C4A6277BFA039BE837352AC2FA039912FA03AFAA271E
S31A0003C60B7BFA039C6037352ACAFA039912FA03C30E277BFA0328
S31A0003C6209BE837352AD0FA039912FA039BD83F0A350427F73427
S31A0003C635103FFA276F376A0002AA04EC0C275E37DCFC0C37DC0C
S31A0003C64AEC0E9C023765000C375700022776B61C27F5B03C3457
S31A0003C65F1035207C0237B50001FA030516341035207C0C37B5C8
S31A0003C6740001FA0305162726000CB2DAA504EC0EAC00373500EF
S31A0003C68937FA03050A3401350837DC37B12AD237DCD5003705C3
S31A0003C69E3F06350427F734103FEA276F376A0004AA06376500EE
S31A0003C6B31C376A00083765001E376A000A2725000C2726000496
S31A0003C6C8BC2837650004A506FA039AB2376A000EAA10376500D7
S31A0003C6DD0E376A000437650010376A00063765000C3737000221
S31A0003C6F2376A000C27260008BC2837650008A50AFA039AB23771
S31A0003C7076A0012AA1437650012376A000837650014376A000A28
S31A0003C71C3765000C37370001376A000C3765000837680004BE36
S31A0003C73108B6223765000A37680006B31837650008376A0000AF
S31A0003C7463765000A376A000237650004A506FA03C634B0223741
S31A0003C75B650004376A000037650006376A000237650008A50A1E
S31A0003C770FA03C63437BD005A34083520277927FB3765000C3734
S31A0003C785380001B70CB52437380002B70A37380003B714B0168C
S31A0003C79A37BD00B4B00037BD0168375C2779375C34083540B0A5
S31A0003C7AF0037B100B43F16350427F734103FF4276F376A000274
S31A0003C7C4FA03C2B4AA04FA03C27A277BFA03C48C277B376A00CB
S31A0003C7D90037650002A504FA03277AAA06F567ED06DA0037DC71
S31A0003C7EEFC0137DCAD08FA03C25A3401351037650008FA03092B
S31A0003C80306F574ED06DA0437DCFC0537DCAD0AFA03AF423401D6
S31A0003C81835103765000AFA0324F6ED0637DCFC0837DCAD02FA3A
S31A0003C82D03C30E3401351037650002FA030906F568ED02DA00CF
S31A0003C842ED0637DCFC0B37DCAD02A5023F0C350427F734102755
S31A0003C8576F3775A67037F5A672FA0302743716B7103735A67045
S3190003C86C37B5000AFA030226FA03C17EFA03C558350427F7E7
S31A0003C88034103FFE276F27FBEA003775A6E27C01377AA6E23756
S31A0003C89578A6E8B604373500C0FA03CCA4E50037053401350899
S31A0003C8AA37DC37B1A6EA37DCD5003705277BFA03CCB63F02352A
S31A0003C8BF0427F73410276F3402350834083540373500A5F81F13
S31A0003C8D4B3003705277BFA03C880350427F734103FFE276F37CB
S31A0003C8E96A0000B00CED00D500370527230000277BFA03C880DC
S31A0003C8FEED001600B6E63F02350427F734103FFC276F376A002F
S31A0003C91300AA02B00CED00D500370527230000277BFA03C8806F
S31A0003C92837650002272100022776B6E03F04350427F734103FB9
S31A0003C93DFC276F376A0000AA02B00CED00D500370527230000F9
S31A0003C952277BFA03C8C237650002272100022776B6E03F04350B
S31A0003C9670427F73410276F3778A6E4B3003775A6E47CFF377A68
S31A0003C97CA6E02735A6E227743402350837DC37B12B0C37DC37A9
S31A0003C99155000037370080FA03CCA437F5A6E6350427F7341085
S31A0003C9A6276F3775A6E23778A6E6B50027F5B0063775A6E62788
S31A0003C9BBFB37F0A6E2350427F73410276FB00437350020FA0346
S31A0003C9D0C8803775A6E23778A6E6B5EA350427F734103FFC27F6
S31A0003C9E56F376A0000AA022774277427747C40FA03CCA4272532
S31A0003C9FA0000ED02D500370527230002277BFA03CCB627230068
S31A0003CA0F00ED00377D0007B3E03F04350427F734103FFE276F1D
S31A0003CA24376A000037BC0032A500372AAC00377C0008B30237D5
S31A0003CA39B50008AA003775A7F237680000B74AB42637BD00784D
S31A0003CA4E3408352037600000FA03CCA4373500FFFA03CCB63714
S31A0003CA6375A7F27C01377AA7F237680000B5E4B01E37350078F6
S31A0003CA783770A7F2FA03CCA42775FA03CCB63775A7F27CFF37E1
S31A0003CA8D7AA7F237680000B2E63F02350427F73410276F373563
S31A0003CAA2000337B52B14FA03C9E03735000437B52B1CFA03C939
S31A0003CAB7E03735000537B52B24FA03C9E03735000637B5A7EA40
S31A0003CACCFA03C9E02735A7F23735000737B52B2CFA03C9E0272E
S31A0003CAE1753402350837DC37B1A6EA37DC27FBDA007C013738C9
S31A0003CAF600FFB3E4F50717FAA7CF17FAA7AFF5E117FAA7CE172F
S31A0003CB0BFAA7AEF5EF17FAA7E017FAA7C0F5F517FAA7E617FA30
S31A0003CB20A7C6F5DF17FAA79AF5A417FAA746F5EB17FAA768F5D8
S31A0003CB350717FAA77617FAA77917FAA77017FAA76BF5E117FA4A
S31A0003CB4AA76E17FAA77817FAA77417FAA76AF5EF17FAA77E1709
S31A0003CB5FFAA78317FAA78417FAA76F350427F734103FFE276FC3
S31A0003CB74376A0000FA039AC637FAA6E4376500007C02FA039A39
S31A0003CB89C637FAA6E62735A6E22735A6E03775A6E437BD00001B
S31A0003CB9E37380001B60637B80010B60037BD000917BDA6E83702
S31A0003CBB3350038FA03CC9837350005FA03029437350038FA03F1
S31A0003CBC8CC9837350005FA03029437350038FA03CC9837350076
S31A0003CBDD05FA03029437350028FA03CC9837350005FA030294A9
S31A0003CBF23775A6E437380001B6063775A6E637380010B602371D
S31A0003CC07350028B00037350020FA03CCA437350008FA03CCA428
S31A0003CC1C3735000CFA03CCA437350006FA03CCA437350002FACE
S31A0003CC3103CCA437350005FA0302943735000FFA03CCA437351A
S31A0003CC46000CFA03CCA4FA03CA9C37350004FA03C96A373509DF
S3140003CC5BD6FA03C8E2FA03C9C43F02350427F722
S31A0003CC6A370527FF27FF27FF27FF373B00E01775FA4117FAFAB4
S31A0003CC7F41F74017FAFA41F6BF17FAFA41274C177AFA41373A22
S31A0003CC94FF1F27F73420F5FF27FA27FB36C4B0223420F5FF2780
S31A0003CCA9FA27FB36B827FBF60F36BCB0103420F5FF27FA27FBFF
S31A0003CCBE750236A627FBF60FF72036A6350237B5001937B000C8
S31A0003CCD301B6F627F73420371527FA37B5073A37FA008CF5FFD9
S31A0003CCE827FA371517FAFA1717FAFA11F53417FAFA15380CF9FD
S31A0003CCFD1E3820F9243920F920350227F73420F5FF27FA37150A
S31A0003CD1217FAFA1717FAFA1117FAFA15350227F73420F5FF27E1
S31A0003CD27FA1775F90C17F5FA11350237B6083771FF3707371CE8
S3110003CD3C37B6300F370B3717370527F7CC
S31A0003CD48375C277B37B50002379C37BC800037F5357A37CD275E
S31A0003CD5DF7342036E2C500DA003D013C0137300001B6EE3502F8
S31A0003CD7227F7342036CCC500D800B6063D013C0137300001B63D
S30C0003CD87EC27FB350227F739
S31A0003CD8E554E4B4E4F574E20455843455054494F4E00554E4B9A
S31A0003CDA34E4F574E20494E5445525255505400425245414B508E
S31A0003CDB84F494E5400425553204552524F5200534F46545741BB
S31A0003CDCD524520494E5445525255505400494C4C4547414C20AA
S31A0003CDE2494E535452554354494F4E004449564953494F4E204C
S31A0003CDF74259205A45524F00554E494E495449414C495A45444A
S31A0003CE0C20494E54455252555054004C4556454C312041564576
S31A0003CE2143004C4556454C322041564543004C4556454C3320FC
S31A0003CE3641564543004C4556454C342041564543004C455645A8
S31A0003CE4B4C352041564543004C4556454C362041564543004CD0
S31A0003CE604556454C3720415645430053505552494F555320491F
S30E0003CE754E544552525550540027
S31A0003CE7E00010001000100010001000100020002000200020088
S31A0003CE930200020003000300030003000300040004000400055D
S31A0003CEA8000500050006000600070007000800090009000A0024
S31A0003CEBD0B000C000D000E000F001000110013001400160017A1
S31A0003CED20019001B001E0020002200250028002B002F003300D4
S31A0003CEE737003B00400045004A00500057005E0065006D00769F
S31A0003CEFC0080008A009500A100AE00BB00CA00DB00EC00FF01DE
S31A0003CF111301290141015B0177019501B501D801FE022602530E
S31A0003CF26028202B502ED0329036A03AF03FBFFFF0004080D1152
S31A0003CF3B161A1F23282C3035393D42464A4F53575B5F64686C7A
S31A0003CF507074787C7F83878B8F92969A9DA1A4A7ABAEB1B5B886
S31A0003CF65BBBEC1C4C6C9CCCFD1D4D6D9DBDDDFE2E4E6E8E9EB33
S31A0003CF7AEDEEF0F2F3F4F6F7F8F9FAFBFCFCFDFEFEFFFFFFFF35
S31A0003CF8FFFFFFFFFFFFFFFFEFEFDFCFCFBFAF9F8F7F6F4F3F2EE
S31A0003CFA4F0EEEDEBE9E8E6E4E2DFDDDBD9D6D4D1CFCCC9C6C463
S31A0003CFB9C1BEBBB8B5B1AEABA7A4A19D9A96928F8B87837F7C3F
S31A0003CFCE7874706C68645F5B57534F4A46423D3935302C2823DA
S31A0003CFE31F1A16110D0804000A6E6F70096E6F7468696E670A56
S31A0003CFF876657273696F6E09736F6674776172652076657273C1
S31A0003D00D696F6E0A7265626F6F74097761726D207265626F6F33
S31A0003D022740A72657374617274096C657373207468616E206161
S31A0003D037207265626F6F740A666163746F727964656661756CBD
S31A0003D04C747309726573657420706172616D65746572730A70E5
S31A0003D061726F66696C65206E0973656C6563742070726F6669D9
S31A0003D0766C65206E756D626572206E0A6368616E6E656C206E23
S31A0003D08B0973686F77206368616E6E656C206E20286F7220618C
S31A0003D0A06C6C290A6368616E6E656C206E2072096368616E6E5D
S31A0003D0B5656C206E2069732073696D706C657820617420722039
S31A0003D0CA6B487A0A6368616E6E656C206E20722074096368614F
S31A0003D0DF6E6E656C206E206973206475706C657820722F740A0B
S31A0003D0F472656D6F74652063616C6C09636F6E6669677572650B
S31A0003D10920616E6F74686572207365742076696120726164696B
S31A0003D11E6F0A6469737009616C6C20706172616D657465727334
S31A0003D1330A6469737020746B6476730973656C65637420737547
S31A0003D14862736574206F6620706172616D65746572730A7770E1
S31A0003D15D745F7374617368096174206D6F737420313030206CC0
S31A0003D172617465737420776179706F696E74730A7374617409A1
S31A0003D187736F6D6520696E707574207374617475730A70657271
S31A0003D19C6D096E6F6E766F6C6174696C6520736176650A09630F
S31A0003D1B168616E676573206172652074656D706F72617279206F
S31A0003D1C66F74686572776973650A68656C7020666F6F09646588
S31A0003D1DB73637269626520706172616D6574657220666F6F0A6F
S31A0003D1F0666F6F0973686F7720706172616D6574657220666F3D
S31A0003D2056F0A666F6F206261720973657420706172616D65749A
S31A0003D21A657220666F6F20746F2022626172220A736574206643
S31A0003D22F6F6F09636C65617220706172616D6574657220666F1D
S31A0003D2446F0A0A0021706F6C69636500236469676900247068F0
S31A0003D2596F6E650027616972637261667400276165726F706C58
S31A0003D26E616E65002A736E6F776D6F62696C65002B726564633C
S31A0003D283726F7373002D686F757365002E78002F646F74003029
S31A0003D298300031310032320033330034340035350036360037A7
S31A0003D2AD37003838003939003A66697265003B63616D70003C52
S31A0003D2C26D6F746F726379636C65003C62696B65003E636172C2
S31A0003D2D7004161696400456579650048686F74656C004B7363BD
S31A0003D2EC686F6F6C004F62616C6C6F6F6E0050706F6C69636570
S31A0003D301005272760055627573005868656C69636F70746572AE
S31A0003D31600597961636874005B6A6F67676572005C74726961A2
S31A0003D32B6E676C65005F77780061616D62756C616E6365006285
S31A0003D34062696379636C6500646761726167650064666972651F
S31A0003D355646570006666697265747275636B0067676C696465E0
S31A0003D36A720068686F73706974616C006A6A656570006B747208
S31A0003D37F75636B006E6E6F6465006F656D657267656E63796F9C
S31A0003D39470006F656F630070726F766572007070757070790019
S31A0003D3A972616E74656E6E610073736869700073706F77657248
S31A0003D3BE626F61740074747275636B73746F7000757472756315
S31A0003D3D36B007676616E00777761746572007979616769002138
S31A0003D3E8656D657267656E63790023677265656E646967690097
S31A0003D3FD276372617368002B636875726368002D6866686F75EB
S31A0003D41273650039676173003B7069636E6963003F696E666F14
S31A0003D4270041626F78004C6C69676874686F757365004E6E61B8
S31A0003D43C7669676174696F6E00507061726B696E67005272650C
S31A0003D4517374617572616E740058706861726D6163790000009E
S31A0003D466000000010253000203AE000304780004050800050505
S31A0003D47B78000605D300080663000A06D3000C072E000F079EF4
S31A0003D4900013081400170874001C08D600220938002909950098
S31A0003D4A53109EE003B0A4B00470AA800550B0200650B59007815
S31A0003D4BA0BAF008F0C0700AA0C5D00CA0CB300F00D0A011E0D29
S31A0003D4CF6101540DB801940E0E01E00E65023B0EBC02A70F12EE
S31A0003D4E403270F6903BF0FBF04741016054A106C064910C20767
S31A0003D4F978111808DF116E0A8A11C50C85121B0EDF127111AABB
S31A0003D50E12C714FB131D18EC13731D9A13CA2328142029C1144C
S31A0003D52376319714CC3AE6152245F41578531515CE62AD16241B
S31A0003D5387532167A8B3116D0A5501726C456177DE92E17D3FF1C
S3080003D54DFF1801BA
S31A0003D55037BCCD8E7A0300FE37BCCDA07A0300FE37BCCDB27A2D
S31A0003D5650300FE37BCCDBD7A0300FE37BCCDC77A0300FE37BCBA
S31A0003D57ACDDA7A0300FE37BCCDEE7A0300FE37BCCDFF7A03000C
S31A0003D58FFE37BCCE177A0300FE37BCCE237A0300FE37BCCE2FDE
S31A0003D5A47A0300FE37BCCE3B7A0300FE37BCCE477A0300FE37BD
S31A0003D5B9BCCE537A0300FE37BCCE5F7A0300FE37BCCE6B7A03B8
S3070003D5CE00FE54
S31A0003D5D0274C343FF5FF27FA27330102B600273301002731017B
S31A0003D5E50EB606F50417FA010E2733011037F5010427F427F473
S31A0003D5FA27F437F0010437F1F71227FF27FF27FF37FA010427CC
S31A0003D60F36010CB7062731010CB6003804FA412736010AB7004C
S31A0003D6242731010A373B0060373AFF3F27310106B60E17F501D4
S31A0003D6391917F80117B704FA00032AF5FF27FA273301062736DE
S31A0003D64E010AB62027310108B616371527FA379C379D17FC2465
S31A0003D6630A89030000277BF5FF27FA377A010A27330108357E8A
S3070003D678277709
S31A0003D67A3715379D3710379C37B5FF00372F37BD088817FC016F
S31A0003D68F1827B027B77BE27BE27BE27BE27BE27BE27BE27BE2C8
S31A0003D6A47BE27BE27BE227B4BAFE2772377A011A17FC01182706
S31A0003D6B9B027B77BE27BE27BE27BE27BE27BE27BE27BE27BE280
S31A0003D6CE7BE27BE227B4BAFE27723770011A374A000027B02717
S31A0003D6E3B77BE27BE27BE27BE27BE27BE27BE27BE27BE27BE2D0
S31A0003D6F87BE227B437F5011C377A011C3775011E373100BF379C
S31A0003D70DF4011CBA06342027F9012E35022775377A011E17F5DB
S31A0003D7220119F10217FA011917F801173786FF5427F73425F50E
S31A0003D737FF27FA379C17FC01124B00000037B5008037F1F90AD9
S31A0003D74C37FAF9163810F92217BC0112355227773A01F70FFFD1
S31A0003D761E237F5F72027FD37FA011437BC04203A04F70FFFCEF3
S31A0003D77637F5F72427FD37F1011417FC01168A0037CCF102172C
S31A0003D78BFA011737BC04423A10F70FFFAC37F5F72827FD37FA9A
S31A0003D7A0011437BC04563A40F70FFF9837F5F72C27FD37F10156
S31A0003D7B51417FC01168A0037CCF10217FA011737BC040CB08E2E
S31A0003D7CA3738231CB456273C2C12273C2C1017FC2C0EB72C1702
S31A0003D7DFF508CAF840B634850237B80011B52C37B80201B4260F
S31A0003D7F42705000037CC37BC5E1CB0FECC0027060000B6F48AA0
S31A0003D8090027352C0E17FC5E1EB72E17BC2C0E850037FA5E1EB8
S31A0003D81E27050002F58017FA08CA27F727352C1227352C1017FF
S31A0003D833FC2C0EB70A27352C0E37F55E1E8A0017BC5E1E27F7AB
S31A0003D848371527FA379C37300282B5D237381E183784FF6C271E
S31A0003D85D3C2C12273C2C1017FC2C0EB7D837380504B54A3738D2
S31A0003D8720A08B54237380F0CB53A37381410B53237381914B54B
S31A0003D8872A3602360036FE36FC373B0100173E08CAB5FE27F71A
S31A0003D89C85022703000237B601FF37CD177508CA4A0475801712
S31A0003D8B17A08CA27F736D436D236D036CE173F08CAB5D427F704
S31A0003D8C63425366CB45E37F52C0037B430A037FA2C0035522719
S31A0003D8DB7734253656B448273F2C06B54237F52C0037B430A035
S31A0003D8F037FA2C0017362C06B63017FC2C08B7227580C5043743
S31A0003D905FA2C0685023C0417BC2C0A37CD17BC2C0C273508CBCA
S31A0003D91A37B5064A37FA008A3552277737B5062C37FA008A35C5
S31A0003D92F5227773425360035522777371527FA379C37F52C009E
S31A0003D94437F12C0237FA2C023717370537CC17C508CC37BC00E0
S31A0003D9590017CAF92637B5004037C1F91637CAF9160810F9223A
S31A0003D96E37B512C037F12C0437FA2C0427F7342536B6B4A8372E
S31A0003D983F52C0037B430A037FA2C0037B5057637FA008A3552A4
S31A0003D998277734253698B48A177508CB3703273F2C06B50A3747
S31A0003D9ADF52C0037B430A037FA2C0037057805B722177A08CB2D
S31A0003D9C217362C06B61417FC2C0A3C01177C2C0CB71417BC2CE3
S31A0003D9D70A7580C50037FA2C063552277727342C063552277734
S31A0003D9EC37B5807E37FA2C0637B5058C37FA008A17FC2C0885CC
S3180003DA010037FA2C0837F535C48A0017BC35C43552277704
S31A0003DA143421F5FF27FA3820F92327330122B600273301203533
S3080003DA2942277711
S31A0003DA2C34273715379C371027FA2771FC0C37360040B71437AB
S31A0003DA41BC830A37451000278A7C0237360FFF374A1000357210
S31A0003DA5627773A01FC0C002837BC93103745100237481000B73F
S31A0003DA6B1227C5370537FAFC0E7C0137360FFF374A10023572F6
S30F0003DA8027773880FC0B35722777F1
S31A0003DA8A3421F5FF27FA3820F92217F5FA111775F90C37B68884
S31A0003DA9F0337B48803B60C371527FA17FA31A837B5078637FA2D
S31A0003DAB4008C3542277717F5FA11F603F403B60C17F5F90CF6E3
S31A0003DAC988F488B7023714F503F30027F73421F5FF27FA17F5B8
S31A0003DADEFA111775F90C37B6880337B48803B61037B527103780
S31A0003DAF3F1F91837FAF9183820F92235422777F52017FAFA1514
S31A0003DB08370536AAB616F51017FAFA157104369EB60AF50417D9
S31A0003DB1DFAFA1571043692B6FE27F5370BF53417FAFA153820F1
S31A0003DB32F9223706B724371527FA379C379D340E371A277B3722
S31A0003DB47BC09EB27C517FA31A8277BFA039394353837B5073ADA
S30D0003DB5C37FA008C35422777E6
S31A0003DB643460374C37B50002379C27FA373B00E075AA177A5553
S31A0003DB79557555177A2AAA7580177A555575AA177A55557555B6
S31A0003DB8E177A2AAA75304A000A800000FFFA350327F734603781
S31A0003DBA34C37DC37B50002379C27FA37DC373B00E075AA177A0E
S31A0003DBB855557555177A2AAA75A0177A5555CA0037074400BB1F
S30A0003DBCDF6350327F7FE
S30B0003DBD200010100000042
S31A0003DBD807B606D5FEC9F4EDF4B5002D0BBD0B1600DBF8FCF869
S31A0003DBED5A084102CEF337FDF611B50007EE5414100CD5FD3940
S31A0003DC02F7C9FACAFAAA01AD1117219628BB2196111701ADFAE5
S31A0003DC17AAFACA8000808386898C8F9295989B9EA2A5A7AAAD97
S31A0003DC2CB0B3B6B9BCBEC1C4C6C9CBCED0D3D5D7DADCDEE0E23C
S31A0003DC41E4E6E8EAEBEDEEF0F1F3F4F5F6F8F9FAFAFBFCFDFDDA
S31A0003DC56FEFEFEFFFFFFFFFFFFFFFEFEFEFDFDFCFBFAFAF9F8ED
S31A0003DC6BF6F5F4F3F1F0EEEDEBEAE8E6E4E2E0DEDCDAD7D5D3B1
S31A0003DC80D0CECBC9C6C4C1BEBCB9B6B3B0ADAAA7A5A29E9B98A7
S31A0003DC9595928F8C8986837F7C797673706D6A6764615D5A58BE
S31A0003DCAA55524F4C494643413E3B393634312F2C2A28252321A4
S31A0003DCBF1F1D1B1917151412110F0E0C0B0A090706050504030F
S31A0003DCD402020101010000000000000001010102020304050513
S31A0003DCE90607090A0B0C0E0F1112141517191B1D1F2123252865
S31A0003DCFE2A2C2F313436393B3E414346494C4F5255585A5D6171
S30E0003DD1364676A6D707376797C0E
S31A0003DD1C4028232948414D4452203132302030322E30312E32A5
S31A0003DD31303036204D4452313530003923363338303532372AB0
S31A0003DD4634310A260A1E0A180A0C0A0400005363616E6E6572F2
S31A0003DD5B004469676970656174657200004B49535300005472AC
S31A0003DD7061636B657200566F696365000A460A420A3C0A360077
S31A0003DD850035306D5700003230306D57003157000035570000ED
S31A0003DD9A0AAA0AA20A980A920A8C0A820A780A700A680A6000D3
S31A0003DDAF004F6E636F7265000053656154616C6B005A6F6469B5
S31A0003DDC46163000045617274684D61746500547269704D617441
S31A0003DDD9650000536952460000416973696E004D6167656C6C2D
S31A0003DDEE616E00004761726D696E000067656E65726963000A03
S31A0003DE03FC0AF60AF00AEA0AE40ADE0AD80AD20ACC0AC80000DB
S31A0003DE18317838003278343000003278323400003478323000DF
S31A0003DE2D00327832300000317832300000347831360000327803
S31A0003DE42313600003178313600006E6F6E6500000B120B100B58
S31A0003DE570A00006175746F0000320031000AFC0BAA0BA20B9A7A
S31A0003DE6C0B920B8A0B820B7A0B740B6E0B680B620B560B4A0BBB
S31A0003DE81400B360000776573742B7769646500656173742B771C
S31A0003DE9669646500736F7574682B7769646500006E6F7274680A
S31A0003DEAB2B776964650000776573740000656173740000736F33
S31A0003DEC0757468006E6F72746800776964652D37000077696477
S31A0003DED5652D360000776964652D350000776964652D34000052
S31A0003DEEA776964652D330000776964652D320000776964652D33
S31A0003DEFF3100000C220C180C0C0C020BF80BF00BE60BDC0BDAA1
S31A0003DF140B120B100BD80BD60BD40BD200003600350034003365
S31A0003DF29003000656D657267656E6379007072696F7269747969
S31A0003DF3E00007370656369616C00636F6D6D69747465640072AC
S31A0003DF53657475726E696E6700696E2D7365727669636500004F
S31A0003DF68656E2D726F75746500006F66662D6475747900000C32
S31A0003DF7D3A0C340AFC00004D49534F00004454523200000AFCAC
S31A0003DF920C480C3A00002A000C5C0C580C5200004D49432D4538
S31A0003DFA700696400006F6666000C760C6E0C6800006974656D35
S31A0003DFBC00006F626A65637400006E6F726D616C00000AFC0C35
S31A0003DFD16E0C6800000AFC0C960C8E00006B6579706164000090
S31A0003DFE677656174686572000AFC0CAC0CA60000776964650014
S31A0003DFFB0072656C617900000521C6344A001000000000000071
S31A0003E01021A6FF000006219A31C700010000000009F8218EFFC3
S31A0003E025000003218631D800020000000000002158FF000003AD
S31A0003E03A214E33840002000000180000212CFF000006212234BF
S31A0003E04F1B0001000000000B0220FCFF00000320F434F2000230
S31A0003E06400000000000020CCFF00000720C631B20004000237A6
S31A0003E07930000020A4FF000007209C31B60004000000000000E8
S31A0003E08E2086FF000001207A35720001000000000000205AFF13
S31A0003E0A3000003205434620002000000000000203211000001EC
S31A0003E0B8202831F100010000000000002006110000031FFC3456
S31A0003E0CD1800020000001E00001FD6110000031FCC34160002BD
S31A0003E0E20000000500001FA4110000011F9A31F000010000006B
S31A0003E0F70100001F72110000061F6634130001000000000C4A3F
S31A0003E10C1F4A110000071F3C31BA00040000539800001F1EFF03
S31A0003E1210000061F1431C60001000000000A2C1F02FF00000653
S31A0003E1361EF634140001000000000C2C1EDEFF0000031ED43115
S31A0003E14BEC00020000006400001EB8FF0000031EAE31EE00029F
S31A0003E1600000006400001E8EFF0000031E82341E00020000009B
S31A0003E1756400001E60FF0000011E5631C800010000000000003C
S31A0003E18A1E28FF0000011E1C34EC00010000000000001DF0FFCA
S31A0003E19F0000031DE831BE00020000006400001DB8FF0000032E
S31A0003E1B41DAA31DA00020000006400001D94110000031D86317C
S31A0003E1C9DC00020000006400001D72110000031D6231DE0002C3
S31A0003E1DE000000C800001D3E110000031D3431C00002000000A8
S31A0003E1F36400001D1C110000031D1231C20002000000C8000071
S31A0003E2081D1C110000031D0831C400020000012C00001D1C1118
S31A0003E21D0000051D0031CA000C0000000000001CDEFF000005BC
S31A0003E2321CD631E0000C0000000000001CA8FF0000051C9E3409
S31A0003E24702000C0000000000001C6CFF0000051C6233860010D8
S31A0003E25C0000000000001C30FF0000061C28346E00010000006C
S31A0003E271000C601C02020000051BFA3464000A00000000000047
S31A0003E2861BD0020000081BC633F6000200002F3E00001B9E0251
S31A0003E29B0000051B92355100200000000000001B70020000027E
S31A0003E2B01B6431C900010000004000001B52FF0000031B483193
S31A0003E2C5D600020000006400001B2CFF0000031B2433820002C0
S31A0003E2DA0000012C00001AFCFF0000031AF0345E000200000043
S31A0003E2EF0000001AC0040000031AB0339600020000073C000058
S31A0003E3041A84020000031A74339800020000070900001A500281
S31A0003E3190000031A42345A00020000001E00001A1E020000039C
S31A0003E32E1A0E345C000200000E10000019E40200000319D834D2
S31A0003E343E8000200000028000019AE0200000319A234EA000203
S31A0003E3580000000A00001980020000051976339A005000000051
S31A0003E36D000000194C02000005194234980050000000000000AF
S31A0003E38219120200000319083494000200002710000018DC0235
S31A0003E39700000318D23496000200000E10000018A602000005CC
S31A0003E3AC1898350C0024000000000000187A02000005186C35EC
S31A0003E3C1030009000000000000185002000005184633EA000C3C
S31A0003E3D6000000000000181A0200000518123488000A00000000
S31A0003E3EB00000017CA0200000617BE34700001000000000C7E27
S31A0003E40017840200000517783471000A000000000000172E02D7
S31A0003E4150000081720354C000200002F6300001B9E02000001D9
S31A0003E42A17103487000100000000000016F40200000116E434B6
S31A0003E43F6F000100000000000016C20200000316B63546000229
S31A0003E4540000000A0000168802000001167A3530000100000009
S31A0003E469000000165E02000006165A340E0001000000000A4A12
S31A0003E47E16480200000516403420000B000000000000161E0230
S31A0003E4930000051616342B000B00000000000015F402000001C4
S31A0003E4A815E8354E000100000000000015C60200000115BC34F2
S31A0003E4BD0F000100000000000015A802000005159A3436001440
S31A0003E4D2000000000000154C02000003153E34920002000000AB
S31A0003E4E7000000151402000001150A3410000100000000000087
S31A0003E4FC14EE0200000614E234120001000000000B1414D602B0
S31A0003E51100000614CC34110001000000000BB214BE0200000629
S31A0003E52614B034ED0001000000000C9E14780200000314683406
S31A0003E53BF000020000000A000014400200000314363578000274
S31A0003E5500000001E0000141A02000003141034EE000200000014
S31A0003E5650A000013E60200000513D4353100140000000000002D
S31A0003E57A13A802000001139A34F50001000000000000137A025F
S31A0003E58F000003137035000002000000960000135002000003B3
S31A0003E5A4134434F60002000008BD0000132C0200000313203565
S31A0003E5B9740002000000000000130E02000006130A354F000103
S31A0003E5CE000000000AB200000200000612FE35500001000000D5
S31A0003E5E3000C4000000200000612F035730001000000000C8689
S31A0003E5F812DA0200000112D23576000100000000000012BE02B4
S31A0003E60D0077656174686572206461746120746F2061737900D5
S31A0003E62277785F64756D700077686174206973207769726564EB
S31A0003E63720617420524E330000726E335F66756E6374696F6E05
S31A0003E64C00006D616E6970756C61746F72006C63640077696E83
S31A0003E661642076616E65206F6666736574000076616E656F6647
S31A0003E6766673657400007363616C652070756C73652F6D73650F
S31A0003E68B6320746F206D706800616E656D6F7363616C6500008E
S31A0003E6A07363616C6520412F4420746F2064656369562E2073B1
S31A0003E6B56565202762617474270000626174747363616C6500B1
S31A0003E6CA69676E6F726520554E4C4F434B2E20414E35206765C4
S31A0003E6DF6E6572696320412F44000066616974685F696E5F7027
S31A0003E6F46C6C000074656C656D65747279206D617070696E6749
S31A0003E7092E20352B382B4E2063686172732E206E6F20646566E8
S31A0003E71E61756C74000074656C656D657472795F666F726D61D8
S31A0003E7337400006B696C6F6D65746572732E2066617220617796
S31A0003E7486179207265706F727473206172652069676E6F7265AE
S31A0003E75D640000646967695F61726561007365636F6E64732E88
S31A0003E7722069676E6F7265206475706C69636174657300006433
S31A0003E7877570655F61676500007365636F6E64732E2077616920
S31A0003E79C74206F746865722052454C415920746F206163742091
S31A0003E7B16669727374000072656C61795F766973636F73697432
S31A0003E7C679006865736974616E742052454C4159206F72206E30
S31A0003E7DB6F726D616C20646967692E206D79616C696173205298
S31A0003E7F0454C4159207375676765737465640000747261636BE0
S31A0003E80565725F6469676900004D49432D452073746174757313
S31A0003E81A00006D69635F655F6D7367004D49432D45207061748D
S31A0003E82F6800006D69635F655F73736964000073656E64204D3D
S31A0003E84449432D4520666F726D6174746564207265706F727416
S31A0003E859007573655F6D69635F65006B696C6F6D6574657273B9
S31A0003E86E2E207265706F72747320666172206177617920617211
S31A0003E883652069676E6F7265640000776179706F696E745F61CF
S31A0003E89872656100626C616E6B207365706172617465642070B9
S31A0003E8AD72656669786573207065656C65642066726F6D20775D
S31A0003E8C27074206E616D65732E202D6C206C63617365202D6163
S31A0003E8D72061732D6973202D46206865785F7373696400776144
S31A0003E8EC79706F696E745F74696479007265706F7274732074AF
S31A0003E9016F20677073207770747300776179706F696E74730043
S31A0003E91672656C617920736F6D652073656E74656E63657320EA
S31A0003E92B6261636B20746F2061737900006E6D65615F7265678F
S31A0003E940656E000064656661756C74206C6F6E67697475646516
S31A0003E9552E206C696B6520323830362E32312C45006770735F16
S31A0003E96A6C6F6E0064656661756C74206C617469747564652EB7
S31A0003E97F206C696B6520363130332E35322C4E00006770735F13
S31A0003E9946C61740074797065206F662067707320757365640032
S31A0003E9A900677073007265706F727420616C74697475646520CE
S31A0003E9BE696620706F737369626C650073656E645F616C746938
S31A0003E9D374756465006B696C6F6D65746572732E20696E20737D
S31A0003E9E8746174696F6E61727920636F6D7072657373656420C1
S31A0003E9FD7265706F7274730000726164696F5F72616E67650072
S31A0003EA1262617365393120636F6D7072657373696F6E20776810
S31A0003EA27656E20706F737369626C6500007573655F636F6D7022
S31A0003EA3C72657373696F6E0073686F77206163746976652047F5
S31A0003EA516F746F20696E207265706F727400007461726765741B
S31A0003EA665F636F6D6D656E7400007461726765745F73796D629F
S31A0003EA7B6F6C006F626A6563742F6974656D206E616D65206FFD
S31A0003EA90662047505320476F546F2E202A206D65616E73207023
S31A0003EAA5757420756E697175652064696769742E2064656661A4
S31A0003EABA756C743D7770745F6E616D6500007461726765745F6B
S31A0003EACF6E616D650069732074686520746172676574206F62B3
S31A0003EAE46A656374206F72206974656D203F206E6F6E653D64CE
S31A0003EAF9697361626C6520746172676574207265706F7274002C
S31A0003EB0E7461726765745F7479706500726571756972656420C0
S31A0003EB2364657374696E6174696F6E20696E20696E636F6D699C
S31A0003EB386E67207061636B6574732E202A20616E64203F20771E
S31A0003EB4D696C6463617264732E2064656661756C743D2A0000CA
S31A0003EB62616C746E6574000064657374696E6174696F6E206FDC
S31A0003EB77662061707273207265706F7274732C206465666175C4
S31A0003EB8C6C7420415052532D3000617072735F64737400006117
S31A0003EBA17070656E64656420746F206E6F726D616C2072657063
S31A0003EBB66F727473000073686F72745F636F6D6D656E74006196
S31A0003EBCB7070656E64656420746F206C6F6E677061746820723A
S31A0003EBE065706F72747300006C6F6E675F636F6D6D656E740078
S31A0003EBF5007365636F6E6473206265747765656E206C6F6E6739
S31A0003EC0A70617468207265706F7274732E20303D646973616252
S31A0003EC1F6C65006C6F6E675F74696D65006D6574657273206236
S31A0003EC3465747765656E206C6F6E6770617468207265706F7275
S31A0003EC4974732E20303D64697361626C6500006C6F6E675F61C7
S31A0003EC5E72656100666172207265616368696E672074726163FC
S31A0003EC736B65722064696769706174682E20626C616E6B2073EE
S31A0003EC88657061726174656400006C6F6E677061746800006E5D
S31A0003EC9D6F726D616C20747261636B6572206469676970617430
S31A0003ECB2682E20626C616E6B2073657061726174656400006449
S31A0003ECC769676970617468000073696465776179732061636399
S31A0003ECDC656C65726174696F6E206166746572207475726E003C
S31A0003ECF100747261636B5F6C6F7767000073696465776179736F
S31A0003ED0620616363656C65726174696F6E20696E207475726E05
S31A0003ED1B2E20303D64697361626C650000747261636B5F686906
S31A0003ED30676867006B6DB02F6820666163746F72206F66204379
S31A0003ED456F726E657250656767696E672E20303D64697361620B
S31A0003ED5A6C650000747261636B5F7475726E736C6F70650073F7
S31A0003ED6F65636F6E6473206265747765656E207265706F727444
S31A0003ED84732C206174206D696E696D756D00747261636B5F6CE1
S31A0003ED99696D69746572007365636F6E64732062657477656547
S31A0003EDAE6E207265706F7274732E20303D64697361626C65001B
S31A0003EDC300747261636B5F696E74657276616C00006D657465AE
S31A0003EDD872732074726176656C6C6564206265747765656E202B
S31A0003EDED7265706F7274732E20303D64697361626C6500747284
S31A0003EE0261636B5F64697374616E6365000027746F6B656E20B1
S31A0003EE1772696E67272E20302064697361626C652E20312D31B7
S31A0003EE2C35207365747320616C736F20706F72746E756D006B45
S31A0003EE416973735F747269636B00006279746573202861707038
S31A0003EE56726F78292E206C696D697420612073696E676C65206C
S31A0003EE6B6B6579646F776E000074786C696D6974006D736563D5
S31A0003EE802E206368616E6E656C206163636573732074696D69E8
S31A0003EE956E6700736C6F7474696D6500003020706F6C6974653C
S31A0003EEAA2C20323535207069670070657273697374656E63655D
S31A0003EEBF0062756C6C6574696E2067726F7570732C20626C619B
S31A0003EED46E6B20736570617261746564000062756C6C67726F77
S31A0003EEE97570730000322063686172616374657273206F722020
S31A0003EEFE6E616D652E207472792068656C702073796D626F6C29
S31A0003EF137300006D7973796D626F6C00006F626A6563742F69E2
S31A0003EF2874656D206E616D652E20412D5A20302D39206F6E6C8F
S31A0003EF3D792073756767657374656400006D796E616D650000CB
S31A0003EF5277686174206B696E64206F6620616E696D616C204937
S31A0003EF6720616D2E20736565206D796E616D6500006D79747999
S31A0003EF7C7065000070617373776F726420666F722072656D6FF5
S31A0003EF917465206366672E20756E69717565206D7963616C6CB2
S31A0003EFA6207375676765737465640000726670617373776400F8
S31A0003EFBB006B696E64206F662061646D696E20616C6961732C1E
S31A0003EFD020666F722072656D6F7465206366672E2073736964BF
S31A0003EFE520757361626C6500006D79646F6D61696E0000616C47
S31A0003EFFA69617320666F7220646967697065617465722C206C5F
S31A0003F00F696B652052454C41592E207373696420757361626CD5
S31A0003F02465006D79616C6961730063616C6C7369676E20616E3D
S31A0003F0396420737369642C206C696B65204F486E4142432D6E0B
S31A0003F04E00006D7963616C6C0000727373695F336C6564007228
S31A0003F0637373695F326C6564007369676E616C20737472656EB0
S31A0003F07867746820746F206C65647300727373695F316C6564E6
S31A0003F08D006E6F2068616E672064656C61792069662072737334
S31A0003F0A26920776173206F766572207468697300737175656C9E
S31A0003F0B763685F62696C6576656C006D736563206F66206861A8
S31A0003F0CC6E672064656C61790000737175656C63685F74616990
S31A0003F0E16C00006D736563206F66206F70656E696E672064650F
S31A0003F0F66C617900737175656C63685F64656C617900737175FA
S31A0003F10B656C6368206F70656E2F636C6F7365206C6576656CFB
S31A0003F1202E207365652072737369207769746820277374617486
S31A0003F135270000737175656C63680075736520736F667477619F
S31A0003F14A7265206861636B20666F72206463642E206E6F7420A8
S31A0003F15F42555359206F722052535349007573655F736F667485
S31A0003F17464636400757365204255535920696E70757420666F5D
S31A0003F189722064636420616E6420737175656C63682E206E6F18
S31A0003F19E74205253534900007573655F6275737900006D7365CA
S31A0003F1B3637320746F2077616974206265666F72652073656E97
S31A0003F1C864696E67206166736B00646174615F64656C617900BA
S31A0003F1DD006D7365637320746F207761697420666F7220706FBB
S31A0003F1F277657220746F2072697365007077725F64656C617914
S31A0003F207006D7365637320746F207761697420666F7220504CD3
S31A0003F21C4C206C6F636B0000706C6C5F64656C6179004D495320
S31A0003F2314F206E65656473202B355644442070756C6C75700021
S31A0003F2467074745F6F726967696E00007472616E736D69747485
S31A0003F25B657220706F7765720074785F706F77657200006E6F1C
S31A0003F270726D616C6C792032313430302F326D2C2034343930ED
S31A0003F285302F554846000072785F69665F6F666673657400002B
S31A0003F29A7061636B65742073656E7420616674657220766F6964
S31A0003F2AF636520707474007074745F7061636B657400006175FC
S31A0003F2C4746F6D617469632031373530487A206275727374201C
S31A0003F2D96966206475706C65782D766F69636500006175746F9A
S31A0003F2EE6265657000007365636F6E647320746F206C696E67AA
S31A0003F3036572206265666F726520726573756D696E6720736302
S31A0003F318616E00007363616E5F7461696C007365636F6E64736B
S31A0003F32D2066726F6D207074742F737175656C636820746F202F
S31A0003F3426175746F7363616E000069646C655F74696D6500762D
S31A0003F3576F69636520702E207363616E73206368616E6E656C09
S31A0003F36C73207768656E2069646C65006175746F7363616E0022
S31A0003F3810064656369487A2C206C696B652031313838203D20B7
S31A0003F3963131382E382E20303D6F666600006374637373002B18
S31A0003F3AB31327620696E2052545331206F766572726964657337
S31A0003F3C0206C6F636B6F7574000074785F6C6F636B6F757400C2
S31A0003F3D500303D73696D706C65782C207365652027667265712D
S31A0003F3EA270074785F66726571007278206672657175656E6382
S31A0003F3FF792C20747820746F6F2069662074785F667265713D88
S31A0003F4143000667265710000656E67696E65206D6F6E69746FD0
S31A0003F429722E207769726520312F33206F66202B564220746FC0
S31A0003F43E20414E3700006C6F626174740000677073206F7220D9
S31A0003F4536B69737320617474616368656420746F2073657269AD
S31A0003F468616C2031206F722032006170705F706F727400007040
S31A0003F47D61757365206C6F6E67206C697374696E67732E2030E8
S31A0003F4923D756E6C696D6974656400007474796C696E657300D8
S31A0003F4A700303A203139323030206F7220616E7920706572737E
S31A0003F4BC6F6E616C69747920737065636966696320646566611C
S31A0003F4D1756C74000074747962617564006D79206D69737369A0
S31A0003F4E66F6E0000706572736F6E616C697479006E616D6520B0
S31A0003F4FB6F66207468697320736574206F6620706172616D654F
S31A0003F51074657273000070726F66696C655F7461670000014151
S31A0003F525505A4D445200000000000A0014001E00280032003C69
S31A0003F53A00467478715F656E74657200696C6C6567616C004772
S31A0003F54F50524D432C68686D6D73732C412C6C6174692E747556
S31A0003F564642C6E2C6C6F6E67692E7475642C652C7370642C6338
S31A0003F57973652C64646D6D79792C2C000047494D4D45004E07C0
S31A0003F58E5F704750524D432C00004750524D422C000047504769
S31A0003F5A347412C0000000347E52F413D00202D3E00205154501A
S31A0003F5B800002051544F0000065948C5032CA4620001DA1C5039
S31A0003F5CD4D474E57504C00475057504C00206D0000206B6D003C
S31A0003F5E266617200636C6F73650020202020202020202020205C
S31A0003F5F72000002852A28550A5450A686F6C64710072656C6135
S31A0003F60C793A2000646967693A20000052454C415900574944B5
S31A0003F62145000054524143450053656E64206E6F770000506564
S31A0003F6366E64696E6700436C65617200436C65617265640054BB
S31A0003F64B7261636B004E6F6E6500004D61726B00004D61726B5A
S31A0003F6602073657400004E6F20616374696F6E000000001600AF
S31A0003F6753C008600D400D400D400D400D4000800D400D400D40D
S31A0003F68A00D400D400D400D400D400D4001E00D400D400D400D0
S31A0003F69FD400D400D400D400D400D40064004400D400D400D431
S31A0003F6B400D400D400D400D400D4008C20202020202020202068
S31A0003F6C9003A61636B00002D30000051535400414C4C004351F8
S31A0003F6DE0000424C4E003F415052533F0000B0200000206D2FF2
S31A0003F6F3732C20670020002C2073756D3D000023DA23D623D4E8
S31A0003F70823D023CE23CA23C823C423DA4E57000057005357009D
S31A0003F71D0053005345000045004E4500004E00206B6D6820003D
S31A0003F7324C6F636174696F6E20756E6B6E6F776E0000494400C3
S31A0003F7470074785F6C6F636B6F757432005363616E000076F833
S31A0003F75C3A200000706F737369626C65206F7074696F6E7300A8
S31A0003F7710020616E6420002C200000656D707479206368616ED2
S31A0003F7866E656C0073696D706C6578002D002B000A0D00002293
S31A0003F79B00222C207479706520756E6B6E6F776E006F6E000013
S31A0003F7B0626F6F6C2073697A65002C206E616D6520756E6B6EEB
S31A0003F7C56F776E00007461622073697A650000494E56414C49FD
S31A0003F7DA44000024005400640072001C008C0072012420686157
S31A0003F7EF7320756E6B6E6F776E20747970652C20756E61737301
S31A0003F80469676E61626C650A0D00706F737369626C65206F709D
S31A0003F81974696F6E733A206F66662F6F6E0A0D00006E6F74207B
S31A0003F82E612076616C69642073796D626F6C2C20747279206842
S31A0003F843656C702073796D626F6C730000004400AC00C600DAAD
S31A0003F858001A010A00DA01A042757379200020525353492000AE
S31A0003F86D002044545232200000204D49534F2000002053434BA8
S31A0003F882200020496E707574732000002042617474200000209A
S31A0003F8974C6F636B656420200020556E6C6F636B656400657295
S31A0003F8AC6173652000002D207369626C696E673F202D2000778D
S31A0003F8C172697465200000636F6D706172652000004F4B0A0D9D
S31A0003F8D60000206661696C65640A0D002D4D6F72652D00000D7E
S31A0003F8EB202020202020200D003A00746F6F206C6F6E67206135
S31A0003F9006464726573732C20736F7272790A0D002024200070EE
S31A0003F915617373776F72643A200000656E74657220636F6D6D8D
S31A0003F92A616E64732C20657869742077697468205E440A0D005E
S31A0003F93F00746F6F206C6F6E6720636F6D6D616E642C20736F5B
S31A0003F9547272790A0D006E6F20726573706F6E73650A0D00722C
S31A0003F96965626F6F74000072657374617274006E6F700076653A
S31A0003F97E7273696F6E007770745F73746173680064656275675C
S31A0003F993006261747400007065656B000065657065656B000097
S31A0003F9A8726567697374657200004600737461636B7300007796
S31A0003F9BD616C6C636C6F636B0070726F66696C65006E6F207386
S31A0003F9D27563682070726F66696C65206E756D6265720A0D0006
S31A0003F9E700202200002C2077697468206E6F206E616D652C00CE
S31A0003F9FC2069732063757272656E742070726F66696C6500704D
S31A0003FA1165726D0000646973700000666163746F7279646566BC
S31A0003FA2661756C747300796F752070726F6261626C79207761C9
S31A0003FA3B6E7420746F20646F205045524D206E6F770A0D0000F6
S31A0003FA507374617400000D006368616E6E656C006368616E6EEE
S31A0003FA65656C207461626C6520697320656D7074790A0D000028
S31A0003FA7A6E6F7420736F206D616E79206368616E6E656C730AD0
S31A0003FA8F0D000072656D6F746500006E65656420746865206340
S31A0003FAA4616C6C7369676E206F66207468652072656D6F746558
S31A0003FAB9207365740A0D0074656C656D657472790073656E6427
S31A0003FACE6E6F770068656C70000073796D626F6C730072616ED3
S31A0003FAE367653A2030202E2E2E203235350A0D000072616E678A
S31A0003FAF8653A2030202E2E2E2036353533350A0D00006D6178D2
S31A0003FB0D20000020636861726163746572730A0D006E6F2068FE
S31A0003FB22656C7020666F72202200222C20736F7272790A0D0017
S31A0003FB370041535452414C00000D0A41535452414C0D0A0000F4
S31A0003FB4C736574006E6F207375636820706172616D65746572BE
S31A0003FB61202200000C00120018003A001E0000000200010002B1
S31A0003FB76000407D05E430A0D0000656F660A0D00082008000A53
S31A0003FB8B0D0A0D536F6D6520706172616D657465727320686167
S31A0003FBA076652064656661756C7465642E205472792068656CB8
S31A0003FBB5702E0A0D566572696679206D7973796D626F6C2061EB
S31A0003FBCA6E64207461726765745F73796D626F6C2E0A0D0A0D53
S31A0003FBDF0068616D6472202420000022203F0A0D0000120000EE
S30B0003FBF40006000C001CD4
S3150003FBFA2326303E41575E5F6163696E7375767A73
S31A0003FC0A000100020004000800100020004000800100020004D6
S31A0003FC1F000800100020004000800001020408102040800A0DB9
S31A0003FC34646F683A2000303132333435363738394142434445C1
S3100003FC494600000A0D00005C78000076
S31A0003FC5481020101000100010001010100010001000100010004
S31A0003FC690112C008CCF63310AAAAAA0012000000000000001479
S31A0003FC7E00000000000A000A001E00280D0A41535452414C0D23
S31A0003FC930A00000D0A4541525448410D0A00000000000A00104C
S30D0003FCA800240042003800426B
S31A0003FCB0000000000094009400940094009400160040005E207E
S31A0003FCC56869676800206C6F7700002070756C6C646F776E007A
S31A0003FCDA20616374697669747900200020B043003A003B0020B7
S31A0003FCEF30780000000000000E001800580068009800D200FE01
S31A0003FD04011E3234303100003234303500003138323000003233
S31A0003FD19343037000032343336000032343233000032343039C8
S31A0003FD2E0000323435300000313832320000323433380000311D
S31A0003FD43384232300032343038000032343133000020746F6FBC
S31A0003FD58206D616E790020697320756E6B6E6F776E000801087B
S31A0003FD6D010801080100000000000C001800240030003C004869
S3090003FD8200540060C0
S31A0003FD86A674A6A4000000060011000B002700220017001C005D
S31A0003FD9B54004F00440049002D0033003E003800AE00A9009E4F
S31A0003FDB000A30087008D00980092005A0060006B006500810049
S31A0003FDC57C007100760162015D01520157013B0141014C01463F
S31A0003FDDA010E0114011F0119013501300125012A00B400BA0087
S31A0003FDEFC500BF00DB00D600CB00D00108010300F800FD00E143
S31A0003FE0400E700F200EC77782000B0202000206B6D2F6820204D
S31A0003FE1900B043202000002500000102030405060708090A0B31
S31A0003FE2E0C0D0E0F10111213141516171818191A1B1C1D1D1EF2
S31A0003FE431F2020212223232425252627272829292A2A2B2B2C87
S3090003FE582C2DFF0045
S31A0003FE5C0000004000140054010A0400000000000000000006CB
S3180003FE71090F0F00080C0E0F0B090804000E010F110F00BF
S70500030000F7
